:020000040800F2
:10000000707F0020E1220208C5EA0108C7EA010862
:10001000C9EA0108CBEA0108CDEA010800000000A6
:10002000000000000000000000000000D1EA01080C
:10003000CFEA010800000000D3EA0108D5EA010870
:10004000D9EA0108DBEA0108DDEA0108DFEA010874
:10005000EFEB0108F1EB0108F3EB01087BEC010881
:100060000BED01080DED01080FED010891EE0108FF
:1000700093EE010895EE010897EE010899EE01084C
:100080009BEE01089DEE01089FEE0108A1EE01081C
:10009000A3EE0108E5EF0108E7EF0108E9EF010829
:1000A00071F6010873F6010875F6010877F6010884
:1000B00079F601087BF6010861F70108E5F8010807
:1000C000E7F80108E9F80108EBF80108EDF8010884
:1000D000EFF80108F1F80108F3F80108F5F8010854
:1000E000EFF90108F1F90108F3F90108F5F9010840
:1000F000F7F90108F9F90108FBF9010887FA010885
:1001000089FA01088BFA01088DFA010825FB01081C
:1001100027FB010829FB01082BFB01082DFB010827
:100120002FFB010831FB010833FB010835FB0108F7
:1001300000F002F800F05AF80AA090E8000C82449F
:100140008344AAF10107DA4501D100F04FF8AFF27C
:10015000090EBAE80F0013F0010F18BFFB1A43F0A5
:1001600001031847642D0200842D02000A444FF059
:10017000000C10F8013B13F0070408BF10F8014B06
:100180001D1108BF10F8015B641E05D010F8016B4B
:10019000641E01F8016BF9D113F0080F1EBF10F8AF
:1001A000014BAD1C0C1B09D16D1E58BF01F801CBD2
:1001B000FAD505E014F8016B01F8016B6D1EF9D555
:1001C0009142D6D37047000000230024002500266A
:1001D000103A28BF78C1FBD8520728BF30C148BFAA
:1001E0000B6070471FB51FBD10B510BD22F04FFA50
:1001F0001146FFF7F7FF1AF0B0FD22F06DFA03B4D5
:10020000FFF7F2FF03BC22F071FA000070B5FC4D5D
:10021000FF22134605F5807606E000BF10F8014B7B
:1002200054402A5D5A40335D491EF7D243EA02200A
:1002300070BD2DE9F04FF34CF34FDFF8D0936078A9
:10024000002689B041F26F7A4FF4FA5BA4F2DD2503
:10025000062830D1A078E178224601EB0020117900
:100260005279504502EB012109B201D827F810104C
:10027000584503D3A0F5FA6027F81010AE7085F842
:10028000266000204A46235C95F82610401CC0B228
:100290005354491C85F826100728F4D9012240F24E
:1002A0002771DB4821F040FE00202654401CC0B2DC
:1002B0000A28FAD92E716078032801D0042871D158
:1002C00021788DF800108DF80100627950008DF8CA
:1002D0000200A078E17801EB002E002028E000BFAA
:1002E0000EEB000151450ED837F911804FEAE87343
:1002F00008EB13634FEA132C6B4603EB400383F8C0
:1003000003C083F80480594510D307EB4101A1F5E0
:100310008051B1F96010CB1701EB13634FEA132C36
:100320006B4603EB400383F803C01971401CC0B255
:100330008242D5D89DF802106846C91CFFF766FFB7
:10034000B449C0F3072288629DF802300DF1030121
:100350005A549DF8022001A95054AE7085F82660C9
:100360009DF802100020E846091D4B460BE000BF37
:1003700095F8262018F800C003F802C0521C401C53
:1003800085F82620C0B28142F2D2012240F22771C4
:100390009F4821F0C9FD00202654401CC0B20A2805
:1003A000FAD92E716078102845D1A078E17801EB58
:1003B0000020504505D8E179227A02EB012127F887
:1003C0001010584509D3E27907EB40011002227A58
:1003D000A1F580511044A1F86000AE7085F8266048
:1003E00000204F46225C95F82610401CC0B27A547B
:1003F000491C85F826100628F4D306218148FFF70A
:1004000005FF8449C0F30722886295F826107A54C4
:10041000491CC9B201227854491C85F8261040F2C3
:1004200027717B4821F080FD00202654401CC0B27B
:100430000A28FAD92E7109B0BDE8F08F7649084430
:1004400074498039886100787047744A00211154DA
:100450007047724A01211154704770490A5C12B109
:1004600000220A5470470122FBE76C49A13131F8A0
:100470001000002800D001207047392801D83038FA
:10048000C0B2412801D33738C0B27047392803D8E9
:10049000302801D3303804E0462804D8412802D35C
:1004A0003738C0B2704700207047092801D8303073
:1004B00004E00F2804D80A2802D33730C0B27047AE
:1004C0000020704710B5564C20461FF0F3FF5649E8
:1004D00054480022086001F5CE7048601020886002
:1004E0005248B0F87200C1E903028020C1E9050258
:1004F0004FF44050CA61C1E908208A62204620F0CA
:100500003DF82046BDE81040012120F061B8B0F56B
:10051000C06F02D24649085C704746490844A0F5BE
:10052000005090F8C00070472DE9F05F414D0C4637
:100530000646B0F5C06F02D23D48845504E0A819C4
:10054000A0F5005080F8C040DFF8E0B0DFF8D880B8
:100550000BF18009BBF86600A8F1480801283CD1DE
:10056000B9F8041042F208020A44964235D16818DC
:1005700090F8C80008B114B12FE0012C2DD14FF034
:10058000804A5046BAF8247020F0A4FF01210846A2
:1005900020F08FFE4FF6FF71A8F804100021A8F894
:1005A0000010A8F80610B9F804202A4492F8C820D0
:1005B00002B11021A8F802101B495046483920F01A
:1005C000DEFF00231A461946504621F031FA504604
:1005D000AAF82470012121F0BFF99BF8130001282B
:1005E0000BD1B9F8081042F208020A44964204D12D
:1005F000681890F8C80010B104B3BDE8F09F1BE084
:10060000A82C0208DD0200202C2D0020DB07002092
:10061000004800400001002000C0030871100020C5
:1006200044000240043801400C0400200000002077
:100630005212002052180020012CDED1FA4E3488CC
:10064000F94F243F384620F045FF0121C80220F031
:1006500027FE4FF6FF71A8F804100021A8F800103B
:10066000A8F80610B9F808202A4492F8C82002B168
:100670001021A8F80210ED49384620F080FF002331
:100680001A461946384621F0D3F934803846BDE879
:10069000F05F012121F060B92DE9F04F1344E44AE5
:1006A000E44E9F18A6F53064BB7A0022012540F283
:1006B000E53BA6F6E14940F2FD5E04F5C06A8842DA
:1006C00025DD97F80CC0BCF1000F21D0BCF1010F63
:1006D00022D0BCF1020F22D0BCF1030F22D0BCF11A
:1006E000050F26D0BCF1080F30D0BCF1090F35D072
:1006F000BCF10A0F3BD0BCF10B0F41D0BCF10C0F89
:1007000047D0BCF10D0F4DD0BCF10F0F57D05DE0BD
:10071000F55406EB030C1CE006EB030C20E006EBA3
:10072000030C26E003F5407CDC454FD806EB030CB8
:1007300028E04C2B4AD803F1010809F8035009F8C6
:10074000082003F1020809F808203FE0E55404EB13
:10075000030C8CF801208CF8022037E004EB030C2A
:100760008CF800518CF801218CF802212EE004EB6A
:10077000030C8CF800528CF801228CF8022225E040
:1007800004EB030C8CF800538CF801238CF8022343
:100790001CE004EB030C8CF800548CF801248CF85A
:1007A000022413E003F5A06CF4450FD804EB030C0E
:1007B0008CF800558CF801258CF8022506E0FD2BFD
:1007C00004D80AF803500AEB030CC2E7884225D18B
:1007D00097F80CC0BCF1000F21D0BCF1010F22D062
:1007E000BCF1020F22D0BCF1030F22D0BCF1050FE7
:1007F00026D0BCF1080F30D0BCF1090F35D0BCF1C8
:100800000A0F3BD0BCF10B0F41D0BCF10C0F47D00D
:10081000BCF10D0F4DD0BCF10F0F57D05DE0F2547D
:1008200006EB030C1CE006EB030C20E006EB030CCC
:1008300026E003F5407CDC454FD806EB030C28E0AE
:100840004C2B4AD803F1010809F8032009F8085095
:1008500003F1020809F808203FE0E25404EB030C1E
:100860008CF801508CF8022037E004EB030C8CF874
:1008700000218CF801518CF802212EE004EB030CCE
:100880008CF800228CF801528CF8022225E004EB4F
:10089000030C8CF800238CF801538CF802231CE025
:1008A00004EB030C8CF800248CF801548CF802241F
:1008B00013E003F5A06CF4450FD804EB030C8CF89F
:1008C00000258CF801558CF8022506E0FD2B04D894
:1008D0000AF803200AEB030CC2E788421FDA387BD0
:1008E000F0B101281FD002281FD003281FD00528EF
:1008F00023D008282CD009282DD00A282FD00B2847
:1009000031D00C2833D00D2836D00F2807D1FD2B3D
:1009100005D80AF803200AEB0300427085708BE5C6
:10092000F254F018F9E7F01816E0F01818E003F5A3
:1009300040705845F3D8F01816E04C2BEFD809F862
:100940000320591C9B1C09F8012009F8035073E58A
:10095000E254E018E1E7E01800F580700AE0E018E2
:1009600000F5007006E0E01800F5407002E0E018C5
:1009700000F580600270D0E703F5A0607045CED826
:10098000E01800F5A060F5E72DE9FF4F86460D98C9
:10099000284D19182648A5F530630F180020B97B9B
:1009A000012440F2E53AA5F6E14640F2FD5B03F58D
:1009B000C069964525DD97F810C0BCF1000F21D025
:1009C000BCF1010F22D0BCF1020F22D0BCF1030F09
:1009D00022D0BCF1050F2FD0BCF1080F38D0BCF1EC
:1009E000090F3DD0BCF10A0F43D0BCF10B0F49D029
:1009F000BCF10C0F4FD0BCF10D0F55D0BCF10F0F57
:100A00005FD065E06C5405EB010C24E005EB010CB4
:100A100028E005EB010C2EE001F5407CD44557D8C9
:100A200005EB010C30E00000242C0140C403002041
:100A300000C00308521D00204C2949D801F1010CC7
:100A4000745406F80C0001F1020C06F80C003FE0AB
:100A50005C5403EB010C8CF801008CF8020037E0C9
:100A600003EB010C8CF800418CF801018CF80201B9
:100A70002EE003EB010C8CF800428CF801028CF89C
:100A8000020225E003EB010C8CF800438CF8010313
:100A90008CF802031CE003EB010C8CF800448CF88A
:100AA00001048CF8020413E001F5A06CDC450FD8BA
:100AB00003EB010C8CF800458CF801058CF802055D
:100AC00006E0FD2904D809F8014009EB010CC2E752
:100AD000964529DCDDF804C0624525DC97F810C096
:100AE000BCF1000F21D0BCF1010F22D0BCF1020FEC
:100AF00022D0BCF1030F22D0BCF1050F26D0BCF1EF
:100B0000080F2FD0BCF1090F34D0BCF10A0F3AD036
:100B1000BCF10B0F40D0BCF10C0F46D0BCF10D0F57
:100B20004CD0BCF10F0F56D05CE0685405EB010CC3
:100B30001BE005EB010C1FE005EB010C25E001F5C6
:100B4000407CD4454ED805EB010C27E04C2949D810
:100B500001F1010C705406F80C4001F1020C06F88A
:100B60000C003FE0585403EB010C8CF801408CF86A
:100B7000020037E003EB010C8CF800018CF8014116
:100B80008CF802012EE003EB010C8CF800028CF8CB
:100B900001428CF8020225E003EB010C8CF8000303
:100BA0008CF801438CF802031CE003EB010C8CF879
:100BB00000048CF801448CF8020413E001F5A06CE9
:100BC000DC450FD803EB010C8CF800058CF80145CF
:100BD0008CF8020506E0FD2904D809F8010009EBAC
:100BE000010CC2E7DDF804C094451EDA3A7CF2B18C
:100BF000012A1FD0022A1FD0032A1FD0052A23D082
:100C0000082A29D0092A2AD00A2A2CD00B2A2ED029
:100C10000C2A30D00D2A33D00F2A06D1FD2904D852
:100C200009F80100494448708C70BDE8FF8F685492
:100C30002944F8E7294413E0294415E001F54072FE
:100C40005245F2D8294413E04C29EED870544A1C7E
:100C5000891CB0547454E8E758541944E3E7194424
:100C600001F580710AE0194401F5007106E01944AC
:100C700001F5407102E0194401F580610870D2E786
:100C800001F5A0625A45D0D8194401F5A061F5E7F5
:100C900000207047FE49082802D8421E81F84620ED
:100CA000092805D3102803D8A0F1090281F84620AD
:100CB000112805D3182803D8A0F1110281F8462085
:100CC000192805D3202803D8A0F1190281F846205D
:100CD000212805D3282803D8A0F1210281F8462035
:100CE000292805D3302803D8A0F1290281F846200D
:100CF000312805D3382803D8A0F1310281F84620E5
:100D0000392805D3402803D8A0F1390281F84620BC
:100D1000412805D3482803D8A0F1410281F8462094
:100D2000492805D3502803D8A0F1490281F846206C
:100D3000512805D3582803D8A0F1510281F8462044
:100D4000592805D3602803D8A0F1590281F846201C
:100D5000612804D3682802D8613881F846007047BA
:100D6000CB4991F8452091F846309A40082804D89C
:100D700091F83830134481F83830092806D3102808
:100D800004D891F83930134481F83930112806D34A
:100D9000182804D891F83A30134481F83A301928C9
:100DA00006D3202804D891F83B30134481F83B3017
:100DB000212806D3282804D891F83C30134481F820
:100DC0003C30292806D3302804D891F83D3013440C
:100DD00081F83D30312806D3382804D891F83E30C8
:100DE000134481F83E30392806D3402804D891F8BE
:100DF0003F30134481F83F30412806D3482804D8B7
:100E000091F84030134481F84030492806D35028E7
:100E100004D891F84130134481F84130512806D369
:100E2000582804D891F84230134481F842305928A8
:100E300006D3602804D891F84330134481F8433036
:100E4000612805D3682803D811F8440F10440870AE
:100E500070472DE9F05F8F49042048618E48DFF824
:100E600030A2DFF838E290F80180057A447A837A7C
:100E7000C17990F802C090F80390077946799AF802
:100E8000052080790EF29D1BB8F1310F03D0B8F127
:100E9000300F7CD0D8E0DFF80082BCF1310F12D1E6
:100EA000B9F1300F0FD1312F0DD1342E0BD13028A5
:100EB00009D14046322990F80BC0077B467B807BE6
:100EC00002D0412937D0BFE0302D7DD1312C7BD1EC
:100ED000302B79D1BCF1300F76D1032F74D1312E64
:100EE00072D1442870D1002150468AF801100621A1
:100EF0008BF800100121012A5B468AF825104FF07B
:100F000000020AD0664C9D5CA554521C012AFAD9F5
:100F1000427882708AF82610D1E074469D5CA55410
:100F2000B0F87250521C6D1CA0F872508A42F5D372
:100F3000FFF7C8FAC9E0302D46D1302C44D1302B10
:100F400042D1BCF1300F7FD1382F7DD1302E7BD1F3
:100F5000302879D198F80F00302875D198F8100012
:100F6000302871D198F8110030286DD198F812000E
:100F7000302869D198F81300302865D198F814000A
:100F8000302861D198F8150030285DD100E047E0A5
:100F900098F81600302857D198F81700302853D108
:100FA00098F8180030284FD198F8190030284BD104
:100FB00098F81A00302847D198F81B00302843D100
:100FC00098F81C00032800E03EE03DD198F81D0091
:100FD000332839D198F81E00332835D100215046E6
:100FE0008AF8011006218BF800100121012A5B46C6
:100FF0008AF825104FF0000206D0294C9D5CA554BC
:10100000521C012AFAD983E775469C5CAC54B0F8AF
:101010007240521C641CA0F872408A42F5D387E7E4
:10102000BCF1300F10D1B9F1450F0DD1302F0BD1DC
:10103000322E09D1302807D1322905D1032D03D111
:10104000362C01D1432B03D01249042008613CE027
:10105000002051468AF8010002238BF80030362325
:101060008BF8013032248BF802408BF803308BF878
:10107000043003248BF8054044238BF806303723D3
:101080008BF807300823584681F82530012A09E0FB
:10109000000000200010014014020020A8050020DC
:1010A000DB0700204FF0000212D0F84C855CA554FD
:1010B000521C0A2AFAD9487888708AF82630012208
:1010C00040F22771F24820F02FFF0020BDE8F09F8A
:1010D0007446855CA554B1F87250521C6D1CA1F881
:1010E00072509A42F5D323E7EA4830B4816A0A0A7B
:1010F000524201EB0222C2F30711826213095B42E2
:10110000A0F5807001F00F0102EB031280F82B10A4
:1011100002F00F0280F82C20092901D8303100E0BC
:10112000373180F82B10092A01D8303200E03732ED
:1011300080F82C20D54A10F8251F963A03235354E3
:10114000491CC9B283795354491CC9B2C379535459
:10115000491CCBB2037010F8201C253801294FF030
:10116000000111D0C94C555C6554491CC9B28C2989
:10117000F9D94178817080F8263030BC012240F2E4
:101180002771C34820F0D0BEC34D08E0545C6C54B6
:10119000B0F87240641C491CA0F87240C9B2994270
:1011A000F4D330BCFFF78EB92DE9F04F97B0002093
:1011B000BA49059004204861B9480024407811904C
:1011C000452843F06180B648DFF8C0920346857831
:1011D000187BA3F5057B00909BF805000E901E7A06
:1011E00093F80AA093F803E0997993F809C0DA79A3
:1011F000D87A129058791B79A9F19609302D32D0FE
:10120000DFF89C82312D98F80D70169798F81270BF
:10121000159798F80E70139798F80F807AD0A04F12
:10122000302D78D0312D77D0372D76D0382D75D020
:10123000372D74D0382D73D0372D72D0382D71D012
:10124000372D70D0382D6FD0312D6ED0302D6DD020
:10125000312D02F0D980302D02F00881312D02F0BD
:10126000E78703F011B8BEF1300FFAD1302B7DD1F2
:10127000452842F00A81312942F07283342AFBD199
:10128000302EEED1BCF1360F42F06C83BAF1030F71
:10129000E7D112984528E4D100983828E1D10BF124
:1012A000380500272C706C70AC70EC702C716C7170
:1012B000AC71EC712C726C72AC72EC722C73E87BBA
:1012C00028744FF0010C383D6DE16046FFF7E2FCF9
:1012D0007448C619307B312845D1707B34282ED311
:1012E00037282CD8F07AFFF7D1F80146B07AFFF70B
:1012F000CDF801EB0010717BC0B200EB01206A4910
:101300000844A0F550500078C00710D0012085F89F
:1013100045000EE09BE196E3FDE3FDE3FDE3FDE325
:10132000FDE3FDE3FDE3FDE3FDE3FDE3FDE385F820
:1013300045406046FFF714FD307B312813D1707BA8
:10134000322875D1F07AFFF7A1F80146B07AFFF79D
:101350009DF801EB0010FFF788F850B185F8454083
:101360006046FFF7FDFC307B302800E06FE304D0DF
:101370005BE0012085F84500F2E7707B432818D137
:10138000F07AFFF783F80146B07AFFF77FF801EBB8
:1013900000104649C0B2085C18B1012085F845002C
:1013A00001E085F845406046FFF7DAFC307B3028E5
:1013B0003BD1707B30281ED336281CD8F07AFFF73B
:1013C00065F80146B07AFFF761F801EB0011707B18
:1013D000FFF75CF801EB0020FFF799F818B1012046
:1013E00085F8450001E085F845406046FFF7B8FC08
:1013F000307B302819D1707B452865D1F07AFFF712
:1014000045F80146B07AFFF741F801EB001000F50E
:10141000FA50FFF77CF818B1012085F8450001E08B
:1014200085F845406046FFF79BFC307B312817D19B
:10143000707B302876D1F07AFFF728F80146B07A31
:10144000FFF724F801EB00101949085C18B10120DE
:1014500085F8450001E085F845406046FFF780FCCF
:10146000307B32282DD1707B382848D1F07AFFF7B5
:101470000DF80146B07AFFF709F801EB00100D49AD
:10148000085CC8B1012085F8450017E0DB070020A3
:101490000048004000010020A80500200010014085
:1014A00014020020A75F0020521D0020C110002060
:1014B00052190020521A002085F845406046FFF777
:1014C0004FFC307B302817D1707B462863D1F07AEF
:1014D000FEF7DCFF0146B07AFEF7D8FF01EB001003
:1014E000FB49085C18B1012085F8450001E085F84A
:1014F00045406046FFF734FC307B322818D1707BC2
:10150000372848D1F07AFEF7C1FF0146B07AFEF7DE
:10151000BDFF01EB0010EF49085C20B1012085F808
:10152000450002E01EE085F845406046FFF718FCE4
:10153000307B33282FD1707B382818D1F07AFEF712
:10154000A5FF0146B07AFEF7A1FF01EB0010E249CA
:10155000085C40B185F845406046FFF701FC307BF0
:10156000332804D017E0012085F84500F4E7707BAC
:10157000372810D1F07AFEF789FF0146B07AFEF7DE
:1015800085FF01EB0010D249085CE8B385F84540BF
:101590006046FFF7E5FB95F848003F1D401E0CF143
:1015A000010C85F8480010F0FF0F7FF48EAE2A463C
:1015B0006C70022189F80010302189F80110412354
:1015C00089F8023089F8031089F8041089F80510A9
:1015D000412489F8064089F8071089F8081089F82D
:1015E0000910484689F80A4089F80B100173032353
:1015F000437337218173362189F80F10102182F847
:1016000025106879012800E00EE04FF000000FD0AF
:10161000B24B4A46145C1C54401C1E28FAD9687808
:10162000A87085F82610F7E1012085F84500AFE79E
:10163000AB4C4A46135C2354B5F87230401C5B1C1B
:10164000A5F872308842F5D3FEF73CFFD0E3BEF137
:10165000300F42F01986A34F312B7CD13428F8D1BA
:10166000302902D0342903D0CEE3342A02D0D4E387
:10167000342A71D14FF000084FEA0B0617F808C062
:10168000BCF1030F0AD0A8F1090CCCF3870C08F1C8
:10169000010886F847C0B8F1960FEFD3DDF844C0D3
:1016A000BCF1450F2AD1312D28D1BEF1300F25D103
:1016B000312B23D1342821D1302902D034290DD027
:1016C0001CE0342A1AD10020049006F8384F4FF05D
:1016D00001087470B470F470383E0EE0342A0DD1F5
:1016E0000020049006F83C4F4FF021087470B4704D
:1016F000F470347174713C3E8020059096F8470078
:1017000086F848006CE10498059B3D180344764830
:10171000AA7A1844491E8272EA7AC2722A7B02733C
:101720006A7B427386F848104046FFF7B3FA287B7D
:1017300031283BD1687B342824D3372822D8E87A53
:10174000FEF7A4FE0146A87AFEF7A0FE01EB00100A
:10175000C0B2697B01E0D3E3D3E300EB012063492E
:101760000844A0F550500078C00703D0012086F847
:10177000450001E086F845404046FFF7F1FA287B36
:10178000312813D1687B322874D1E87AFEF77EFEC7
:101790000146A87AFEF77AFE01EB0010FEF765FE1F
:1017A00040B186F845404046FFF7DAFA287B3028FA
:1017B00004D05CE0012086F84500F4E7687B43280C
:1017C00018D1E87AFEF762FE0146A87AFEF75EFEBF
:1017D00001EB00104649C0B2085C18B1012086F840
:1017E000450001E086F845404046FFF7B9FA287BFE
:1017F00030283CD1687B30281ED336281CD8E87AA4
:10180000FEF744FE0146A87AFEF740FE01EB001108
:10181000687BFEF73BFE01EB00203649085C18B1FF
:10182000012086F8450001E086F845404046FFF774
:1018300097FA287B30281AD1687B452866D1E87A48
:1018400000F5FA50C0B2FEF721FE0146A87AFEF775
:101850001DFE01EB0010FEF75AFE18B1012086F8BC
:10186000450001E086F845404046FFF779FA287BBD
:10187000312817D1687B302876D1E87AFEF706FE4A
:101880000146A87AFEF702FE01EB00111248405C07
:1018900018B1012086F8450001E086F84540404631
:1018A000FFF75EFA287B32282DD1687B382848D193
:1018B000E87AFEF7EBFD0146A87AFEF7E7FD01EBBB
:1018C00000100D49085CC8B1012086F8450017E0FA
:1018D000521B0020521C002052190020DB07002060
:1018E000A805002014020020A75F0020521D002040
:1018F000C110002052120020521A002086F84540E4
:101900004046FFF72DFA287B302817D1687B462800
:1019100063D1E87AFEF7BAFD0146A87AFEF7B6FD74
:1019200001EB0010FE49085C18B1012086F8450063
:1019300001E086F845404046FFF712FA287B32283E
:1019400018D1687B372848D1E87AFEF79FFD014619
:10195000A87AFEF79BFD01EB0010F249085C20B16C
:10196000012086F8450002E01EE086F8454040462A
:10197000FFF7F6F9287B33282FD1687B382818D158
:10198000E87AFEF783FD0146A87AFEF77FFD01EBBA
:101990000010E549085C40B186F845404046FFF735
:1019A000DFF9287B332804D017E0012086F84500B2
:1019B000F4E7687B372810D1E87AFEF767FD014627
:1019C000A87AFEF763FD01EB0010D549085C50B31F
:1019D00086F845404046FFF7C3F90498001D04907F
:1019E00096F8481000297FF48EAE7470062089F8AE
:1019F0000000012286F825207079494601284FF021
:101A0000000014D0C94B0C5C1C54401C0128FAD9AE
:101A10007078B07086F82620012240F22771C44801
:101A200020F082FAE4E1012086F84500D2E7C14CBB
:101A30000B5C2354B6F87230401C5B1CA6F8723065
:101A40009042F5D300E6BEF1300F42F01D84312BF9
:101A500041F00F85372841F06385392966D1302A56
:101A600041F01A86322E7DD1BCF1380FFBD1BAF18C
:101A7000030FF8D112984528F5D100983328F2D1F8
:101A80000BF122018BF80140022089F80000AA4ADC
:101A90000120C8709462887D4B460709C87D4FEAD3
:101AA000101C087E4FEA1019487E0609887E050939
:101AB000C87E00090190087F00090690487F4FEA20
:101AC000101B887F4FEA1018C87F4FEA101A38465B
:101AD000FEF7EBFCCC781855641CCC703846FEF74A
:101AE000E4FC946A7F4220449062887D00EB0710FA
:101AF000C0B2FEF7DAFC0446C8781C54401CC8701B
:101B0000887D00EB0710C0B2FEF7CFFC946A20443A
:101B1000906260460BE06FE142E27EE2BCE201E3EC
:101B2000B8E2F1E2BCE201E3FEE3FEE3FEE3FEF72E
:101B3000BCFC0446C8781C54401CC8706046FEF7C4
:101B4000B4FC946A20449062C87DCCF1000400EBA0
:101B50000410C0B2FEF7A9FC0746C8781F54401C09
:101B6000C87000E0F7E3C87D00EB0410C0B2FEF7D8
:101B70009CFC946A204490624846FEF796FC04461A
:101B8000C8781C54401CC8704846FEF78EFC946A06
:101B900020449062087EC9F1000400EB0410C0B23A
:101BA000FEF783FC0746C8781F54401CC870087EA7
:101BB00000EB0410C0B2FEF778FC946A20449062F7
:101BC0003046FEF772FC0446C8781C54401CC870AE
:101BD0003046FEF76AFC946A20449062487E744264
:101BE00000EB0410C0B2FEF760FC0646C8781E5435
:101BF000401CC870487E00EB0410C0B2FEF755FCD4
:101C0000946A204490622846FEF74FFC0446C87848
:101C10001C54401CC8702846FEF747FC946A2044B8
:101C20009062887E6C4200EB0410C0B2FEF73DFC6F
:101C30000546C8781D54401CC870887E00EB04100F
:101C4000C0B2FEF732FC946A204490620198FEF71D
:101C50002CFC0446C8781C54401CC8700198FEF740
:101C600024FC946A2044906201984442C87E00EBB0
:101C70000410C0B2FEF719FC0546C8781D54401C7C
:101C8000C870C87E00EB0410C0B2FEF70EFC946A68
:101C9000204490620698FEF708FC0446C8781C545D
:101CA000401CC8700698FEF700FC946A20449062BD
:101CB00006984442087F00EB0410C0B2FEF7F5FB23
:101CC0000546C8781D54401CC870087F00EB0410FE
:101CD000C0B2FEF7EAFB946A204490625846FEF7D1
:101CE000E4FB0446C8781C54401CC8705846FEF7F4
:101CF000DCFB946A20449062487FCBF1000400EB47
:101D00000410C0B2FEF7D1FB0546C8781D54401C34
:101D1000C870487F00EB0410C0B2FEF7C6FB0DE0B0
:101D2000521B0020521C002052190020DB0700200B
:101D300000480040A805002000010020946A2044CB
:101D400090624046FEF7B1FB0446C8781C54401C24
:101D5000C8704046FEF7A9FB946AC8F1000520440C
:101D60009062887F00EB0510C0B2FEF79EFBCC7836
:101D70001855641CCC70887F00EB0510C0B2FEF7CC
:101D800094FB946A204490625046FEF78EFBCC7818
:101D90001855641CCC705046FEF787FB946ACAF154
:101DA000000520449062C87F00EB0510C0B2FEF72A
:101DB0007CFBCC781855641CCC70C87F223900EBB2
:101DC0000510C0B2FEF771FB946A2044012430264E
:101DD000C2F8280091F825503030641C5E556D1C07
:101DE00081F825503C2CF5D9C01C906201F04ABC0A
:101DF00017B00020BDE8F08FBEF1300F42F04482F2
:101E0000312B7DD13428F9D1302906D0342978D02E
:101E1000382976D0432974D0FEE0FA4B302AFBD122
:101E2000302E47D1BCF1340F44D1BAF1300F41D13B
:101E3000129830283ED1009838283BD11698312886
:101E400038D11598032835D1D87C302832D3187D65
:101E500030282FD34046FEF710FB0146987BFEF753
:101E60000CFB01EB00118BF8471058468BF8014032
:101E7000062189F8001001228BF825209BF8051017
:101E80004B4601294FF0000108D0DF4C5D5C6554E2
:101E9000491C0129FAD941788170FCE3DB4D5C5C77
:101EA0006C54B0F87240491C641CA0F87240914216
:101EB000F5D3C7E50020D649302240F21F350A5439
:101EC000401CA842FBD30A201A5C0A54032A1FD0E4
:101ED000401CBE28F8D38BF849408BF84A4058463E
:101EE0008BF80140062189F8001001228BF825208B
:101EF0000E994B4601294FF000010CD0C24C01E075
:101F000039E214E05D5C6554491C0129F7D9C2E748
:101F1000C0490880DFE7BD4D5C5C6C54B0F872408E
:101F2000491C641CA0F872409142F5D38AE5B54B78
:101F3000302A71D1B749B64D00200A881E18B77AE9
:101F40008618AF551E5C032E1AD0401CB428F5D35A
:101F500059468BF80140062089F8000001228BF8D1
:101F600025200E984B4601284FF000000CD0A64CBF
:101F70001D5C2554401C0128FAD9487888708CE7EC
:101F800010440A380880E3E7A04D1C5C2C54B1F8DB
:101F90007240401C641CA1F872409042F5D351E598
:101FA00030287BD136297FD2032A7DD11846FEF70F
:101FB0006DFA0146F878FEF769FA01EB0011B8797D
:101FC000FEF764FA01EB00200121FEF7ADFA5A4654
:101FD0008BF80140062089F8000001218BF82510BC
:101FE0009BF805004C4601284FF0000008D0864BB6
:101FF000255C1D54401C0128FAD95078907080E06F
:10200000824B255C1D54B2F87250401C6D1CA2F826
:1020100072508842F5D315E5EAE3302874D13629A9
:1020200073D2032A42F030811846FEF72FFA014698
:10203000F878FEF72BFA01EB0011B879FEF726FAD3
:1020400001EB00200021FEF76FFA5A468BF80140A1
:10205000062089F8000001208BF825009BF8051068
:102060004B4601294FF0000108D0674C5D5C655478
:10207000491C0129FAD95178917087E0634D5C5C65
:102080006C54B2F87240491C641CA2F87240814240
:10209000F5D3D7E402E007E0302805D0312878D026
:1020A000302803D002F0F0B8452902D0432971D07E
:1020B000F8E7032AF6D11846FEF7E8F90146F87862
:1020C000FEF7E4F901EB001000F5FA500121FEF7EC
:1020D0002BFA58468BF80140062189F8001001219F
:1020E0008BF825109BF805204B46012A4FF0000283
:1020F0000CD0454C9D5CA554521C012AFAD942785B
:1021000082708BF8261087E40EE012E03F4D9C5C55
:10211000AC54B0F87240521C641CA0F872408A4261
:10212000F5D38FE4302804D031286AD0302802D08B
:10213000B8E7452902D0432970D0B3E7032AB1D1CB
:102140001846FEF7A3F90146F878FEF79FF901EB70
:10215000001000F57A700021FEF7E6F959468BF879
:102160000140062089F8000001208BF825009BF82B
:1021700005204B46012A4FF000020CD0224C9D5CFA
:10218000A554521C012AFAD94A788A708BF8260085
:1021900042E40CE085E01D4C9D5CA554B1F8725002
:1021A000521C6D1CA1F872508242F5D34AE43229C8
:1021B000BED1032ABCD11846FEF768F90146F8786B
:1021C000FEF764F901EB0010134921F810400A21D1
:1021D0008BF85A1058468BF80140062189F80010F8
:1021E00001218BF825109BF805204B46012A4FF062
:1021F000000214D0044C9D5CA554521C012AFAD94B
:102200007DE718E014020020DB070020A80500206D
:10221000A75F0020800000201211002072E0FE4D18
:102220009C5CAC54B0F87240521C641CA0F8724024
:102230008A42F5D306E43229BAD1032AB8D1184626
:10224000FEF724F90146F878FEF720F9F34A01EB8E
:102250000011012022F811000A218BF85A105A4669
:102260008BF80140062189F800108BF825009BF8B7
:1022700005104B4601294FF0000106D0E84C5D5C8B
:102280006554491C0129FAD9F5E6E34D5C5C6C54B0
:10229000B2F87240491C641CA2F872408142F5D326
:1022A00007E6032A84D11846FEF7F0F80146F878CD
:1022B000FEF7ECF801EB0010D84A0121A13A1154C5
:1022C0005A468BF80140062089F800008BF825104B
:1022D0009BF805004B4601284FF0000006D0D04D7A
:1022E0001C5C2C54401C0128FAD986E6CA4D1C5CA3
:1022F0002C54B2F87240401C641CA2F87240884210
:10230000F5D3D6E5032A97D11846FEF7BFF8014664
:10231000F878FEF7BBF801EB0010C049A1390C5466
:1023200058468BF8014002E022E0E3E0EBE00621B2
:1023300089F8001001228BF825209BF805104B46E8
:1023400001294FF0000107D0B54C5D5C6554491C74
:102350000129FAD99FE5DAE0AF4D5C5C6C54B0F826
:102360007240491C641CA0F872409142F5D3A0E56C
:10237000BEF1300F96D1AB4D342B5DD3302E91D1C1
:10238000BCF1320F8ED1139903298BD1FEF77EF861
:1023900002462879FEF77AF801463420FEF776F8EF
:1023A000081A02EB00100102A879FEF76FF801EBA2
:1023B0000011E879FEF76AF80844410841F27070AC
:1023C000814216D2E87AFEF761F80246A87AFEF753
:1023D0005DF802EB0013687BFEF758F80246287B95
:1023E000FEF754F802EB00108F4A03EB002022F8AE
:1023F000110058468BF80140062189F8001001228F
:102400008BF825209BF805104B4601294FF0000161
:1024100006D0834C5D5C6554491C0129FAD93AE524
:102420007D4D5C5C6C54B0F87240491C641CA0F893
:1024300072409142F5D33CE5302B7DD14528C1F067
:102440002387302E96D1BCF1320F93D113980328F5
:1024500090D11046FEF71AF80146A879FEF716F853
:1024600001EB001041086879462800D18031FF292E
:1024700019D8E87AFEF70AF80246A87AFEF706F8B5
:1024800002EB0013687BFEF701F80246287BFDF79C
:10249000FDFF02EB0010644A03EB002002EB410257
:1024A00042F6E061505258468BF80140062189F807
:1024B000001001238BF825309BF805104A460129AE
:1024C0004FF000010AD0564D545C6C54491C012950
:1024D000FAD9417881708BF8263014E64E4D545C61
:1024E0006C54B0F87240491C641CA0F872409942C8
:1024F000F5D3DEE4BEF1300FA4D1312B7DD13728E6
:102500007CD1392901D0442979D1302AFCD10BF171
:1025100038000021017041708170C17001714171FA
:102520008171C171017241728172C17201738BF844
:10253000011002223A4B00E0FEE3963BDFF8ECA0EC
:102540001A7001228BF8252052469AF80B00FDF7ED
:102550009DFF0346907AFDF799FF03EB0013D07BB4
:10256000FDF794FF0446907BFDF790FF04EB00100D
:10257000DFF8BC9006902B48C9F828101224807907
:102580004FF00008442805D19BF849001B1AA9F117
:10259000800044880022BEE30AEB040188783028DA
:1025A0007AD1C8785546452877D34878FDF76EFF2D
:1025B0000646285DFDF76AFF06EB0010400805900F
:1025C000C8784628059801D180300590A0380B289E
:1025D0007ED8DFF86080144D4FF4405043F23C0E3B
:1025E00000EB080797F801C020F0010625F806C0A7
:1025F00015F806C04FEA0C2C02E0FDE3FDE3FDE315
:1026000025F806C03F78801C6744AF537045E7D972
:102610000020DFF80CE00FE0A805002012110020D8
:10262000DB070020140200202C2D0020A75F0020D3
:102630000001002000600308AEF1A30E0DF120069A
:102640001EF800703754401C0C28F9D3012006EB0B
:10265000000C375C1CF801CC87EA0C0787F0940764
:102660008737FF433754401C0C28F0D3002006EB7B
:10267000000C375C9CF801C087EA0C0787F039072B
:10268000FF4318373754401C0B28F0D3002006EBCB
:10269000000C375C02E0FDE37EE0FEE09CF801C048
:1026A00007FB0CF7FF433754401C0B28EFD30120E6
:1026B00006EB000C375C1CF801CC07FB0CF787F02D
:1026C00045073754401C0C28F2D30027384600E059
:1026D000DBE005EB400C0CF5405C16F80080BCF923
:1026E00020C0E04501D17F1CFFB2401C0C28EED376
:1026F0000C2F7CD0059D0EEB050010F8A00C079068
:102700008046C0B200F00F05039505092846FDF785
:10271000CCFE0BF125060746DFF8B0C430780CF884
:102720000070401C30702846FDF7BFFED9F82870B5
:102730004D463844C9F828000398FDF7B6FE3778AF
:102740000CF807007F1C37700398FDF7AEFEAF6AE8
:102750003844A862C8F3072000F00F07000980463C
:102760000397FDF7A2FE37780CF807007F1C37703F
:102770004046FDF79AFEAF6A3844A8620398FDF719
:1027800094FE37780CF807007F1C37700398FDF72C
:102790008CFEAE6A3044A8628878554634286ED3E1
:1027A000C87830286ED3FDF771FE06468878FDF7AD
:1027B0006DFE001F06EB00100602285DFDF766FEA9
:1027C00006EB00154878FDF761FE2844460841F203
:1027D0006F70864202D2FE4830F91660F0B200F007
:1027E0000F05000980460395FDF75FFE01E04AE012
:1027F000F7E30BF12505DFF8D4C32F780CF80700B9
:102800007F1C2F704046FDF750FED9F82870074412
:10281000C9F828700398FDF748FE2F780CF80700D8
:102820007F1C2F700398FDF740FED9F828700744ED
:10283000C6F30720C9F8287000F00F0807093846CA
:10284000FDF733FE2E780CF80600761C2E70384605
:10285000FDF72BFED9F8286006444046C9F82860E9
:10286000FDF723FE2E780CF80600761C2E704046ED
:10287000FDF71BFED9F828500544C9F82850887880
:1028800030280AD0BBE107983AE7D148059D00EB14
:10289000450542F6E060285E32E7C8785546422892
:1028A0006CD841286AD34878FDF7F0FD0646285DCC
:1028B000FDF7ECFD06EB00104FEA5008C8784228FF
:1028C00001D108F18008C34850F82800C0B200F0D8
:1028D0000F060009CDE90206FDF7E7FD0BF125061D
:1028E000DFF8E8C237780CF807007F1C37700298D1
:1028F000FDF7DBFDD9F828700744C9F82870039864
:10290000FDF7D3FD37780CF807007F1C377003986C
:10291000FDF7CBFDD9F828700744AE48C9F82870F8
:1029200050F82800C71700EB1760C0F3072000F02D
:102930000F07000980460397FDF7B7FD37780CF8BD
:1029400007007F1C37704046FDF7AFFDD9F82870AF
:102950000744C9F828700398FDF7A7FD37780CF8ED
:1029600007007F1C37700398FDF79FFDD9F828609A
:102970000644C9F82860887830287CD1C878432874
:102980007AD14878FDF782FD0646285DFDF77EFD89
:102990008F4F06EB00108008E03F332857F8206087
:1029A000B04603D0342801D036280AD14FF08045F4
:1029B000AD8CA5F500454FEAE57C05EB9C7506EB73
:1029C000A508232803D0292801D02C2805D14FF0B1
:1029D0008045AD8C3544A5F50048242806D02E2826
:1029E0000CD02F280AD0312808D011E07A48D7F827
:1029F000905000882844A0F5004016E04FF0804534
:102A0000AD8C7719744D2D88A5F5803507EB050839
:102A1000352801D0372809D170480088A0F500403A
:102A2000C51700EB957006EBA00080460BF125055D
:102A300008F0FF066E744FEA1820A8743009FDF7FD
:102A400034FD624E2F78F0557F1C2F70687C000992
:102A5000FDF72BFDD9F828C04F466044C9F828007F
:102A6000687C4FEA101CCCF1000C00EB0C10C0B2DB
:102A7000FDF71BFD01E0C2E031E195F800C006F86A
:102A80000C000CF1010C85F800C0687C4FEA101CAA
:102A9000CCF1000C00EB0C10C0B2FDF706FDD7F82E
:102AA00028C06044B862A87C0009FDF7FEFC95F8D8
:102AB00000C006F80C000CF1010C85F800C0A87CE1
:102AC0000009FDF7F2FCD7F828C06044B862A87C82
:102AD0004FEA101CCCF1000C00EB0C10C0B2FDF75B
:102AE000E4FC95F800C006F80C000CF1010C85F828
:102AF00000C0A87C4FEA101CCCF1000C00EB0C10BD
:102B0000C0B2FDF7D2FCD7F828C06044B8624FEAE3
:102B1000184000F0FF0C85F811C0000AA8744FEAB5
:102B20001C10FDF7C2FC95F800C006F80C000CF173
:102B3000010C85F800C0687C0009FDF7B6FCD7F8E9
:102B400028C06044B862687C4FEA101CCCF1000CCD
:102B500000EB0C10C0B2FDF7A8FC95F800C006F819
:102B60000C000CF1010C85F800C0687C4FEA101CC9
:102B7000CCF1000C00EB0C10C0B2FDF796FCD7F8BE
:102B800028C06044B862A87C0009FDF78EFC95F867
:102B900000C006F80C000CF1010C85F800C0A87C00
:102BA0000009FDF782FCD7F828C06044B862A87C11
:102BB0004FEA101CCCF1000C00EB0C10C0B2FDF77A
:102BC00074FC95F800C006F80C0009E045070020E9
:102BD0002C2D00203C250020242C014024340140D1
:102BE0000CF1010C85F800C0A87C05096D4200EBD2
:102BF0000510C0B2FDF759FCBD6A2844B862887858
:102C0000554631286BD1C878312868D8302866D32A
:102C10004878FDF73BFC0646285DFDF737FC06EBE0
:102C200000104508C878312800D18035FE4850F89A
:102C30002500C0B200F00F0806093046FDF735FC4C
:102C40000BF125010746DFF8E4C308780CF80070A3
:102C5000401C08703046FDF728FCD9F8286006446F
:102C60004046C9F82860FDF720FC0E780CF80600F5
:102C7000761C0E704046FDF718FCD9F82860064413
:102C8000E948C9F8286050F82500C51700EB156021
:102C9000C0F3072000F00F0605092846FDF705FCE4
:102CA000074608780CF80070401C08702846FDF7AD
:102CB000FCFBD9F8285005443046C9F82850FDF7E8
:102CC000F4FB054608780CF80050401C08703046AC
:102CD000FDF7EBFBD9F828100144C9F82810D449B6
:102CE0008879392813D1487AFDF7D0FB0546087A50
:102CF000FDF7CCFB510005EB0010891C884206D87B
:102D0000CC48241D521C44808BF8492068E302F112
:102D10000108241D521C9A42FFF43EACC44881793C
:102D2000392901D18BF849309BF84A10069A0127BE
:102D30005D46A2EB010C5AE169E33846FDF7AAFFB4
:102D40000AEB0406B078302837D1F07851463028A5
:102D500077D3362819D87078FDF798FB0246085DBE
:102D6000FDF794FB02EB0011F078FDF78FFB01EB10
:102D70000020FDF7CCFB00B1012085F84500384666
:102D8000FDF7EEFFB078302817D1F078514645288E
:102D90005AD17078FDF77AFB0246085DFDF776FBA5
:102DA00002EB001000F5FA50FDF7B1FB00B1012075
:102DB00085F845003846FDF7D3FFB17831293CD17D
:102DC000F078342823D35146372820D87078FDF77F
:102DD0005DFB0246085DFDF759FB02EB0010F17840
:102DE000C0B200EB012094490844A0F5505000788F
:102DF000C00700D0012002E03BE391E3FEE385F849
:102E000045003846FDF7ACFFB078312815D1F07891
:102E10005246322832D17078FDF738FB0146105DFA
:102E2000FDF734FB01EB0010FDF71FFB50B1002054
:102E300085F845003846FDF793FFB078302803D079
:102E400019E09BE00120F3E7F0785246432849D18E
:102E50007078FDF71BFB0146105DFDF717FB01EBDA
:102E600000107649C0B2085C00B1012085F8450029
:102E70003846FDF775FFB078312817D1F078514604
:102E800030287BD17078FDF701FB0246085DFDF725
:102E9000FDFA00E033E36A4902EB0010085C00B180
:102EA000012085F845003846FDF75AFFB0785146B5
:102EB000322814D1F07838282DD17078FDF7E6FA51
:102EC0000246085DFDF7E2FA5E4902EB0010085C7D
:102ED00000B1012085F845003846FDF741FFB07884
:102EE000302815D1F0785146462860D17078FDF72A
:102EF000CDFA0246085DFDF7C9FA534902EB00100E
:102F0000085C00B1012085F845003846FDF728FF30
:102F1000B078322815D1F0785146372847D17078EB
:102F2000FDF7B4FA0246085DFDF7B0FA474902EB37
:102F30000010085C00B1012085F845003846FDF717
:102F40000FFFB0785146332831D1F078382818D1A6
:102F50007078FDF79BFA0246085DFDF797FA38494D
:102F600002EB0010085C50B15FF0000085F84500EE
:102F70003846FDF7F5FEB078332802D017E001207F
:102F8000F4E7F0785146372811D17078FDF77EFAD2
:102F90000246085DFDF77AFA2B4902EB0010085C47
:102FA00000B3002085F845003846FDF7D9FE2049DA
:102FB000487AFDF76BFA0246087AFDF767FA4FEA9E
:102FC000880102EB001001EB9701B1EB400F04F117
:102FD000040409D117484480781E85F84A007F1CF4
:102FE00009E018E20120DDE77F1CACF1010CBCF127
:102FF000000F3FF7A2AE25357F1EE87C0109084689
:10300000FDF753FA0346094A28781354401C2870E8
:103010000846FDF74AFAD9F8283049461844C9F855
:103020002800E87C14E000003C2100204507002037
:103030001402002080000020521D0020C11000203A
:1030400052190020521A0020521B0020521C00204E
:1030500000F00F042046FDF728FA2B78D0545B1CB3
:1030600005F825392046FDF720FA8B6A082F184409
:1030700088627DDD2535287D03091846FDF715FAA0
:10308000044628781454401C28701846FDF70DFAA1
:103090008B6A18448862287D00F00F042046FDF7F3
:1030A00004FA2B78D0545B1C05F825392046FDF72F
:1030B000FCF98B6A102F1844886259DD2535687D2C
:1030C00004092046FDF7F1F92B78D0545B1C2B70D6
:1030D0002046FDF7EAF98B6A18448862687D00F0A3
:1030E0000F031846FDF7E1F9044628781454401CF4
:1030F00005F825091846FDF7D8F98B6A182F1844EA
:10310000886235DD2535A87D04092046FDF7CDF917
:103110002B78D0545B1C2B702046FDF7C6F98B6AC8
:1031200018448862A87D00F00F031846FDF7BDF92A
:10313000044628781454401C05F825091846FDF764
:10314000B4F98B6A202F1844886211DD2535E87D9B
:1031500003091846FDF7A9F9044628781454401CC1
:1031600028701846FDF7A1F98B6A1844886200E0C0
:1031700090E0E87D00F00F042046FDF796F92B78EB
:10318000D0545B1C05F825392046FDF78EF98B6A73
:10319000282F184488627DDD2535287E03091846CE
:1031A000FDF783F9044628781454401C287018460B
:1031B000FDF77BF98B6A18448862287E00F00F03C4
:1031C0001846FDF772F9044628781454401C05F897
:1031D00025091846FDF769F98B6A302F1844886273
:1031E00058DD2535687E03091846FDF75EF904466B
:1031F00028781454401C28701846FDF756F98B6A3D
:1032000018448862687E00F00F042046FDF74DF9EF
:103210002B78D0545B1C05F825392046FDF745F97D
:103220008B6A382F1844886234DD2535A87E04095E
:103230002046FDF73AF92B78D0545B1C2B702046C2
:10324000FDF733F98B6A18448862A87E00F00F03FB
:103250001846FDF72AF9044628781454401C05F84E
:1032600025091846FDF721F98B6A402F184488621A
:1032700010DD2535E87E03091846FDF716F90446EA
:1032800028781454401C28701846FDF70EF98B6AF4
:10329000184400E092E08862E87E00F00F031846D0
:1032A000FDF703F9044628781454401C05F8250955
:1032B0001846FDF7FAF88B6A482F184488627DDDBE
:1032C0002535287F03091846FDF7EFF804462878CE
:1032D0001454401C28701846FDF7E7F88B6A184410
:1032E0008862287F00F00F031846FDF7DEF80446D9
:1032F00028781454401C05F825091846FDF7D5F820
:103300008B6A502F184488626ADD2535687F03096F
:103310001846FDF7CAF8044628781454401C287053
:103320001846FDF7C2F88B6A18448862687F00F07F
:103330000F042046FDF7B9F82B78D0545B1C05F834
:1033400025392046FDF7B1F88B6A582F184488625A
:1033500046DD2535A87F03091846FDF7A6F8044683
:1033600028781454401C28701846FDF79EF88B6A84
:1033700018448862A87F00F00F031846FDF795F8FF
:10338000044628781454401C05F825091846FDF712
:103390008CF88B6A602F1844886221DD2535E87F20
:1033A00004092046FDF781F82B78D0545B1C2B7064
:1033B0002046FDF77AF88B6A184400E010E0886236
:1033C000E87F00F00F042046FDF76FF82B78D0540B
:1033D0005B1C2B702046FDF768F88A6A10448862EF
:1033E000D9F82810C91CC9F82810FDF77DFEFE4841
:1033F000807944287EF4FCAC00208BF849008BF8DF
:103400004A00FEF7F5BC00BFBEF1300F3CD1312BB6
:10341000FCD13428FAD1342A75D1A6F1300009281C
:1034200071D85A468BF80140062089F80000012027
:103430008BF825000E994B4601294FF0000107D06B
:10344000EA4C5D5C6554491C0129FAD9FEF713BEAC
:10345000E74C5D5C6554B2F87250491C6D1CA2F8D3
:1034600072508142F5D3FEF7EFB800BFBEF1300FC6
:10347000CCD1DD4D302B08D0312B51D04FF4FA5246
:10348000342B77D3302E7AD05EE2312874D14329A1
:1034900073D1302AFCD1302EF6D1BCF1310F6DD171
:1034A000BAF1030FF0D112984428EDD100984428C6
:1034B000EAD15B468BF80140022189F800103021E7
:1034C00089F80110392189F80210032189F80310C5
:1034D000362189F80410432189F8051006228BF85B
:1034E00025200E99484601294FF000010CD0BF4C11
:1034F000455C6554491C0A29FAD9587898708BF8AC
:103500002620FEF789BAFDE3B94D445C6C54B3F84C
:103510007240491C641CA3F872409142F5D3A2E7A3
:10352000B14937286AD2302EAED1BCF1320F66D104
:10353000BAF1030FA8D1FCF7A9FF02028879FCF7C2
:10354000A5FF02EB0012C879FCF7A0FF1044400869
:103550000BF118018BF80140022289F800200122AA
:103560004A73A44A4B469462A34C34F82000C4B278
:103570008C77F9E389E002E0F0E16FE2E7E3BCF188
:10358000320F7DD1BAF1030F86D1FCF77FFF0146E0
:103590002879FCF77BFF01EB00100102E879FCF7CA
:1035A00075FF0346A879FCF771FF03EB0010084490
:1035B000A0F580404008904201D3A0F5FA600BF1DD
:1035C00018018BF80140022389F8003001234B7366
:1035D000884B4A469C62894C34F81000C4B28C7700
:1035E000000AC8772009FCF760FF4C7B1055641C6B
:1035F0004C73887F0009FCF758FF01E04CE04DE078
:103600009C6A20449862887F0409644200EB04109D
:10361000C0B2FCF74AFF4C7B1055641C4C73887F8A
:103620000409644200EB0410C0B2FCF73EFF9C6A40
:1036300020449862C87F0009FCF737FF4C7B105587
:10364000641C4C73C87F0009FCF72FFF9C6A204460
:103650009862C87F0409644200EB0410C0B2FCF712
:1036600024FF4C7B1055641C4C73C87F01094942F0
:1036700000EB0110C0B2FCF718FF996A0844F2E3AE
:1036800087E000BFFDF730FDBBE6312B04D0342BC3
:103690007ED3302E7DD057E1302EFCD15249BCF183
:1036A000340FF8D1BAF1030FF5D1FCF7EFFE0202A7
:1036B0008879FCF7EBFE02EB0012C879FCF7E6FE16
:1036C000104445080BF118028BF80140022089F8DC
:1036D00000004849012050738C62474C4B4654F817
:1036E000250004EB8505C4B2C61700EB166094777D
:1036F000000AD0772009FCF7D8FE547B1855641CCB
:103700005473907F0009FCF7D0FE8C6A20448862D5
:10371000907F0409644200EB0410C0B2FCF7C5FEC0
:10372000547B1855641C5473947F2009404204EB69
:103730000010C0B2FCF7B9FE8C6A20448862D07FCA
:103740000009FCF7B2FE547B1855641C5473D07FFB
:103750000009FCF7AAFE8C6A20448862D07F040925
:10376000644200EB0410C0B2FCF79FFE547B185576
:10377000641C5473D07F0409644200EB0410C0B28F
:10378000FCF793FE8C6A204488626868C4B201E04A
:10379000E2E058E0C51700EB15609477000AD07797
:1037A0002009FCF782FE547B1855641C5473907FEB
:1037B0000009FCF77AFE8C6A20448862907F040935
:1037C000644200EB0410C0B2FCF76FFE547B185546
:1037D000641C5473907F0409644200EB0410C0B26F
:1037E000FCF763FE8C6A0BE014020020DB0700206C
:1037F000A8050020000100203C2100202C2D0020E5
:1038000020448862D07F0009FCF74FFE547B185596
:10381000641C5473D07F0009FCF747FE8C6A204477
:103820008862D47F2009404204EB0010C0B2FCF74C
:103830003CFE547B1855641C5473D07F02095242DD
:1038400000EB021079E2BCF1340F7DD1BAF1030F25
:10385000FBD1FCF71BFE01462879FCF717FE001F81
:1038600001EB00100102A879FCF710FE01EB00113A
:10387000E879FCF70BFE084400EBD0704010904252
:1038800001D3A0F5FA6059468BF80140022289F86D
:10389000002001228BF82520FE4A4D469462FE4C02
:1038A00004EB400334F91000B3F90260002E7CDA17
:1038B000761C00EB0640EDE088741809FCF7F5FD76
:1038C0000B78E8545B1C0B70487C0009FCF7EDFD9D
:1038D000936A18449062487C03095B4200EB031032
:1038E000C0B2FCF7E2FD0B78E8545B1C0B70487C1F
:1038F00003095B4200EB0310C0B2FCF7D6FD936AEC
:1039000018449062887C0009FCF7CFFD0B78E854DE
:103910005B1C0B70887C0009FCF7C7FD936A184498
:103920009062887C03095B4200EB0310C0B2FCF795
:10393000BCFD0B78E8545B1C0B70887C0109494284
:1039400000EB0110C0B200E013E0FCF7AEFD916A9D
:1039500008449062FEF748BA302B0AD145287DD33F
:10396000302EFAD1CD4ABCF1340F03D0BCF1320F66
:1039700075D069E1BAF1030FFBD10846FCF786FD6B
:1039800051790902A1F58A4101EB0011D079FCF7C8
:103990007DFD084400EBD07059468BF801400222AF
:1039A00089F800204D46012200E010E041F27073DA
:1039B0008BF8252003EB6006B64AB74800EB4603B8
:1039C0009462B3F9024030F91600002C5FDBC4B2F8
:1039D0002531C61700EB16604C74000A8874200964
:1039E000FCF763FD0C782855641C0C70487C0009BA
:1039F000FCF75BFD946A20449062487C04096442B1
:103A000000EB0410C0B2FCF750FD0C782855641C84
:103A10000C70487C0409644200EB0410C0B2FCF74F
:103A200044FD946A20449062887C0009FCF73DFDC7
:103A30000C782855641C0C70887C0009FCF735FD57
:103A4000946A20449062887C0409644200EB04106C
:103A5000C0B2FCF72AFD0C78285501E075E171E051
:103A6000641C0C70887C0409644200EB0410C0B232
:103A7000FCF71BFD946A20449062B3F90200C3B2C4
:103A8000C41700EB14604B74C0F3072014E7641EE6
:103A900000EB0440C0F1FF30C3432531D8B2487475
:103AA0001C0A8C740009FCF700FD0C782855641C76
:103AB0000C70487C0009FCF7F8FC946A2044906282
:103AC000487C0409644200EB0410C0B2FCF7EDFC32
:103AD0000C782855641C0C70487C0409644200EB87
:103AE0000410C0B2FCF7E1FC946A20449062887C28
:103AF0000009FCF7DAFC0C782855641C0C70887CF3
:103B00000009FCF7D2FC946A20449062887C040986
:103B1000644200EB0410C0B2FCF7C7FC0C782855D7
:103B2000641C0C70887C0409644200EB0410C0B271
:103B3000FCF7BBFC946A20449062180CC3B24B742F
:103B4000000AB9E6BAF1030F7ED18BF801400225D5
:103B50004B4689F80050DFF83C9101258BF8255041
:103B6000C9F82840FCF792FC01029079FCF78EFC22
:103B700001EB0011D079FCF789FC0844A0F56060E6
:103B80004408454842F6E06100EB4402A02C515E37
:103B900072D3AB2C70D8DFF808C14FF4405243F217
:103BA0003C0800BF02EB0C077E7822F0010546536B
:103BB000465D360246533F78921C3E44465342458A
:103BC000F0D9384E002508AA775D57556D1C0C2D8D
:103BD000FAD3012502EB050C575D1CF801CC87EAEE
:103BE0000C0787F094078737FF4357556D1C0C2D42
:103BF000F0D3002502EB050C575D9CF801C087EA65
:103C00000C0787F03907FF43183757556D1C0B2DEC
:103C1000F0D3002502EB050C575D9CF801C007FBB3
:103C20000CF7FF4357556D1C0B2DF3D3012502EB09
:103C3000050C575D1CF801CC07FB0CF787F0450716
:103C400057556D1C0C2D00E08DE0F0D300273D464C
:103C500000EB450C0CF5405C12F80580BCF920C067
:103C6000E04501D17F1CFFB26D1C0C2DF0D30C2F51
:103C700002D0301910F8A01C002902DAC1F1FF307F
:103C8000C143C8B20BF12502090A507491740009AE
:103C90000AE00000000100202C2D0020140200206A
:103CA0000060030838070020FCF7FFFB1178585428
:103CB000491C1170507C0009FCF7F7FBD9F828402B
:103CC00049462044C9F82800547C2009404204EBAE
:103CD0000010C0B2FCF7E9FB14781855641C14708E
:103CE000507C0409644200EB0410C0B2FCF7DDFB19
:103CF0008C6A20448862907C0009FCF7D6FB14781B
:103D0000185500E09BE2641C1470907C0009FCF7DD
:103D1000CCFB8C6A20448862907C0409644200EBEE
:103D20000410C0B2FCF7C1FB14781855641C147061
:103D3000927C1009404202EB0010C0B2FCF7B5FBC8
:103D40008A6A1044C01C88629CE4302E06D1FE4969
:103D5000BCF1320F02D1BAF1030F06D0FA4A45285E
:103D600001D2302E7ED08FE230E0FCF78FFB0202D2
:103D70008879FCF78BFB02EB0012C879FCF786FB15
:103D800011184120FCF782FB02023020FCF77EFB79
:103D900002EB00123020FCF779FB1044081A00EB0C
:103DA000D07040100BF118018BF80140022289F805
:103DB000002001224A73E54A4B469462E44C54F8D1
:103DC0002000C4B2C5178C7700EB1560000AC877D5
:103DD0002009FCF76AFB4C7B1855641C4C73887FE8
:103DE0000009FCF762FB946A20449062887F040912
:103DF000644200EB0410C0B2FCF757FB4C7B185533
:103E0000641C4C73887F0409644200EB0410C0B248
:103E1000FCF74BFB946A20449062C87F0009FCF7D2
:103E200044FB4C7B1855641C4C73C87F0009FCF79D
:103E30003CFB946A20449062C87F0409644200EB12
:103E40000410C0B2FCF731FB4C7B1855641C4C735A
:103E5000C87F0109494200EB0110C0B2FCF725FB05
:103E6000916A01E002E0DFE1084473E5BCF1340F40
:103E700078D1BAF1030F75D143281DD2FCF706FBA8
:103E800001029079FCF702FB01EB0011D079FCF7FD
:103E9000FDFA01444120FCF7F9FA03023020FCF757
:103EA000F5FA03EB00133020FCF7F0FA1844081A77
:103EB00000EBD07040101DE0FCF7E8FA01029079A9
:103EC000FCF7E4FA01EB0011D079FCF7DFFA0144CA
:103ED0004320FCF7DBFA03023020FCF7D7FA03EBB0
:103EE00000133020FCF7D2FA1844081AC11700EB6F
:103EF0009170801059468BF80140022389F80030F8
:103F000001238BF82530914B4D469C625279432A10
:103F100075D3904E332856F82020144603D0342809
:103F200001D0362809D14FF08042928CA2F5004290
:103F3000D71702EB977204EBA202232803D029289B
:103F400001D02C2805D14FF08042928C2244A2F55A
:103F50000042242807D02E280DD02F280BD031283E
:103F600009D011E090E17C48D6F890200088024406
:103F7000A2F5004215E04FF08042928CA618764AD6
:103F80001288A2F580323244352801D0372808D172
:103F900072480088A0F50040C21700EB927004EB55
:103FA000A002002A02DAC2F1FF30C2432531D0B2AA
:103FB0004874140A8C740009FCF777FA0C782855B9
:103FC000641C0C70487C0009FCF76FFA9C6A204462
:103FD0009862487C0409644200EB0410C0B2FCF70C
:103FE00064FA0C78285504F101040C704C7C4FEAFB
:103FF0001410C0F1000004EB00108CE0FFE7544CFB
:1040000054F8202004EB8004A08812EB00405BD41D
:10401000D0B22531D617487402EB1662120A8A74A0
:104020000009FCF742FA0A78A854521C0A70487C2E
:104030000009FCF73AFA9A6A10449862487C02092F
:10404000524200EB0210C0B2FCF72FFA0A78A854D3
:10405000521C0A70487C0209524200EB0210C0B2A6
:10406000FCF723FA9A6A10449862887C0009FCF7EE
:104070001CFA0A78A854521C0A70887C0009FCF7C4
:1040800014FA9A6A10449862887C0209524200EB42
:104090000210C0B2FCF709FA0A78A854521C0A7040
:1040A000887C0209524200EB0210C0B2FCF7FDF915
:1040B0009A6A104498626068C2B2C41700EB146038
:1040C0004A74C0F3072063E0C0F1FF30C2432531DA
:1040D000D0B24874140A8C740009FCF7E6F90C7825
:1040E0002855641C0C70487C0009FCF7DEF99C6ABA
:1040F00020449862487C0409644200EB0410C0B27A
:10410000FCF7D3F90C782855641C0C70487C040922
:10411000644200EB0410C0B2FCF7C7F99C6A20446B
:104120009862887C0009FCF7C0F90C782855641C5B
:104130000C70887C0009FCF7B8F99C6A20449862EE
:10414000887C040964420BE0140200200001002076
:104150003C2500204C2C0020242C0140243401401C
:1041600000EB0410C0B2FCF7A0F90C782855641CD1
:104170000C70887C0409644200EB0410C0B2FCF7A8
:1041800094F99C6A20449862100CC2B24A74000AE6
:1041900088741009FCF789F90A78A854521C0A702F
:1041A000487C0009FCF781F99A6A10449862487CBF
:1041B0000209524200EB0210C0B2FCF776F90A780D
:1041C000A854521C0A70487C0209524200EB0210AB
:1041D000C0B2FCF76AF99A6A10449862887C0009B8
:1041E000FCF763F90A78A854521C0A70887C00090D
:1041F000FCF75BF99A6A10449862887C0209524283
:1042000000EB0210C0B2FCF750F90A78A854521C17
:104210000A70887C0109494200EB0110C0B2FCF72A
:1042200044F9996A08449862C01C98628CE500BF02
:10423000BEF1300F28D1312B26D1342824D1F948B2
:10424000302921D1302A1FD1302E1DD1BCF1340F9D
:104250001AD1BAF1300F17D11299302914D100991F
:10426000382911D1169930290ED1139930290BD143
:10427000B8F1300F08D1017C302905D1407C3028BD
:1042800002D1159803280AD0E64900200C54401C9E
:10429000C828FBD3E44904200861FDF7A9BD5A46AC
:1042A0008BF80140062089F8000001218BF82510C9
:1042B0000E984B4601284FF0000007D0DB4C1D5CE8
:1042C0002554401C0128FAD9FDF797BED84D1C5C37
:1042D0002C54B2F87240401C641CA2F87240884210
:1042E000F5D3FDF7B1B92DE9F04FD249D24C0844CE
:1042F00042F61A7162180379891EB2F90060CF4A3A
:1043000003F00F0C675EC5784FF000084FF001090D
:10431000A2F18001BCF1040F07D1DFF824A3842DA2
:1043200007D0942D26D0A42D5AD0BCF1050F7DD0F6
:1043300098E0C2F82C8083780B6440794C46823830
:1043400000EBD07040108000001D486419184E2901
:104350000FD20021554608E05E1835F8166016B9F0
:1043600004FA01F6B044491C89B28142F4D3C2F880
:104370002C801DE29D09CD644379DF0706D004EB54
:10438000850404F54054B4F95A4006E0CDB104EB7D
:10439000850404F54054B4F94A4080782044886488
:1043A000823B03EBD37040108000001DC2F82C80CC
:1043B00048648C6C4B4621184E29DAD200215546B0
:1043C0000BE080783044EAE7661835F8166016B9D5
:1043D00003FA01F6B044491C89B28142F4D3C6E71E
:1043E0009D09CD644379DE0706D004EB850404F50E
:1043F0004054B4F9584006E0DDB104EB850404F5FF
:104400004054B4F94840807820448864823B03EBF0
:10441000D370401083001B1DC2F82C804B64896C44
:104420004C46C8184E28A4D2002000E010E05546A3
:104430000BE080783844E8E70E1835F8166016B9B6
:1044400004FA00F6B044401C80B29842F4D38EE7E0
:10445000DFF8ECA1842DAAF1510A22D0942D3ED090
:10446000A42D75D0BCF1080F09D3DFF8D8B1842D85
:104470000BF5C06E69D0942D68D0A42D67D0BCF127
:10448000030F09D8DFF8C0A140F2E73B842D7DD0AF
:10449000942D7CD0A42D7BD0802D7AD0822DFCD081
:1044A00045E2C2F82C8083780B6440794C46823810
:1044B00000EBD07040108000001D486419184E2990
:1044C000B1D20021554607E05E18AE5D16B104FA80
:1044D00001F6B044491C89B28142F5D347E79D09F2
:1044E000CD644379DF0706D004EB850404F540541E
:1044F000B4F95A4006E0CDB104EB850404F540540C
:10450000B4F94A40807820448864823B03EBD3703E
:1045100040108000001DC2F82C8048648C6C4B4613
:1045200021184E29CCD2002155460AE0807830442B
:10453000EAE76618AE5D16B103FA01F6B044491C0D
:1045400089B28142F5D312E702E03BE090E0F4E06B
:104550009D09CD644379DE0706D004EB850404F59C
:104560004054B4F9584006E0F5B104EB850404F575
:104570004054B4F94840807820448864823B03EB7F
:10458000D370401080004B46001D03E037E157E137
:104590008FE1C7E1C2F82C8048648C6C21184E2949
:1045A0008ED2002155460AE080783844E5E7661847
:1045B000AE5D16B103FA01F6B044491C89B28142DE
:1045C000F5D3D4E6C2F82C8084780D2B03D81F4D88
:1045D00005EB03252C440C64407940F2FF568238E9
:1045E00000EBD07040108000001D48640D6C4C46FC
:1045F0002918B14201D20D2B04D9FF2992D20F2BD9
:1046000026D0F3E300215E4607E06F18F75D17B18F
:1046100004FA01F7B844491C89B28142F5D3C2F8C3
:104620002C80ECE71402002000100140DB07002082
:10463000A805002000C003082C2D00200001002048
:104640001211002052120020521D002000F8FFFF1E
:1046500000214346764607E06F18F75D17B104FA6C
:1046600001F73B44491C89B28142F5D3D362BDE3D3
:104670009D098A46CD644179CF0706D004EB8504B5
:1046800004F54054B4F95A4006E0FDB104EB85044A
:1046900004F54054B4F94A4080782044CAF84800F0
:1046A000823901EBD17040108000001DC2F82C80CF
:1046B0004C465146CAF84400BCF10D0F09D84FEAE8
:1046C0000C258E6CA5F50065354403E080783044F8
:1046D000E4E78D6C0D642946054440F2FF56B5426F
:1046E00002D2BCF10D0F07D9FF2D8AD2DD432D0771
:1046F00087D1BCF10D0F0ED800255E4607E04F199B
:10470000F75D17B104FA05F7B8446D1CADB28542E8
:10471000F5D3C2F82C80DB431B07A8D1454676466B
:1047200007E0CF18F75D17B104FA03F73D445B1CAF
:104730009BB28342F5D3D56258E39D098A46CD6486
:104740004179CE07564606D004EB850404F5405463
:10475000B4F9584006E065B304EB850404F5405411
:10476000B4F9484080782044CAF84800823901EB07
:10477000D17040108000001DC2F82C807064B56CB0
:104780004C463146BCF10D0F03D805EB0C25A5F5C1
:1047900000650D642946054440F2FF56B54202D239
:1047A000BCF10D0F0BD9FF2DC6D2DD432D0703D071
:1047B0001CE380783844D7E7BCF10D0F0ED80025F4
:1047C0005E4607E04F19F75D17B104FA05F7B844E4
:1047D0006D1CADB28542F5D3C2F82C80DB431B07BC
:1047E000AAD14546764607E0CF18F75D17B104FA1F
:1047F00003F73D445B1C9BB28342F5D39BE7C2F8B1
:104800002C80847804EB03230B6440794C46823877
:1048100000EBD07040108000001D1D1848645D45FD
:104820008AD20021554608E05E18AE5DF60702D038
:1048300004FA01F6B044491C89B28142F4D396E5EA
:104840009D09CD644379DF0706D004EB850404F5A8
:104850004054B4F95A4006E0E5B104EB850404F590
:104860004054B4F94A40807820448864823B03EB8A
:10487000D37040108000001DC2F82C8048648B6CFF
:104880004C4603EB0C231D180B645D4590D20021B0
:1048900055460BE080783044E7E75E18AE5DF607DA
:1048A00002D004FA01F6B044491C89B28142F4D323
:1048B0005DE59D09CD644379DE0706D004EB8504F0
:1048C00004F54054B4F9584006E0E5B104EB850422
:1048D00004F54054B4F94840807820448864823B11
:1048E00003EBD37040108000001DC2F82C80486498
:1048F0008B6C4C4603EB0C231D180B645D458FD26B
:10490000002155460BE080783844E7E75E18AE5D3D
:10491000F60702D004FA01F6B044491C89B281427C
:10492000F4D324E590F805C0BCF1800F2CD0DFF85B
:10493000A0C8DFF8A0980CF5C0789CF859C041F2E7
:10494000873EA9F5806A42F6E06B862D21D0962D30
:1049500044D0A62D69D0862D1ED0962D7DD0A62DB3
:104960007CD0862D1BD0962D79D0A62D78D0862D83
:1049700018D0962D75D0A62D74D0862D15D0962DD5
:1049800071D0A62D70D031E280784B6400EB03200B
:10499000D8E14579862D0CD04579882D7DD0457993
:1049A000842D6ED04579822D6CD04579802D6AD0CA
:1049B0001CE2807800EB03204008C1E9100334F9C1
:1049C0001030D362BCF1520FDDD104EB40000B6517
:1049D000B0F902204A65B0F90400E9E04579862D76
:1049E0003DD3872D7BD887789809C0F1000C03EB65
:1049F0008C134B6407EB03235B08C8640B64862DA0
:104A000006D004EB800000F54050B0F95A0006E0F3
:104A100038B104EB800000F54050B0F94A0018446A
:104A200033E0F01831E0D062E0E14579862D17D30C
:104A3000872D79D886789809C0F1000C03EB8C1388
:104A40004B6406EB03235B08C8640B64862D10D00F
:104A500004EB800000F5405008E040E064E0AAE08C
:104A6000D4E002E127E16FE194E116E0B0F95800EB
:104A7000D5E748B104EB800000F54050B0F948009C
:104A8000CDE77DE0D9E040E1F818886441F66F0198
:104A9000884274D834F91000C5E7807800EB032011
:104AA0004008C1E91003BCF1520F11D141F2853326
:104AB00098420DD804EB400303F5FA63B3F90050B4
:104AC0000D65B3F902504D65B3F90430C8F81030E4
:104AD0007045A8D804EB4000B0F9D00732E1457921
:104AE000882D68D3892D69D887789809C0F1000C82
:104AF00003EB8C134B6407EB03235B08C8640B6464
:104B0000882D06D004EB800000F54050B0F95A0023
:104B100006E038B104EB800000F54050B0F94A00DF
:104B2000184424E0F01822E04579882D6ED3892DB1
:104B300025D886789809C0F1000C03EB8C134B64E0
:104B400006EB03235B08C8640B64882D06D004EBD6
:104B5000800000F54050B0F95800E1E730B104EBB7
:104B6000800000F54050B0F94800D9E7F818886493
:104B7000704504D804EB4000B0F9D00753E719E0C2
:104B8000807800EB03204008C1E91003C72802D851
:104B900059F82030D362BCF1520F0BD1C52809D887
:104BA00059F8203009EB80000B6542684A6580683F
:104BB000C8F810001AE14579842D56D3EDB2852D41
:104BC00056D887789809C0F1000C03EB8C134B641E
:104BD00007EB03235B08C8640B64842D06D004EB49
:104BE000800000F54050B0F95A0006E060B104EBD7
:104BF000800000F54050B0F94A0018448864C72886
:104C000073D859F820000EE7F018F7E74579842D9E
:104C100051D3852D69D885789809464203EB8613D0
:104C20004B64C86405EB032304EB80005B0800F5CC
:104C300040500B64B0F95800DFE7807800EB0320A8
:104C40004008C1E91003BCF1520F0BD1FD2809D86F
:104C50005AF820400AEB80030C655C684C659B6841
:104C6000C8F810305AF820006CE04579822D6BD3DB
:104C7000EDB2832D6BD887789809C0F1000C03EB57
:104C80008C134B6407EB03235B08C8640B64822D11
:104C900006D004EB800000F54050B0F95A0006E061
:104CA00038B104EB800000F54050B0F94A001844D8
:104CB00025E0F01823E04579822D6BD3832D14D89D
:104CC00086789809C0F1000C03EB8C134B6406EB5B
:104CD00003235B08C8640B64822D07D004EB8000BB
:104CE00000F54050B0F95800E1E77EE030B104EB48
:104CF000800000F54050B0F94800D8E7F818886403
:104D0000FF2873D85AF820008DE6807800EB032046
:104D10004008C1E91003BCF1520F0FD1FD280DD896
:104D200004EB400333F90B500D6542F6E2655D5F1D
:104D30004D6542F6E4655B5FC8F8103004EB400354
:104D400033F90B0008646EE64579802D4ED3EDB241
:104D5000812D4BD887789809C0F1000C03EB8C1398
:104D60004B6407EB03235B08C8640B64802D06D0FB
:104D700004EB800000F54050B0F95A0006E038B16D
:104D800004EB800000F54050B0F94A00184424E0DC
:104D9000F01822E04579802D28D3812D26D88678F9
:104DA0009809C0F1000C03EB8C134B6406EB032352
:104DB0005B08C8640B64802D06D004EB800000F50E
:104DC0004050B0F95800E1E730B104EB800000F545
:104DD0004050B0F94800D9E7F8188864FF2805D892
:104DE00004EB400131F90B001DE6FFE70020BDE8B0
:104DF000F08F2DE9F84FF849F84C0F1842F61A7168
:104E00006318891E387934F90190B3F900A0F44988
:104E100000F00F050022012397F803C0A1F18006DE
:104E2000042D0AD1DFF8BC83BCF1840F08D0BCF19B
:104E3000940F22D0BCF1A40F54D0052D77D094E06C
:104E4000CA62BD7835647879823800EBD070401042
:104E50008000001D2C1870644E2C0DD2002408E038
:104E60002E1938F8166016B903FA04F63244641C99
:104E7000A4B28442F4D3CA6220E28509F564787949
:104E80005FEAC07C06D004EB850404F54054B4F915
:104E90005A4006E0B5B104EB850404F54054B4F97A
:104EA0004A40BD782C44823800EBD0704010B46486
:104EB0008000001D2546CA62044470644E2CDBD27B
:104EC00000240CE0BD780AEB0504ECE72E1938F855
:104ED000166016B903FA04F63244641CA4B2844284
:104EE000F4D3C8E78509F56478795FEAC07C06D019
:104EF00004EB850404F54054B4F9584006E0BDB114
:104F000004EB850404F54054B4F94840BD782C44C2
:104F1000823800EBD0704010B4648000001D25463C
:104F2000CA62044470644E2CA6D200240DE00FE047
:104F3000BD7809EB0504EBE72E1938F8166016B9B1
:104F400003FA04F63244641CA4B28442F4D392E718
:104F5000DFF89082BCF1840FA8F151082AD0BCF18F
:104F6000940F43D0BCF1A40F79D0082D0CD3DFF8F7
:104F700078B2BCF1840F0BF5C06E6DD0BCF1940F0C
:104F80006BD0BCF1A40F69D0032D0CD8DFF85CB254
:104F900040F2E73EBCF1840F7ED0BCF1940F7CD090
:104FA000BCF1A40F7AD0BCF1800F78D0BCF1820F95
:104FB000FBD046E2CA62BD7835647879823800EB6E
:104FC000D07040108000001D2C1870644E2CABD2A5
:104FD000002408E02E1918F8066016B103FA04F64A
:104FE0003244641CA4B28442F4D344E78509F564D6
:104FF00078795FEAC07C06D004EB850404F5405460
:10500000B4F95A4006E0B5B104EB850404F5405408
:10501000B4F94A40BD782C44823800EBD07040107F
:10502000B4648000001D2546CA62044470644E2C9E
:10503000CDD200240CE0BD780AEB0504ECE72E1974
:1050400018F8066016B103FA04F63244641CA4B2E0
:105050008442F4D30FE702E03BE079E0F1E0850918
:10506000F56478795FEAC07C06D004EB850404F52A
:105070004054B4F9584006E0DDB104EB850404F572
:105080004054B4F94840BD782C44823800EBD070CD
:105090004010B464800003E039E157E192E1CDE1D2
:1050A000001D2546CA62044470644E2C8FD2002431
:1050B0000CE0BD7809EB0504E7E72E1918F8066047
:1050C00016B103FA04F63244641CA4B28442F4D349
:1050D000D1E6CA62BC780D2803D8454D05EB002502
:1050E0002C4434647C7940F2FF57823C04EBD47446
:1050F0006410A400241D7464366C3519BD4201D2BD
:105100000D2804D9FF2D93D20F2813D0D6E0002507
:105110005F460BE006EB050C17F80CC0BCF1000F66
:1051200002D003FA05FC62446D1CADB2A542F1D376
:10513000CA62E9E70020754607E03718EF5D17B14E
:1051400003FA00F73A44401C80B2A042F5D392E63D
:105150004FEA901CB146C6F84CC07E795FEAC6782B
:1051600006D004EB8C0404F54054B4F95A4008E02E
:10517000BCF1000F3ED004EB8C0404F54054B4F9AC
:105180004A40BF7807EB0407823E06EBD6746410F2
:10519000C9F84870A400241DCA62C9F84440D9F86F
:1051A00048704E460D2D03D807EB0527A7F500677D
:1051B00037643E46274440F2FF5C674501D20D2D1F
:1051C0001DD9FF2FA2D2C7433F0716D076E00000BB
:1051D000000000203C25002000C003082C2D0020EA
:1051E000000100201211002052120020521D002048
:1051F00000F8FFFFBF785744C6E70D2D11D80025F2
:105200005F460BE006EB050C17F80CC0BCF1000F75
:1052100002D003FA05FC62446D1CADB2A542F1D385
:10522000CA62C0430007D1D1754607E03718EF5D69
:1052300017B103FA00F73A44401C80B2A042F5D3FC
:1052400019E64FEA901CB246C6F84CC07E795FEA78
:10525000C67806D004EB8C0404F54054B4F95840E9
:1052600008E0BCF1000F2AD004EB8C0404F5405494
:10527000B4F94840BF782744823E06EBD6746410E8
:10528000CAF84870A400241DCA62CAF84440DAF87B
:10529000487056460D2D03D807EB0527A7F5006784
:1052A00037643E46274440F2FF5C674501D20D2D2E
:1052B0000AD9FF2F8AD2C7433F0703D02DE2BF7818
:1052C0004F44D9E70D2D12D800255F460CE000BFF2
:1052D00006EB050C17F80CC0BCF1000F02D003FA66
:1052E00005FC62446D1CADB2A542F1D3CA62C04355
:1052F0000007E3D1754607E03718EF5D17B103FAF1
:1053000000F73A44401C80B2A042F5D3B3E5CA622C
:10531000BC7804EB002535647879823800EBD070D6
:1053200040108000001D70642E187645C6D20024FF
:105330005E4608E02F19F75DFF0702D003FA04F775
:105340003A44641CA4B28442F4D394E54FEA901C1E
:10535000C6F84CC078795FEAC07806D004EB8C04BC
:1053600004F54054B4F95A4008E0BCF1000F19D0DC
:1053700004EB8C0404F54054B4F94A40BF783C4433
:10538000823800EBD0704010B4648000001D04EB44
:105390000525CA62C6E910502E1876458ED2002423
:1053A0005E460CE0BF780AEB0704E9E72F19F75DCA
:1053B000FF0702D003FA04F73A44641CA4B2844203
:1053C000F4D358E54FEA901CC6F84CC078795FEAF0
:1053D000C07806D004EB8C0404F54054B4F958406E
:1053E00008E0BCF1000F19D004EB8C0404F5405424
:1053F000B4F94840BF783C44823800EBD07040108C
:10540000B4648000001D04EB0525CA62C6E9105093
:105410002E1876458AD200245E460CE0BF7809EB50
:105420000704E9E72F19F75DFF0702D003FA04F735
:105430003A44641CA4B28442F4D31CE57A79802AED
:1054400037D0FB4BF94A4FF4803BD3F890804FF0B4
:10545000804342F6E06EBCF1860F38D0BCF1960F67
:1054600060D0BCF1A60F7AD0BCF1860F32D0BCF16F
:10547000960F75D0BCF1A60F73D0BCF1860F2CD05F
:10548000BCF1960F6ED0BCF1A60F6CD0BCF1860FAC
:1054900026D0BCF1960F67D0BCF1A60F79D0BCF135
:1054A000860F20D0BCF1960F74D0BCF1A60F72D03D
:1054B00057E3BA78706402EB00203064BA793B7A23
:1054C00002EB032200EB0240C6E9122325E07D79BE
:1054D000862D0CD07D79882D7ED07D79842D7CD051
:1054E0007B79822B7AD07B79802B78D039E3BB789B
:1054F000706403EB0020400804EB40033064B3F910
:105500000230002B0BDB4FEA0343CB6234F8105020
:1055100034F810002D0471D4A1E0C86221E334F9FD
:10552000102027E197F805C0BCF1860F1AD3BCF113
:10553000870F15D8BD7883095F4200EB8710F364AD
:10554000706405EB002040083064BCF1860F0CD07D
:1055500004EB830303F54053B3F95A304CE022E0E7
:1055600080E09DE002E19AE0A3E133B104EB830324
:1055700003F54053B3F94A303EE050440346B0646B
:1055800004EB4300B0F9020000283ADA34F9133092
:10559000A2E0EEE16BE29EE2401EC04380B2A2F8C0
:1055A0007C00281AE2E197F805C0BCF1860F76D39B
:1055B000BCF1870F74D8BD7883095F4200EB871078
:1055C000F364706405EB002040083064BCF1860F82
:1055D0000BD004EB830303E020E0B2E0ABE133E265
:1055E00003F54053B3F9583006E043B104EB8303AD
:1055F00003F54053B3F948301844BFE728E0484466
:10560000BCE74FEA0045CD6234F81300000434F8DB
:105610001300C1D4A2F87C0028447EE7BB787064F4
:1056200003EB0020400841F286333064984274D87E
:1056300004EB4005B5F9D237002BFFF670AF4FEA07
:105640000343CB62B5F8D0070004B5F8D00706D500
:10565000401EC04380B2A2F87C00181A86E1A2F86E
:105660007C003BE097F805C0BCF1880F7ED3BCF10D
:10567000890F7CD8BD7883095F4200EB8710F36403
:10568000706405EB002040083064BCF1880F08D03E
:1056900004EB830303F54053B3F95A3008E093E079
:1056A0001EE03BB104EB830303F54053B3F94A30EA
:1056B00018443CE050443AE004EB4503B3F9D20708
:1056C00000283BDB4FEA0044CC62B3F8D00700046B
:1056D000B3F8D00777D401E20BEB004018441CE785
:1056E00097F805C0BCF1880F6ED3BCF1890F14D8B0
:1056F000BD7883095F4200EB8710F364706405EBAB
:10570000002040083064BCF1880F07D004EB83030D
:1057100003F54053B3F95830CAE753E033B104EB13
:10572000830303F54053B3F94830C1E748440546C5
:10573000B06441F286308542BED912E234F91530A8
:10574000CAE7022819D2BB78706403EB0020400836
:105750003064C72836D2374C04EB80035B68002BDB
:1057600006DB1B04CB6254F820003AE12DE031E067
:1057700054F820200BEB034076E0B8788008B6E0C0
:10578000362808D19C8CA4F50044E51704EB9574E9
:1057900002EBA404CC62232803D0292801D02C28B2
:1057A00004D19C8C1444A4F50044CC6224287DD000
:1057B0002E287CD02F287AD0312878D0352877D061
:1057C000372875D0CDE1CBE055E097F805C0BCF1A6
:1057D000840F6ED30CF0FF0CCDF800C0BCF1850F28
:1057E00068D8B44697F802908609774200EB871094
:1057F000CCF84C60CCF8440009EB00204708CCF80A
:1058000040700098842806D004EB860404F54054C8
:10581000B4F95A4006E07EB104EB860404F5405426
:10582000B4F94A40CCF8484009E0000000000020EC
:105830004C2C00203C2500205446CCF848A0022DDA
:1058400014D2E3192546C72B74D2FE4800EB83041B
:105850006468002C04DB7C1900EB84039B88BBE0AC
:1058600050F823200BEB0440104456E69CF84820E7
:1058700002EB99003AE097F805C0BCF1840F78D3A9
:10588000BCF1850F56D8B24697F802E086097742F8
:1058900000EB8710CAF84C60CAF844000EEB0020F9
:1058A0004708CAF84070BCF1840F04E029E02EE0FC
:1058B00036E061E063E006D004EB860404F5405472
:1058C000B4F9584006E046B104EB860404F54054B0
:1058D000B4F94840CAF8484002E04C46CAF848903B
:1058E000022DAED39AF8482002EB9E00C0B2D64AF1
:1058F000332852F82020CA623FF444AF3428FBD04A
:105900003EE7D24800884044A0F5004005E69B8C65
:10591000D418CE4B1B88A3F580332344CB624DE7CC
:10592000CB480088A0F50040C31700EB937002EB52
:10593000A000F2E547E0BB78706403EB0020430869
:105940003364FE2B3FD8C34800EB83046468002C0B
:1059500086DB4FEA0444CC6250F82300030409D5E7
:10596000401EC04380B2A2F87C00201A00F58030AF
:10597000D3E53BE02044D0E57B79822B7DD37D7954
:10598000832D7DD88309BF78C3F1000C00EB8C1008
:10599000F364706407EB002040083064822D06D069
:1059A00004EB830303F54053B3F95A3006E05BB1CF
:1059B00004EB830303F54053B3F94A30184404461B
:1059C000B064FE2802D9CCE05044F8E7A14800EBCF
:1059D00084035B68002B34DB4FEA0343CB6250F84F
:1059E000240004043FF534AE184496E57D79822DF9
:1059F00078D3832D22D88309BF78C3F1000C00EB44
:105A00008C10F364706407EB002040083064822D32
:105A100006D004EB830303F54053B3F9583006E096
:105A20006BB104EB830303F54053B3F948301844DA
:105A30000446B06441F66E008442C7D991E0484400
:105A4000F6E750F8242095E6BB78706403EB00205D
:105A50004FEA5000306434E04FEA004403EB0E009C
:105A6000CC62038800881B043FF57AAF36E004E07F
:105A700006E000BF03EB0E026FE07B79802B70D352
:105A80007D79812D6DD88309BF78C3F1000C00EBBF
:105A90008C10F364706407EB002040083064802DA4
:105AA00006D004EB830303F54053B3F95A3006E004
:105AB00093B104EB830303F54053B3F94A30184420
:105AC000B064FE284DD804EB400342F6E260185E55
:105AD0000028CFDBC0E705E05044F1E7A2F87C00E6
:105AE00020441AE57D79802D3BD3812D39D8830957
:105AF000BF78C3F1000C00EB8C10F364706407EB0B
:105B0000002040083064802D06D004EB830303F5A9
:105B10004053B3F9583006E0DBB104EB830303F5DF
:105B20004053B3F948301844B064FE2819D804EB48
:105B3000400442F6E260205E00280CDB4FEA00439E
:105B400004EB0E00CB620488008824047FF5E4ACEB
:105B50007EE54844E8E704EB0E02B2F90030BBE50D
:105B6000FFE70020BDE8F88F2DE9F04F3A4942F6F3
:105B70001A720C183449951EE031237931F905B0B9
:105B800031F902E0354D03F00F0C00270122E678D1
:105B900089B0A5F18009BCF1050F07D1DFF8C080FD
:105BA000842E6DD0942E66D0A42E79D0DFF8B480E8
:105BB000BCF1080F07D3A8F5C06A842E71D0942ECB
:105BC00070D0A42E6FD0BCF1030F07D8DFF898A0D7
:105BD000842E69D0942E68D0A42E67D0DFF88CA0D4
:105BE000AAF102070597BF1E0497BF1E0397BF1EA9
:105BF0000297BF1E0197BF1E009707F21A770797FB
:105C0000BAF9007006971A4F862E97F859707DD012
:105C1000962E7CD0A62E7BD0862E7AD0962E79D04A
:105C2000A62E78D0862E77D0962E76D0A62E75D03A
:105C3000862E74D0962E73D0A62E72D0862E71D05A
:105C4000962E19E03C2500204C2C0020242C0140ED
:105C5000243401403C21002000C003080001002042
:105C60007110002052180020521D0020325C0020CC
:105C70000000002004E029E072D0A62E71D038E2A6
:105C80006079823800EBD07040108100091DC9F89E
:105C90004410A37858184E28F1D20020EC6A12E084
:105CA00060E09BE0E4E051E1BEE1E3E122E200BF1D
:105CB00002FA00F5254208EB000501D05A5500E034
:105CC0005F55401C80B28842F2D3D8E79E09C9F8DC
:105CD0004C60637948465FEAC37C06D001EB8601DD
:105CE00001F54051B1F95A1006E02EB301EB8601DF
:105CF00001F54051B1F94A10A4782144823B8164F6
:105D000003EBD37149108900091D0CE032E2F7E280
:105D100059E332E277E3D7E332E273E3D3E332E2EB
:105D2000FCE3FCE332E24164D9F8483058184E28CD
:105D3000A5D20020ED6A10E0A4780EEB0401DDE7A7
:105D400002FA00F42C4203EB000402D008F804200D
:105D500001E008F80470401C80B28842F0D38EE75E
:105D6000F8E3F8E39E09C9F84C60637948465FEAB6
:105D7000C37C06D001EB860101F54051B1F9581002
:105D800006E0BEB101EB860101F54051B1F94810C2
:105D9000A4782144823B816403EBD37149108900CC
:105DA000091D4164D9F8483058184E288DD200207A
:105DB000EC6A10E0A4780BEB0401EBE702FA00F5C3
:105DC000254203EB000502D008F8052001E008F8A1
:105DD0000570401C80B28842F0D350E70D2B05D8E7
:105DE000F849A07801EB0321014400E0A178C9F84B
:105DF0004010607940F2FF56823800EBD0704010BE
:105E00008000001D0C18C9F84400B44201D20D2BCB
:105E100004D9FF2CA3D20F2B17D030E700248946DA
:105E2000D5F82CB00EE000BF02FA04F616EA0B0F0C
:105E300009EB040C02D00AF80C2001E00AF80C70FF
:105E4000641CA4B28442EFD3E5E70023ED6A0CE0C2
:105E500002FA03F42C4201EB030402D008F80420F8
:105E600001E008F804705B1C9BB28342F0D306E7A4
:105E70009809C9F84C006679B346F6074E4606D035
:105E800001EB800000F54050B0F95A0006E050B335
:105E900001EB800000F54050B0F94A00A1780844B9
:105EA000C9F84800ABF1820000EBD07040108000D0
:105EB000001D7064B46C3146BCF10D0F03D804EBC7
:105EC0000C24A4F500640C642146044440F2FF56FF
:105ED000B44202D2BCF10D0F0CD9FF2C9DD2DC4391
:105EE000240704D0CBE6A1780EEB0100D8E7BCF183
:105EF0000D0F15D800248946D5F82CB00EE000BF50
:105F000002FA04F616EA0B0F09EB040C02D00AF8A9
:105F10000C2001E00AF80C70641CA4B28442EFD398
:105F2000DB431B07A3D1EC6A0DE000BF02FA03F5C7
:105F3000254201EB030502D008F8052001E008F82E
:105F400005705B1C9BB28342F0D398E69809C9F8B0
:105F50004C006679B646F6074E4606D001EB800047
:105F600000F54050B0F9580006E050B301EB800056
:105F700000F54050B0F94800A1780844C9F848003D
:105F8000AEF1820000EBD07040108000001D706404
:105F9000B46C3146BCF10D0F03D804EB0C24A4F50E
:105FA00000640C642146044440F2FF56B44202D21D
:105FB000BCF10D0F0CD9FF2C94D2DC43240704D084
:105FC0005DE6A1780BEB0100D8E7BCF10D0F15D809
:105FD00000248946D5F82CB00EE000BF02FA04F682
:105FE00016EA0B0F09EB040C02D00AF80C2001E0B2
:105FF0000AF80C70641CA4B28442EFD3DB431B0785
:10600000A3D1ED6A0DE000BF02FA03F42C4201EBCC
:10601000030402D008F8042001E008F804705B1CB7
:106020009BB28342F0D364E0A07800EB0321C9F86F
:106030004010637940F2E730823B03EBD3735B108F
:106040009B001B1DCC18C9F844308442B8D20020F4
:106050005446EE6A0BE000BF02FA00F5354201EB50
:10606000000501D0625500E06755401C80B298429F
:10607000F2D33EE09E09C9F84C60637948465FEA76
:10608000C37806D001EB860101F54051B1F95A10F1
:1060900006E0EEB101EB860101F54051B1F94A107D
:1060A000A4782144823B816403EBD37149108900B9
:1060B000091D4164836C40F2E73003EB0C235C184C
:1060C000C9F840308442AED2EE6A002055460EE058
:1060D000A4780EEB0401E5E702FA00F4344203EB86
:1060E000000401D02A5500E02F55401C80B28842A0
:1060F000F2D32EE29E09C9F84C60637948465FEA04
:10610000C37806D001EB860101F54051B1F9581072
:1061100006E0EEB101EB860101F54051B1F94810FE
:10612000A4782144823B816403EBD3714910890038
:10613000091D4164836C40F2E73003EB0C235C18CB
:10614000C9F84030844294D200205446EE6A0EE0F2
:10615000A4780BEB0401E5E702FA00F5354203EB06
:10616000000501D0625500E06755401C80B28842AE
:10617000F2D3EEE16679862E0CD06679882E7CD03B
:106180006679802E7AD06679842E78D06679822ED0
:1061900076D0DEE194F802C0C9F844300CEB03235A
:1061A0005B08C9F84030542F0ED0562F2ED05C2FEC
:1061B0004BD05E2F65D0082874D314F8080C8028C3
:1061C00075D171E000F8FFFFE86A48B1F74CA042D2
:1061D00004DB64422044E86288F8162010B103E032
:1061E00088F8142088F8142004464FF4616290FB6C
:1061F000F2F002FB10423C2692FBF6F421F8130069
:1062000001EB430006FB14214480A0E1E86A00286A
:1062100018D004DAE54C2044E86288F815200446DA
:106220004FF4616094FBF0F200FB124021F8132060
:106230004FF03C0490FBF4F201EB430104FB12002D
:106240004A80ACE188F81420E9E74FF0000041F201
:10625000827200BFA2EB000431F8145003EB00047B
:1062600000F1010080B221F814500528F2D901EBA9
:106270004301BAF8000088816BE1EBE040E2F4E30F
:10628000F4E3002041F282721C18151A401C31F808
:10629000144080B221F815400528F5D901EB4300E0
:1062A00081892AE128E002E014F8072C12B3EA6A97
:1062B00021F81320D71702EB17473C2804D03E28BB
:1062C00009D0802812D044E114F8070C08B1102836
:1062D000D2D1381406E014F8070C08B11028CBD13D
:1062E000B9F8540001EB4301488032E114F8070C7F
:1062F0000028C1D1EB622CE1A88D21F8130028E120
:106300006779862F7ED3872F7DD89E0994F80280E7
:10631000C6F1000C03EB8C13C9F84C60C9F844308B
:1063200008EB03235B084A46C9F84030862F06D0A5
:1063300001EB860606F54056B6F95A6006E076B1DE
:1063400001EB860606F54056B6F94A60334493647D
:10635000082830D314F8083C802B06D101E07344A0
:10636000F5E714F8070C002870D0906C41F26F76B6
:10637000B0426CD93C2B6BD03E2B6AD0802B15D011
:10638000E7E0102A9FD100BF41F26E7290427DD9A2
:10639000DFE0102B97D100BF41F26E73984276D99F
:1063A000D7E000BF01EB40004280D2E014F8070CB8
:1063B0000028D9D0CDE0184641F26F7237E3AA8D9C
:1063C00021F81020C5E06779862F7CD3872F7BD8F2
:1063D0009E0994F80280C6F1000C03EB8C13C9F8F7
:1063E0004C60C9F8443008EB03235B084A46C9F8FF
:1063F0004030862F08D001EB860606F54056B6F9E8
:10640000586008E091E10FE176B101EB860606F5F0
:106410004056B6F94860334493640828CBD314F847
:10642000086C802E06D101E05B44F5E714F8070CF8
:10643000002899D0184641F26F73984270D93C2ECB
:1064400006D03E2E05D0802EB0D082E00CE317E1BE
:106450004AE14FE194F802C0C9F844300CEB032341
:106460005B0841F2813CC9F840305C2F15D05E2FAB
:106470002ED041F2853C542F42D0562F6FD041F29E
:106480008732082869D3934268D801E0C4E2CBE29E
:1064900014F8086C802E7CD18AE0634585D80020F2
:1064A00041F28272141A31F814501C1801EB4404A2
:1064B000401C80B2A4F8D0570528F3D9BAF80000E0
:1064C00001EB430101E059E1DEE0A1F8DC0740E027
:1064D0006345BAD8002041F282721C18151A01EBEC
:1064E0004404401CB4F8D04780B221F81540052878
:1064F000F3D901EB4300B0F8DC17AAF8001019E259
:106500006345A2D8E86A60B1284CA04204DB64422B
:106510002044E86288F8162028B106E0A7E20AE3E2
:10652000DEE088F8142088F814204FF4616490FBB2
:10653000F4F2064601EB430000F5FA6004FB126139
:1065400002803C2391FBF3F203FB12114280E962CB
:10655000818014E2D6E3FDE301E05DE039E06345CC
:10656000B5D8E86A00281DD004DA104C2044E8624F
:1065700088F8152004464FF4616290FBF2F001EBBD
:10658000430101F5FA6102FB104208804FF03C0321
:1065900000E010E092FBF3F0488003FB1020E8627B
:1065A0008880ECE188F81420E4E7000080510100C5
:1065B00014F8070C58B3E86A01EB43014FEAE0779F
:1065C000804600EB1747A1F8D0873C2E06D03E2E20
:1065D0000DD014F8080C802815D0D0E114F8070C61
:1065E00008B11028B5D19342B3D2381408E014F89A
:1065F000074C0CB1102CACD19342AAD2B9F854007C
:10660000A1F8D207BBE114F8070C0028A1D163451B
:106610009FD803F57A736DE693429AD801EB430154
:10662000A88DA1F8D007AAE16779882F7DD3892F9B
:106630007CD89E0994F80280C6F1000C03EB8C1301
:10664000C9F84C60C9F8443008EB03235B084A469C
:10665000C9F84030882F06D001EB860606F5405673
:10666000B6F95A6006E046B101EB860606F54056DB
:10667000B6F94A6003F57A7368E603F57A736EE655
:10668000EE6A21F8106075E66779882F76D3892F36
:1066900087D89E0994F80280C6F1000C03EB8C1396
:1066A000C9F84C60C9F8443008EB03235B084A463C
:1066B000C9F84030882F06D001EB860606F5405613
:1066C000B6F9586006E046B101EB860606F540567D
:1066D000B6F9486003F57A739DE603F57A73A3E68D
:1066E000EB6A21F81030AAE614F8072C002A3FF4D0
:1066F0004BAE46E614F8073C002B3FF44DAE48E69F
:1067000094F802C0C9F844300CEB03235B084E46F2
:10671000C9F8403042F6EC6942F6E06C5C2F15D0C7
:106720005E2F2CD042F6E26901E029E12BE142F62E
:10673000E46A542F39D0562F5CD008287CD3FF2B25
:106740007BD814F8080C80287FD17BE0F92B9FD8E8
:10675000002041F28272141A1D1801EB4505401CFD
:1067600031F8144080B225F80C400528F3D901EB2C
:106770004301BAF8002021F8092000E15BE1F92B80
:10678000FBD8002041F282721C18151A01EB440458
:10679000401C34F80C4080B221F815400528F3D98C
:1067A00001EB430131F80910A7E6FD2BE5D8E86AB3
:1067B00048B1FA4CA04204DB64422044E86288F805
:1067C000162010B103E088F8142088F8142004463D
:1067D0004FF4616290FBF2F001EB430302FB1042C5
:1067E00023F80C003C2092FBF0F100FB112023F871
:1067F00009101DE0FD2BC0D8E86A00281FD004DA7C
:10680000E64C2044E86288F8152004464FF46162A3
:1068100090FBF2F001EB430302FB104123F80C0064
:106820004FF03C0291FBF2F023F8090002FB10103C
:10683000E86223F80A00AAE373E00BE005E088F8B9
:106840001420E2E714F8070C20B101EB4302E86AD8
:1068500022F80C00B246FE2B56D814F8080C3C283F
:1068600006D03E2813D03C281CD03E281AD04BE03E
:1068700014F8070C08B11028DDD1E86A01EB4301D8
:10688000C21700EB1240021421F809200AE014F8A4
:10689000070C08B11028CED101EB4302BAF854001E
:1068A00022F8090014F8070C08B110282CD15B1C41
:1068B0000D2B29D3122B27D80598B9491C22B0F9E2
:1068C000000048610498B0F90000401E0861039878
:1068D000B0F90000C86081460298B0F900008860F5
:1068E00080460198B0F90000486007460098B0F96A
:1068F00000600E60684607991BF041FD4B4642461A
:106900003946304619F082F914F8080C802892D1E3
:10691000DAF84000FD288ED841F270710844E86230
:1069200035E301EB4301A88D21F80C000D2BF7D3C3
:10693000122BF5D805981C22B0F900109848416137
:106940000499B1F90010491E01610399B1F9007071
:10695000C7600299B1F9006086600199B1F90050F1
:1069600045600099B1F900400460684607991BF042
:1069700006FD3B4632462946204619F047F906E314
:106980006279802A43D394F80580B8F1810F6ED8DC
:106990009E09A778C6F1000C03EB8C13C9F84C6074
:1069A000C9F8443007EB03235B084A46C9F8403076
:1069B000B8F1800F05D001EB860643F25A07F75F66
:1069C00005E04EB101EB860643F24A07F75F41F25C
:1069D000707633443B445CE041F270773B4473444F
:1069E00057E000BF14F8070CF0B341F66E071846E5
:1069F000BB4202D8EB6A21F810303C2E51D03E2E1B
:106A00007FF421AD14F8073C63B1102B0AD0BEE22D
:106A1000102A0FD1B8420DD8EA6AD31702EB1342FD
:106A20001214BFE4B84205D8B9F85420BAE4904231
:106A30007FF6C5ACABE26779802F65D3812F7AD81A
:106A40009E0994F80280C6F1000C03EB8C13C9F880
:106A50004C60C9F8443008EB03235B084A46C9F888
:106A60004030802F0AD003E020E026E062E1D1E050
:106A700001EB860643F25807F75FA8E72EB101EB5A
:106A8000860643F24807F75FA1E741F270773B447F
:106A90005B44936408280CD314F8086C802EA4D1AE
:106AA000A0E714F8072C002AB4D0B1E7D9F84800C1
:106AB00035E7184641F66F02B9E794F802C0C9F805
:106AC00044300CEB03235B08C9F840305C2F1CD02A
:106AD0005E2F31D0542F43D0562F65D0C82B13D200
:106AE000E96ACA1701EB1242150C2D044D1B2D4902
:106AF000C72B41F8235007D2082805D314F8080CF7
:106B00003C2877D03E287BD041E2C12B12D8254AC1
:106B1000002041F28274251A31F915601D18401CBD
:106B200080B242F825600528F5D900BF02EB830149
:106B3000069888612BE2C6E0C12B55D8194A00207F
:106B400041F282741D18261A401C32F8255080B27A
:106B500021F816500528F5D902EB8300018BCCE40F
:106B6000C52B41D8E86A48B10C49884204DB494248
:106B70000844E86288F8162010B103E088F8142071
:106B800088F814204FF4616290FBF2F40146054846
:106B900002FB141240F823401BE005E08051010085
:106BA000306300203C250020C52B1DD8E86A002852
:106BB0001DD004DAF8490844E86288F815204FF43B
:106BC000616190FBF1F20446F44840F8232001FB98
:106BD00012424FF03C0192FBF1F400EB830001FB09
:106BE00014214460E9628160D1E103E008E088F8A3
:106BF0001420E4E714F8070C98B3102831D0C6E14C
:106C000014F8070C70B310282CD0C0E101EB8301FD
:106C10004860BCE16779842F74D3852F73D89E09AF
:106C200094F80280C6F1000C03EB8C13C9F84C6099
:106C3000C9F8443008EB03235B084A46C9F84030E2
:106C4000842F06D001EB860101F54051B1F95A10AD
:106C500061E046B101EB860101F54051B1F94A10FE
:106C600059E0FAE0FCE00EEB0301082891640846C5
:106C700024D3C72809D8E96ACB1701EB13436FF374
:106C80000F03CB1AC54941F8203014F8081C3C29E1
:106C900046D03E2949D07AE110296BD1C62869D85F
:106CA000E96ACA1701EB12410A1405E0102961D103
:106CB000C6285FD8D9F85420B84928E1C72859D840
:106CC000B649EA6A2BE16779842F43D3852F51D8DF
:106CD0009E0994F80280C6F1000C03EB8C13C9F8EE
:106CE0004C60C9F8443008EB03235B084A46C9F8F6
:106CF0004030842F08D001EB860101F54051B1F9F5
:106D0000581008E0AFE0B1E03EB101EB860101F5BB
:106D10004051B1F948101944A7E70BEB0301A4E770
:106D200014F8071C0029B9D0B6E714F8071C00298D
:106D3000BED0BBE794F802C0C9F844300CEB032383
:106D40005B08C9F840305C2F15D05E2F24D0542F3B
:106D500038D000E0E6E0562F5BD0E96ACA1701EBB5
:106D60001242150C2D044D1B8D49FF2B41F8235069
:106D7000FFF4C2AE0BE1F92B4AD8894A002041F258
:106D80008274251A31F915601D18401C80B242F832
:106D900025600528F5D9C9E6F92B39D8804A0020A5
:106DA00041F282741D18261A401C32F8255080B218
:106DB00021F816500528F5D902EB8300008BAAF8BC
:106DC0000000B7E5FD2B23D8E86A48B17249884234
:106DD00004DB49420844E86288F8162010B103E059
:106DE00088F8142088F8142001464FF4616091FB64
:106DF000F0F46B4A00FB141042F823403C2190FB56
:106E0000F1F402EB830201FB14005460E86290602D
:106E1000BDE0FD2B1DD8E86A00281BD004DA5E49CE
:106E20000844E86288F8152002464FF4616092FB3E
:106E3000F0F45B4900FB142241F823404FF03C0082
:106E400092FBF0F401EB830100FB14204C60E8623C
:106E500088609CE088F81420E6E74FEA2240D5E6F7
:106E6000D9F85400D2E66279822A3ED394F805809C
:106E7000B8F1830F39D89E09A778C6F1000C03EB4F
:106E80008C13C9F84C60C9F8443007EB03235B0846
:106E90004A46C9F84030B8F1820F06D001EB8601AE
:106EA00001F54051B1F95A1062E036B101EB8601AB
:106EB00001F54051B1F94A105AE00EEB03010828E0
:106EC0009164084627D3FF2809D8E96ACB1701EB5C
:106ED00013436FF30F03CB1A314941F8203014F8F4
:106EE000081C3C2949D03E294CD050E010294ED1F5
:106EF000FE284CD8E96ACA1701EB12410A1405E0D2
:106F0000102944D1FE2842D8D9F85420244901EB55
:106F1000800042603BE0FF2839D82149EA6A41F805
:106F2000202034E06779822F31D3832F2FD89E0918
:106F300094F80280C6F1000C03EB8C13C9F84C6086
:106F4000C9F8443008EB03235B084A46C9F84030CF
:106F5000822F06D001EB860101F54051B1F958109E
:106F600006E03EB101EB860101F54051B1F9481050
:106F70001944A4E70BEB0301A1E714F8071C00294F
:106F8000B6D0B3E714F8071C0029BBD0B8E709B0A6
:106F90000020BDE8F08F0000805101003C2500205A
:106FA0003C2100202DE9F04FFE49FF4D084442F6F8
:106FB0001A718B1E027935F901B035F903A0DFF89B
:106FC000EC9302F00F0C01230021C7788DB009F17A
:106FD0008004BCF1050F06D1F54E842F43D0942FC9
:106FE00060D0A42F7ED0BCF1080F07D3DFF8C4E334
:106FF000842F78D0942F77D0A42F76D0BCF1030FB4
:1070000007D8DFF8B4E3842F70D0942F6FD0A42F6B
:107010006ED0DFF898834FF40041A8F18008CE03CA
:1070200098F859304FF0FF3E862F6ED0962F6DD0D6
:10703000A62F6CD0862F6BD0962F6AD0A62F69D042
:10704000862F68D0962F67D0A62F71D0862F70D04C
:10705000962F6FD0A62F6ED0862F6DD0962F6CD026
:10706000A62F6BD0EBE34279823A02EBD272521038
:107070009200121DC9F844208578A8184E28F1D234
:107080000020E46A0BE000BF03FA00F7274206EB9A
:10709000000701D0EB5500E0E955401C80B290425A
:1070A000F2D3DFE74FEA921CC9F84CC047794A4651
:1070B0005FEAC77806D005EB8C0505F54055B5F9B4
:1070C0005A5008E0BCF1000F27D005EB8C0505F500
:1070D0004055B5F94A5080782844823F906407EBC8
:1070E000D77006E031E06DE0B8E025E1A4E1C9E148
:1070F00008E2401085002D1D5564D9F8482050192C
:107100004E28AFD20020E46A1CE03BE215E3FDE329
:107110003BE293E3FBE33BE28FE380785844DCE718
:1071200003FA00F7274202EB000708D0F35507E007
:10713000EEE330E2EDE3EDE330E2ECE3ECE3F155D6
:10714000401C80B2A842EBD38CE74FEA921CC9F8EE
:107150004CC047794A465FEAC77806D005EB8C05F4
:1071600005F54055B5F9585008E0BCF1000F17D0AF
:1071700005EB8C0505F54055B5F948508078284455
:10718000823F906407EBD770401085002D1D556439
:10719000D9F8482050194E28D6D20020E46A0EE0D3
:1071A00080785044ECE700BF03FA00F7274202EB77
:1071B000000701D0F35500E0F155401C80B2A84211
:1071C000F2D34FE70D2A05D87C4E857806EB0226D0
:1071D0002E4400E08678C9F8406040799A468238AB
:1071E00000EBD07040108000001D3346351840F28F
:1071F000FF56C9F84400B54201D20D2A04D9FF2D2B
:10720000A2D20F2A16D02DE70025D4F82C800EE04C
:107210000AFA05F717EA080F04D003EB050C0EF87D
:107220000CA002E05F190EF807106D1CADB285428C
:10723000EED3E6E7E76A0022614D54460BE000BF5B
:1072400004FA02F63E4203EB020601D0AC5500E020
:10725000A955521C92B28242F2D303E79709C9F8AA
:107260004C7046795FEAC678C84606D005EB8705BC
:1072700005F54055B5F95A5006E067B305EB8705AB
:1072800005F54055B5F94A5080782844823EC9F842
:10729000480006EBD67040108000001DC8F844007E
:1072A0009A46D8F848504346BCF10D0F03D805EB79
:1072B0000C25A5F500651D642B46054440F2FF56DC
:1072C000B54202D2BCF10D0F0BD9FF2D9BD2D54395
:1072D0002D0703D0C6E680785844D7E7BCF10D0FE0
:1072E00015D80025D4F82C800FE000BF0AFA05F766
:1072F00017EA080F04D003EB050C0EF80CA002E00F
:107300005F190EF807106D1CADB28542EED3D24363
:107310001207A2D1E66A2A4D54460AE004FA02F79F
:10732000374203EB020701D0EC5500E0E955521C4F
:1073300092B28242F2D395E69709C9F84C70467929
:107340005FEAC678C84606D005EB870505F54055C7
:10735000B5F9585006E027B305EB870505F540550C
:10736000B5F9485080782844823EC9F8480006EBB9
:10737000D67040108000001DC8F844009A46D8F826
:1073800048504346BCF10D0F03D805EB0C25A5F57D
:1073900000651D642B46054440F2FF56B54214D2E9
:1073A00010E018E000C003082C2D00208000002011
:1073B0007110002052120020521D002000F8FFFF23
:1073C00052180020BCF10D0F0BD9FF2DB3D2D543BD
:1073D0002D0703D046E680785044C5E7BCF10D0F79
:1073E00015D80025D4F82C800FE000BF0AFA05F765
:1073F00017EA080F04D003EB050C0EF80CA002E00E
:107400005F190EF807106D1CADB28542EED3D24362
:10741000120790D1E66AFB4D54460AE004FA02F7DF
:10742000374203EB020701D0EC5500E0E955521C4E
:1074300092B28242F2D315E6857805EB0225C9F8AF
:107440004050407940F2E732823800EBD070401073
:107450008000001D2E18C9F844009642BAD2E76A8F
:10746000002274460BE000BF03FA02F63E4205EB31
:10747000020601D0A35500E0A155521C92B28242EF
:10748000F2D3EFE59709C9F84C7046794A465FEAAE
:10749000C67806D005EB870505F54055B5F95A5075
:1074A00006E0EFB105EB870505F54055B5F94A5003
:1074B00080782844823E906406EBD67040108500A8
:1074C0002D1D5564906C00EB0C26721940F2E730CC
:1074D000C9F840608242AED2E76A002074460EE0EE
:1074E00080785844E6E700BF03FA00F23A4206EB20
:1074F000000201D0A35400E0A154401C80B2A84275
:10750000F2D3AFE59709C9F84C7046794A465FEA6D
:10751000C67806D005EB870505F54055B5F95850F6
:1075200006E0EFB105EB870505F54055B5F9485084
:1075300080782844823E906406EBD6704010850027
:107540002D1D5564906C00EB0C26721940F2E7304B
:10755000C9F84060824294D200207246E76A0EE089
:1075600080785044E6E700BF03FA00F43C4206EBA3
:10757000000401D0135500E01155401C80B2A84210
:10758000F2D36FE54779862F0CD04779882F7DD0CD
:107590004779802F7BD04579842D79D04179822914
:1075A00077D05FE58078494600EB02204008C9E9C2
:1075B00010023D2B12D03F2B7CD0E16A25F8101031
:1075C0004FEAE172002901EB124201DB111401E0E4
:1075D0000EEB224105EB4000418043E58A6D002A15
:1075E00009DBD31702EB13431E0C3604961B1B1446
:1075F000C4E90D6305E0531EDB431E0C9BB2C4E9D6
:107600000D36D9F85C10002909DBCB1701EB1343C9
:107610001E0C36048E1B1B14C4E90F6305E04B1EC1
:10762000DB431E0C9BB2C4E90F36E76B666BD217C7
:1076300007FB06F325F810304FEA1348C4F84480DE
:10764000D4F838C007FB0C87A764236C03FB0677CC
:1076500005EB400677803F0C03FB0C73C4E9137302
:10766000B3801B14F380B2EBE17F8AD035F8104071
:107670007188B288E443C943D243DB43641C2404C9
:1076800089B292B29BB2240C0FD104E02AE2FDE34E
:10769000FDE3FDE30EE0491C0904090C05D1521C71
:1076A0001204120C01D15B1C9BB225F810407180B2
:1076B000B280F4E08A6D002A01DB626302E0531EAF
:1076C000DB436363D9F85C10002901DBA16302E0AE
:1076D0004B1EDB43A363D4E90D76B7FBF6F306FB41
:1076E0001376C4E90F3625F810301C1405EB40035F
:1076F000D2175C809E803614DE80B2EBE17FB4D07E
:10770000998835F810405A88C943E4438FB2D24370
:10771000F143641C240492B289B2240C01D1521C9E
:1077200092B27F1C3E04360C01D1491C89B225F867
:1077300010405A809E80D98094E44779862F7CD36C
:10774000872F7BD891098678C1F1000C02EB8C124F
:10775000C9F8442006EB02225208C9F84C104846EA
:10776000C9F84020862F06D005EB810101F5405174
:10777000B1F95A1006E071B105EB810101F54051F4
:10778000B1F94A10114481643D2B15D03F2B7DD0B7
:1077900041F28630B4E20BEB0201F4E7E06A25F82F
:1077A00011004FEAE072002800EB12426FDB101468
:1077B00005EB4101488055E40A4641F284318A4292
:1077C000BAD8816D002909DBCB1701EB13431E0CDE
:1077D00036048E1B1B14C4E90D6305E04B1EDB430E
:1077E0001E0C9BB2C4E90D36D9F85C0000280BDBF7
:1077F000C31700EB13431E0C3604861B1B14C4E98D
:107800000F6307E052180020431EDB431E0C9BB29F
:10781000C4E90F36E76B666B07FB06F325F81230F9
:107820004FEA1348C4F84480D4F838C007FB0C87EB
:10783000A764236C03FB067702E0AFE230E250E17D
:1078400005EB4206C91777803F0C03FB0C73C4E9B4
:107850001373B3801B14F380B1EBE07FABD035F82A
:1078600012407188B088E443C943C043DB43641CC1
:10787000240489B280B29BB2240C0CD1491C0904A7
:10788000090C08D1401C0004000C01E009E0FDE3F4
:1078900001D15B1C9BB225F812407180B080F3804F
:1078A00052E40B4641F284318B4284D8816D002929
:1078B00001DB616302E04A1ED2436263D9F85C00D7
:1078C000002801DBA06302E0421ED243A263D4E998
:1078D0000D76B7FBF6F206FB1276C4E90F2625F803
:1078E0001320171405EB4302C917578096803614EE
:1078F000D680B1EBE07FD3D035F813009188C44334
:10790000F843C9438FB280B2F14306E015E096E038
:1079100094E0FDE3FDE3FDE3FDE3641C260489B28E
:10792000360C01D1401C80B27F1CBCB2F4E300BF16
:1079300025F8136050809480EFE34779862F7DD33C
:10794000872F7CD891098678C1F1000C02EB8C124C
:10795000C9F8442006EB02225208C9F84C104846E8
:10796000C9F84020862F06D005EB810101F5405172
:10797000B1F9581006E0B1B105EB810101F54051B4
:10798000B1F94810114481643D2B0FD03F2B7FF497
:10799000FFAE0B4641F284318B4286D8816D0029BF
:1079A00063DB616364E00AEB0201ECE70A4641F243
:1079B0008431A9E1816D00297EDBCB1701EB1343F4
:1079C0001E0C36048E1B1B14C4E90D63D9F85C0031
:1079D000002872DBC31700EB13431E0C3604861B12
:1079E0001B14C4E90F63E76B666BC91707FB06F34B
:1079F00025F812304FEA1348C4F84480D4F838C050
:107A000007FB0C87A764236C03FB067705EB420694
:107A100077803F0C03FB0C73C4E91373B3801B1412
:107A2000F380B1EBE07F5CD0708835F81240B1880C
:107A3000C043E443C94380B289B201E029E2AFE127
:107A4000DB43641C24049BB2240C09D1401C0004B9
:107A5000000C05D1491C0904090C01D15B1C9BB227
:107A600025F812407080B18019E74A1ED243626344
:107A7000D9F85C00002801DBA06302E0421ED2437B
:107A8000A263D4E90D76B7FBF6F206FB1276C4E9E1
:107A90000F2625F81320171405EB4302C91757804A
:107AA00096803614D680B1EBE07FBCD035F8131049
:107AB0009088CC43F94301E0FAE3FAE3C04387B28C
:107AC000F043641C240489B280B2240C01D1491C07
:107AD00089B27F1CBEB25BE125F8134051809680CD
:107AE000D080E0E18078494600EB02204008C9E9F7
:107AF00010023D2B17D03F2B7DD041F286318842BA
:107B0000EFD8E16A05EB40004FEAE172002901EB92
:107B10001242A0F8D01701DB111401E00EEB224154
:107B2000A0F8D217BFE141F284329042D9D88A6DD1
:107B3000002A09DBD31702EB13431E0C3604961BF5
:107B40001B14C4E90D6305E0531EDB431E0C9BB2FE
:107B5000C4E90D36D9F85C1000290ADBCB1701EB1C
:107B600013431E0C36048E1B1B14C4E90F633346EB
:107B700005E04B1EDB431E0C9BB2C4E90F36666B5F
:107B800005EB400003FB06F7A0F8D0773F0C6764D5
:107B9000A56BD21703FB0577A764236C06FB03765E
:107BA000A0F8D267360C03FB0563C4E91363A0F8A1
:107BB000D4371B14A0F8D637B2EBE17F91D0B0F8E0
:107BC000D047B0F8D217B0F8D427E443C943D24322
:107BD000DB43641C240489B292B29BB2240C09D109
:107BE000491C0904090C05D1521C1204120C01D1C4
:107BF0005B1C9BB200E006E000F5FA600480418067
:107C00008280C3804FE141F2843290428AD88A6DEB
:107C1000002A01DB626302E0531EDB436363D9F891
:107C20005C10002901DBA16302E04B1EDB43A36370
:107C3000D4E90D76B7FBF6F306FB1376C4E90F36ED
:107C400005EB4000D217A0F8D0371B14A0F8D237AC
:107C50003314A0F8D467A0F8D637B2EBE17FD1D0C7
:107C6000B0F8D417B0F8D047C943B0F8D2278DB2D6
:107C7000E443D943D243641C230492B289B21B0C5F
:107C800001D1521C92B26D1C2C04240C01D1491C50
:107C900089B200F5FA60038042808480C18002E1ED
:107CA0004779882F7AD3892F79D896098178C6F1B8
:107CB000000C02EB8C1201EB02214908C9F84C6060
:107CC000C9E910124846882F06D005EB860202F556
:107CD0004052B2F95A2006E076B105EB860202F571
:107CE0004052B2F94A2001F57A71114481643D2B6A
:107CF00072D03F2B71D10BE001F57A715944F5E751
:107D000081427FF64BADCEE08A427FF653AECAE0A9
:107D10000B4641F26C718B42C1D8816D002901DBA9
:107D2000616302E04A1ED2436263D9F85C00002816
:107D300001DBA06302E0421ED243A263D4E90D76C8
:107D4000B7FBF6F206FB1276C4E90F2625F81320DE
:107D5000141405EB4302C917548096803614D6805C
:107D6000B1EBE07F9BD035F813109088CF43C04330
:107D7000E1431FFA80FCF0437F1C3C0489B280B2CF
:107D8000240C01D1491C89B20CF1010C1FFA8CF6AC
:107D9000002E7FF4A1AE401C80B29DE6E6E1E8E152
:107DA0004779882F75D3892FADD896098178C6F188
:107DB000000C02EB8C1201EB02214908C9F84C605F
:107DC000C9E910124846882F08D005EB860202F553
:107DD0004052B2F9582008E016E00EE086B105EBFB
:107DE000860202F54052B2F9482001F57A71114439
:107DF00081643D2B08D03F2B0AD041F26E707FE7A3
:107E000001F57A715144F3E70A4641F26C717BE760
:107E10000B4641F26C718B42C6D8816D002901DBA3
:107E2000616302E04A1ED2436263D9F85C00002815
:107E300001DBA06302E0421ED243A263D4E90D76C7
:107E4000B7FBF6F206FB1276C4E90F2625F81320DD
:107E5000141405EB4302C917548096803614D6805B
:107E6000B1EBE07F1FD09788E14335F81300FC4366
:107E7000C043A7B2F443401C000489B2A4B2000C72
:107E800001D1491C89B27F1C3E0403E00CE0F8E2FA
:107E9000ECE35CE2360C01D1641CA4B225F81300BB
:107EA00051809680D48006E28178FE4801EB022161
:107EB0004908C0E910123D2B7DD03F2B7CD0FF2913
:107EC000F1D2E06A42F6E0674FEAE072002800EB88
:107ED0001242064605EB4100C65303DB1614BA1CDA
:107EE000865204E00EEB224242F6E2668253EE4EE8
:107EF00042F6047006EB0008801E06EB000B001F24
:107F000006EB000A801E06EB0009801E06F53C57B2
:107F10000644E6480B900D2924D3122922D81038A4
:107F2000B8F900104161BBF900101C22491E016123
:107F3000B7F90010C1600A91BAF900108160099187
:107F4000B9F9001041600891B6F90010016007917D
:107F500068460B991AF013FA0DF11C0CBCE80F00DF
:107F600017F054FECF48006C401C0D2827D3122870
:107F700025D8CE49B8F9000010391C224861BBF958
:107F80000000401E0861B7F90000C8608346BAF9D6
:107F9000000088608046B9F900004860B6F90060CA
:107FA00007460E6068460B991AF0E9F95B464246AF
:107FB0003946304601E00BE083E017F027FEB94870
:107FC000803890F859003D2802D03F287AD0E5E368
:107FD000B448036CFC2BFAD8816D002909DBCA1761
:107FE00001EB1242160C36048E1B1214C4E90D620A
:107FF00005E04A1ED243160C92B2C4E90D26C06DAC
:1080000000280ADBC21700EB1242160C3604861B4E
:108010001214C4E90F62324605E0421ED243160C28
:1080200092B2C4E90F2605EB4303666B42F6E065A6
:108030001D4402FB06FCA5F800C04FEA1C4CC4F826
:1080400044C0A76BC91702FB07CCC4F848C0226C18
:1080500006FB02C642F6E26C9C44ACF80060360CAB
:1080600002FB0762C4E9136242F6E4641C4442F670
:10807000E666228012143344B1EBE07F1A80A6D06A
:108080002988BCF800002688C94300E095E1C04378
:10809000F643D243491C090480B2B6B292B2090C2D
:1080A00009D1401C0004000C05D1761C3604360CA6
:1080B00001D1521C92B22980ACF8000026801A80AF
:1080C0006CE3FFE77748066CFC2EF9D8816D002938
:1080D00001DB616302E04A1ED2436263C06D002887
:1080E00001DBA06302E0421ED243A263D4E90D7318
:1080F000B7FBF3F203FB1273C4E90F2305EB46044D
:1081000042F6E065254442F6E2662A80121405E054
:10811000B0E09FE17CE2E1E212E1B0E1A719B61C18
:1081200026443A80338042F6E66C1B146444C91737
:108130002380B1EBE07FC3D028883188C043D2438D
:10814000C943DB43401C000492B289B29BB2000CCD
:1081500001D1521C92B2491C0904090C01D15B1CCB
:108160009BB228803A803180238017E34779802FA3
:10817000A6D3FFB2812F7DD891098678C1F1000C7A
:1081800002EB8C12C9F8442006EB02225208C9F80F
:108190004C104846C9F84020802F05D005EB8101DE
:1081A00043F25A068E5F05E071B105EB810143F29F
:1081B0004A068E5F41F270711144314481643D2B57
:1081C00008D03F2B76D17EE041F2707632440BEB43
:1081D0000201F3E70A4641F66C018A426BD8816DD1
:1081E000002909DBCB1701EB13431E0C36048E1B51
:1081F0001B14C4E90D6305E04B1EDB431E0C9BB250
:10820000C4E90D36D9F85C00002809DBC31700EB80
:1082100013431E0C3604861B1B14C4E90F6305E0D0
:10822000431EDB431E0C9BB2C4E90F36E76B666B43
:10823000C91707FB06F325F812304FEA1348C4F8B4
:108240004480D4F838C007FB0C87A764236C03FB79
:10825000067705EB420677803F0C03FB0C73C4E9FD
:1082600013731C14B380F480B1EBE07F23D035F896
:10827000123000E04AE1B088DF43C043718883B226
:10828000E043C9437F1C3C0489B280B2240C14D162
:10829000491C0904090C10D15B1C1B041B0C0CD1DC
:1082A000401C09E0800000202C2D002040630020AD
:1082B0008BE092E077E07FE080B225F81240718099
:1082C000B380F0806AE20B4641F66C018B4273D8B2
:1082D000816D002901DB616302E04A1ED2436263C3
:1082E000D9F85C00002801DBA06302E0421ED24303
:1082F000A263D4E90D76B7FBF6F206FB1276C4E969
:108300000F2625F81320141405EB4302C9175480D7
:1083100096803614D680B1EBE07F4DD035F813004F
:108320009188C743E043C9438CB2F1437F1C3E04AC
:1083300080B289B2360C01D1401C80B2641CA4B258
:10834000002C7FF4F5AA491C89B2FFF7F1BA4779EE
:10835000802F31D3812F7DD891098678C1F1000C0F
:1083600002EB8C12C9F8442006EB02225208C9F82D
:108370004C104846C9F84020802F05D005EB8101FC
:1083800043F258068E5F05E081B105EB810143F2AF
:1083900048068E5F41F270711144314481643D2B77
:1083A0000FD03F2B21D041F66E00A9E441F2707648
:1083B00032440AEB0201F1E762E00EEB2240FFF7E4
:1083C000F7B90A4641F66C019EE44B1EDB431E0CD6
:1083D0009BB2C4E90D36FFF7F9BA431EDB431E0C0E
:1083E0009BB2C4E90F36FFF7FEBA0B4641F66C01AB
:1083F0008B4245D8816D002901DB616302E04A1E92
:10840000D2436263D9F85C00002801DBA06302E07C
:10841000421ED243A263D4E90D76B7FBF6F206FB07
:108420001276C4E90F2625F81320141405EB430235
:10843000C917548096803614D680B1EBE07F1FD0E8
:1084400035F813009188C743E043C94380B21FFA4F
:1084500081FC00E0C5E0F1437F1C3C0489B2240CA0
:1084600001D1401C80B20CF1010C1FFA8CF6002ED9
:1084700001D1491C89B225F8134050809680D180E3
:108480008CE13D2B3FD03F2B3DD0022A1ED280787D
:1084900000EB02204008C9E91202C62833D8E16A7D
:1084A0004FEAE17201EB12424FEA12434FEA0343F3
:1084B0000029A1EB0303FA4941F8203001DB121433
:1084C00001E00EEB224201EB800068E08078E36A75
:1084D000F44A20F0030410F0030F135113D180105D
:1084E000233815280FD2DFE800F00DD80E0E0E0E3F
:1084F0000D0E0E0D0E0B0B0E0B0E0D0DDA0DDA0020
:10850000B184CAE0B18449E1018047E14779842F11
:108510007ED3852F7DD890F802A09009C0F1000885
:1085200002EB8812C9F844200AEB02225208C9F86B
:108530004C00C846C9F84020842F22D005EB8000AB
:1085400000F54050B0F95A001044C9F848003D2BDE
:1085500026D03F2B24D0BCF1020F22D2D8F84810ED
:10856000C6291DD8E06A4FEAE07200EB12424FEADA
:1085700012434FEA03430028A0EB0303C84874DA10
:10858000ADE048B105EB800000F54050B0F94A007D
:108590001044C8F84800DAE70BEB0200F9E7426044
:1085A000FCE0D8F84800E46A00EB9A00821ABD4863
:1085B00053461AF0030F40F822404AD1981023384E
:1085C000152846D2DFE800F00C69EAEAEAEA0CEA8C
:1085D000EA0CEA0B0BEA0BEA0C0C6B0C6B008FE756
:1085E00090E74779842F79D3852F32D890F802B05D
:1085F0009009C0F1000802EB8812C9F844200BEB87
:108600000222C9F84C005208C846C9F8402001E0CF
:108610006CE06EE0842F1DD005EB800000F540502B
:10862000B0F958001044C9F848003D2B11D03F2B39
:108630000FD0BCF1020F91D3D8F84800E46A00EBE8
:108640009B00821A97485B461BF0030F40F82240BC
:1086500010D0A3E058B105EB800000F54050B0F910
:1086600048001044C8F84800DFE733E019E00AEB9F
:108670000200F7E798102338152864D2DFE800F0ED
:108680000C0D8E8E8E8E0C8E8E0C8E0B0B8E0B8E9A
:108690000C0C0F0C0F0033E734E7834834E78348B2
:1086A00032E7817801EB02214908C9E9101248E05C
:1086B0003F2B73D0FE2971D8E06A4FEAE07200EBDD
:1086C00012424FEA12434FEA03430028A0EB030390
:1086D000774804DB40F82130121404E034E040F81D
:1086E00021300EEB224200EB810058E741798229CC
:1086F00054D34679832E51D891098778C1F1000C63
:1087000002EB8C12C9F8442007EB02225208C9F888
:108710004C104846C9F84020822E06D005EB810156
:1087200001F54051B1F95A1006E039B105EB81016C
:1087300001F54051B1F94A1011442DE00BEB020153
:108740002AE03D2BB4D129E04679822E26D3832E10
:1087500024D891098778C1F1000C02EB8C12C9F87A
:10876000442007EB02225208C9F84C104846C9F8C9
:108770004020822E06D005EB810101F54051B1F970
:108780005810D9E731B105EB810101F54051B1F93C
:108790004810D1E70AEB02018164D2E70DB0002056
:1087A000BDE8F08F00207047424930B50A184249B1
:1087B00012F8025C002391F8320001F16A04F92DED
:1087C00003D112F8012CFF2A03D06278012A02D0CB
:1087D00003E02278FAE7012801D081F83230002046
:1087E00030BD354934486A314A7890F832301A43FE
:1087F00000D0012280F832204A70002070472E49B4
:108800002E4B3731C87F11F8052C1A54401CC877FD
:10881000002070472849294A563108780244401EF2
:1088200012F8012C01F8242C087001F11400427098
:10883000002070472049214891F85620104410F834
:10884000010C81F832006A314870002070471A48E4
:1088500090F8321009B1002100E0012180F83210B7
:10886000002070471349164A095C52F82110084746
:10887000114A10B592F855100023012922D002F1B7
:108880006A014C780C7092F832404C700949085CCF
:10889000F7F73DFED8B1012082F8320019E0000060
:1088A0003C2500204C2C0020242C01402434014085
:1088B0003C21002000C003080000002024630020A9
:1088C000E06E002082F8553082F85630DEE782F8FC
:1088D0003230002010BDFE4A10B592F8551000232A
:1088E000012911D002F16A014C780C7092F83240E3
:1088F0004C70F849085C00F58070F7F708FE40B14D
:10890000012082F8320006E082F8553082F85630B5
:10891000EFE782F83230002010BDED4A10B592F832
:1089200055100023012911D002F16A014C780C7016
:1089300092F832404C70E749085C00F50070F7F798
:10894000E6FD40B1012082F8320006E082F85530A1
:1089500082F85630EFE782F83230002010BDDC4A52
:1089600010B592F855100023012911D002F16A01C7
:108970004C780C7092F832404C70D649085C00F587
:108980004070F7F7C4FD40B1012082F8320006E0E4
:1089900082F8553082F85630EFE782F83230002006
:1089A00010BDCB4A10B592F855100023012911D003
:1089B00002F16A014C780C7092F832404C70C54953
:1089C000085C00F58060F7F7A2FD40B1012082F855
:1089D000320006E082F8553082F85630EFE782F830
:1089E0003230002010BDBA4A10B592F8551000235D
:1089F000012911D002F16A014C780C7092F83240D2
:108A00004C70B449085C00F5A060F7F780FD40B1F8
:108A1000012082F8320006E082F8553082F85630A4
:108A2000EFE782F83230002010BDA94A10B592F865
:108A300055100023012911D002F16A014C780C7005
:108A400092F832404C70A349085C00F5FA50F7F7F1
:108A50005EFD40B1012082F8320006E082F8553018
:108A600082F85630EFE782F83230002010BD994985
:108A700000B5085CF7F74BFD9549002230B191F83D
:108A8000320028B1012081F8320001E081F8322063
:108A9000002000BD8F4900B5085C00F58070F7F735
:108AA00036FD8B49002230B191F8320028B1012007
:108AB00081F8320001E081F83220002000BD8549B4
:108AC00000B5085C00F50070F7F721FD8049002231
:108AD00030B191F8320028B1012081F8320001E074
:108AE00081F83220002000BD7A4900B5085C00F50D
:108AF0004070F7F70CFD7649002230B191F8320052
:108B000028B1012081F8320001E081F832200020F4
:108B100000BD704900B5085C00F58060F7F7F7FC10
:108B20006B49002230B191F8320028B1012081F860
:108B3000320001E081F83220002000BD654900B517
:108B4000085C00F5A060F7F7E2FC6149002230B153
:108B500091F8320028B1012081F8320001E081F85B
:108B60003220002000BD5B4900B5085C00F5FA50DA
:108B7000F7F7CDFC5649002230B191F8320028B108
:108B8000012081F8320001E081F83220002000BD90
:108B9000504900B5085CF7F7BAFC4D4940B991F867
:108BA0003200012804D0002081F83200002000BDEE
:108BB0000120F9E7474900B5085C00F58070F7F738
:108BC000A6FC434940B991F83200012804D00020A6
:108BD00081F83200002000BD0120F9E73D4900B5D1
:108BE000085C00F50070F7F792FC394940B991F83C
:108BF0003200012804D0002081F83200002000BD9E
:108C00000120F9E7334900B5085C00F54070F7F73B
:108C10007EFC2F4940B991F83200012804D0002091
:108C200081F83200002000BD0120F9E7294900B594
:108C3000085C00F58060F7F76AFC254940B991F8B7
:108C40003200012804D0002081F83200002000BD4D
:108C50000120F9E71F4900B5085C00F5A060F7F7AF
:108C600056FC1B4940B991F83200012804D000207D
:108C700081F83200002000BD0120F9E7154900B558
:108C8000085C00F5FA50F7F742FC114940B991F839
:108C90003200012804D0002081F83200002000BDFD
:108CA0000120F9E70A4A10B592F85510002301296E
:108CB00014D002F16A014C780C7092F832404C707A
:108CC0000449085CF7F723FC68B182F8323003E00E
:108CD0000000002000C00308002010BD82F85530BD
:108CE00082F85630ECE7012082F83200EFE7F74ACD
:108CF00010B592F855100023012911D002F16A0134
:108D00004C780C7092F832404C70F149085C00F5D8
:108D10008070F7F7FCFB40B182F83230002010BDC4
:108D200082F8553082F85630EFE7012082F83200A1
:108D3000F4E7E64A10B592F855100023012911D046
:108D400002F16A014C780C7092F832404C70E049A4
:108D5000085C00F50070F7F7DAFB40B182F83230BA
:108D6000002010BD82F8553082F85630EFE7012020
:108D700082F83200F4E7D54A10B592F85510002376
:108D8000012911D002F16A014C780C7092F832403E
:108D90004C70CF49085C00F54070F7F7B8FB40B164
:108DA00082F83230002010BD82F8553082F85630FB
:108DB000EFE7012082F83200F4E7C44A10B592F8D8
:108DC00055100023012911D002F16A014C780C7072
:108DD00092F832404C70BE49085C00F58060F7F7AD
:108DE00096FB40B182F83230002010BD82F8553039
:108DF00082F85630EFE7012082F83200F4E7B34AF8
:108E000010B592F855100023012911D002F16A0122
:108E10004C780C7092F832404C70AD49085C00F50B
:108E2000A060F7F774FB40B182F83230002010BD2B
:108E300082F8553082F85630EFE7012082F8320090
:108E4000F4E7A24A10B592F855100023012911D079
:108E500002F16A014C780C7092F832404C709C49D7
:108E6000085C00F5FA50F7F752FB40B182F8323057
:108E7000002010BD82F8553082F85630EFE701200F
:108E800082F83200F4E7924900B5085CF7F73FFB3F
:108E90008E49002218B181F83220002000BD91F8DF
:108EA00032000028F9D0012081F83200F5E7884926
:108EB00000B5085C00F58070F7F729FB83490022B4
:108EC00018B181F83220002000BD91F8320000284E
:108ED000F9D0012081F83200F5E77D4900B5085C42
:108EE00000F50070F7F713FB7849002218B181F8FC
:108EF0003220002000BD91F832000028F9D0012076
:108F000081F83200F5E7724900B5085C00F5407061
:108F1000F7F7FDFA6D49002218B181F832200020E0
:108F200000BD91F832000028F9D0012081F832000C
:108F3000F5E7674900B5085C00F58060F7F7E7FAE8
:108F40006249002218B181F83220002000BD91F85A
:108F500032000028F9D0012081F83200F5E75C49A1
:108F600000B5085C00F5A060F7F7D1FA5749002278
:108F700018B181F83220002000BD91F8320000289D
:108F8000F9D0012081F83200F5E7514900B5085CBD
:108F900000F5FA50F7F7BBFA4C49002218B181F8F6
:108FA0003220002000BD91F832000028F9D00120C5
:108FB00081F83200F5E7464900B5085CF7F7A7FAF3
:108FC000424948B191F83200012805D05FF0000015
:108FD00081F83200002000BD0120F9E73C4900B5CE
:108FE000085C00F58070F7F792FA384940B191F8C3
:108FF0003200012804D0002081F83200002000BD9A
:109000000120F9E7324900B5085C00F50070F7F778
:109010007EFA2E4940B191F83200012804D0002098
:1090200081F83200002000BD0120F9E7284900B591
:10903000085C00F54070F7F76AFA244940B191F8EE
:109040003200012804D0002081F83200002000BD49
:109050000120F9E71E4900B5085C00F58060F7F7CC
:1090600056FA1A4940B191F83200012804D0002084
:1090700081F83200002000BD0120F9E7144900B555
:10908000085C00F5A060F7F742FA104940B191F88A
:109090003200012804D0002081F83200002000BDF9
:1090A0000120F9E70A4900B5085C00F5FA50F7F726
:1090B0002EFA064940B191F83200012804D0002070
:1090C00081F83200002000BD0120F9E700000020F7
:1090D00000C00308F84910B591F855300022012B63
:1090E0000FD001F16A035C781C7091F832405C701B
:1090F000F24B185CF24B185C40B1012081F8320051
:1091000006E081F8552081F85620F1E781F83220F9
:10911000002010BDE949085CE9490A5CE6480021E5
:109120001AB190F8321011B1012180F832100020EC
:109130007047E249085CE249095CDF4841B990F8B0
:109140003210012904D0002180F83210002070472D
:109150000121F9E7D84910B591F855300022012BCB
:109160000FD001F16A035C781C7091F832405C709A
:10917000D24B185CD24B185C40B181F832200020F1
:1091800010BD81F8552081F85620F1E7012081F8C3
:109190003200F4E7C949085CC9490A5CC6480021A5
:1091A0001AB990F8321011B1012180F83210002064
:1091B0007047C249085CC249095CBF4841B190F898
:1091C0003210012904D0002180F8321000207047AD
:1091D0000121F9E7B84910B591F855300022012B6B
:1091E00010D001F16A035C781C7091F832405C7019
:1091F000B24B185CB34B185CC00708D0012081F853
:10920000320006E081F8552081F85620F0E781F819
:109210003220002010BDA949085CAA49085C4FF023
:109220000001C207A44803D090F8321011B1012107
:1092300080F8321000207047A049085CA149085C02
:10924000C1079D4808D190F83210012904D00021AF
:1092500080F83210002070470121F9E7964910B5D7
:1092600091F855300022012B10D001F16A035C788F
:109270001C7091F832405C70904B185C914B185CFC
:10928000C00708D081F83220002010BD81F8552099
:1092900081F85620F0E7012081F83200F4E7874991
:1092A000085C8849085C4FF00001C207824803D17E
:1092B00090F8321011B1012180F83210002070476F
:1092C0007E49085C7F49085CC1077B4808D090F85C
:1092D0003210012904D0002180F83210002070479C
:1092E0000121F9E7744910B591F855300022012B9E
:1092F00010D001F16A035C781C7091F832405C7008
:109300006E4B1B5C7048185CC00708D0012081F8C8
:10931000320006E081F8552081F85620F0E781F808
:109320003220002010BD6549095C6748085C4FF099
:109330000001C207604803D090F8321011B101213A
:1093400080F83210002070475C49095C5E48085C78
:10935000C107594808D190F83210012904D00021E2
:1093600080F83210002070470121F9E7524910B50A
:1093700091F855300022012B10D001F16A035C787E
:109380001C7091F832405C704C4B1B5C4E48185C72
:10939000C00708D081F83220002010BD81F8552088
:1093A00081F85620F0E7012081F83200F4E74349C4
:1093B000095C4548085C4FF00001C2073E4803D1F4
:1093C00090F8321011B1012180F83210002070475E
:1093D0003A49095C3C48085CC107374808D090F816
:1093E0003210012904D0002180F83210002070478B
:1093F0000121F9E7304910B591F855300022012BD1
:1094000010D001F16A035C781C7091F832405C70F6
:109410002A4B1B5C2D48185CC00708D0012081F83E
:10942000320006E081F8552081F85620F0E781F8F7
:109430003220002010BD2149095C2448085C4FF00F
:109440000001C2071C4803D090F8321011B101216D
:1094500080F83210002070471849095C1B48085CEE
:10946000C107154808D190F83210012904D0002115
:1094700080F83210002070470121F9E70E4910B53D
:1094800091F855300022012B10D001F16A035C786D
:109490001C7091F832405C70084B1B5C0B48185CE8
:1094A000C00715D081F83220002010BD81F855206A
:1094B00081F85620F0E700000000002000C00308FB
:1094C00052190020521D0020521E0020521F002061
:1094D000012081F83200E7E7FB49095CFB48085CA2
:1094E0004FF00001C207FA4803D190F8321011B1D1
:1094F000012180F8321000207047F349095CF348DD
:10950000085CC107F24809D090F83210012905D053
:109510005FF0000180F83210002070470121F9E768
:10952000EB4910B591F855300022012B10D001F114
:109530006A035C781C7091F832405C70E24B1B5CF3
:10954000E448185CC00708D0012081F8320006E02A
:1095500081F8552081F85620F0E781F8322000206C
:1095600010BDD949095CDB48085C4FF00001C20717
:10957000D74803D090F8321011B1012180F8321091
:1095800000207047D049095CD248085CC107D04828
:1095900008D190F83210012904D0002180F832104F
:1095A000002070470121F9E7C94910B591F85530FD
:1095B0000022012B10D001F16A035C781C7091F835
:1095C00032405C70C04B1B5CC248185CC00708D0BE
:1095D00081F83220002010BD81F8552081F85620F6
:1095E000F0E7012081F83200F4E7B749095CB94897
:1095F000085C4FF00001C207B54803D190F8321063
:1096000011B1012180F8321000207047AE49095C89
:10961000B048085CC107AE4808D090F83210012964
:1096200004D0002180F83210002070470121F9E7B2
:10963000A74910B591F855300022012B0FD001F148
:109640006A035C781C7091F832405C709E4B185C29
:10965000A14B185C40B1012081F8320006E081F88E
:10966000552081F85620F1E781F83220002010BD06
:109670009549085C98490A5C954800211AB190F810
:10968000321011B1012180F83210002070478E494C
:10969000085C9149095C8E4841B990F83210012963
:1096A00004D0002180F83210002070470121F9E732
:1096B000874910B591F855300022012B0FD001F1E8
:1096C0006A035C781C7091F832405C707E4B185CC9
:1096D000814B185C40B181F83220002010BD81F828
:1096E000552081F85620F1E7012081F83200F4E797
:1096F0007549085C78490A5C754800211AB990F8E8
:10970000321011B1012180F83210002070476E49EB
:10971000085C7149095C6E4841B190F8321001292A
:1097200004D0002180F83210002070470121F9E7B1
:10973000674910B591F855300022012B10D001F186
:109740006A035C781C7091F832405C705E4B185C68
:10975000624B33F8100040B181F83220002010BD78
:1097600081F8552081F85620F0E7012081F8320079
:10977000F4E75549085C594931F810205448002154
:109780001AB990F8321011B1012180F8321000207E
:1097900070474F4910B591F855300022012B10D079
:1097A00001F16A035C781C7091F832405C70464BA2
:1097B000185C4A4B33F8100040B1012081F83200A8
:1097C00006E081F8552081F85620F0E781F8322034
:1097D000002010BD3C49085C404931F810203C484D
:1097E00000211AB190F8321011B1012180F8321025
:1097F000002070473449085C384931F8101034486B
:1098000041B190F83210012904D0002180F83210C3
:10981000002070470121F9E72B49085C2F4931F8F6
:1098200010102B48012909D090F83210012905D0D9
:109830005FF0000180F83210002070470121F9E745
:10984000234910B591F855300022012B11D001F1B8
:109850006A035C781C7091F832405C701A4B185C9B
:109860001E4B513B185C012808D081F832200020A3
:1098700010BD81F8552081F85620EFE7012081F8CE
:109880003200F4E71049085C144951390A5C0021A0
:109890000F48012A03D190F8321011B1012180F84C
:1098A0003210002070470849085C0C495139095CA6
:1098B0000748012914D090F83210012910D0002156
:1098C00080F832100020704700C00308521F0020AB
:1098D0000000002052200020521B00201211002006
:1098E0000121EDE7F84910B591F855300022012B20
:1098F0000FD001F16A035C781C7091F832405C7003
:10990000F24B185CF24B185C40B181F83220002019
:1099100010BD81F8552081F85620F1E7012081F82B
:109920003200F4E7E949085CE9490A5CE6480021AD
:109930001AB990F8321011B1012180F832100020CC
:10994000C1E7E249085CE249095CDF4841B190F8AF
:109950003210012904D0002180F832100020B2E733
:109960000121F9E7D84991F832205AB1D94AB1F822
:109970007E10515CC90705D0D449A2F6E142085CCB
:109980000121115400209EE7CF4991F832205AB1AD
:10999000D04AB1F87E10515CC90705D0CB49A2F678
:1099A000E142085C0021115400208CE7C64910B543
:1099B00091F8322052B1C74AB1F87E10515CC90704
:1099C00004D0C249085C0121F6F7AEFD002010BDAD
:1099D000BD4910B591F8322052B1BE4AB1F87E109F
:1099E000515CC90704D0B949085C0021F6F79CFD19
:1099F000002010BDB44910B591F8322062B1B54ACB
:109A0000B1F87E10515CC90706D0B049085C01214D
:109A100000F58070F6F788FD002010BDAA4910B54A
:109A200091F8322062B1AB4AB1F87E10515CC9079F
:109A300006D0A649085C002100F58070F6F774FD99
:109A4000002010BDA04910B591F8322062B1A14AA2
:109A5000B1F87E10515CC90706D09C49085C012111
:109A600000F50070F6F760FD002010BD964910B5B6
:109A700091F8322062B1974AB1F87E10515CC90763
:109A800006D09249085C002100F50070F6F74CFD05
:109A9000002010BD8C4910B591F8322062B18D4A7A
:109AA000B1F87E10515CC90706D08849085C0121D5
:109AB00000F54070F6F738FD002010BD824910B562
:109AC00091F8322062B1834AB1F87E10515CC90727
:109AD00006D07E49085C002100F54070F6F724FDB1
:109AE000002010BD784910B591F8322062B1794A52
:109AF000B1F87E10515CC90706D07449085C012199
:109B000000F58060F6F710FD002010BD6E4910B51D
:109B100091F8322062B16F4AB1F87E10515CC907EA
:109B200006D06A49085C002100F58060F6F7FCFC6D
:109B3000002010BD644910B591F8322062B1654A29
:109B4000B1F87E10515CC90706D06049085C01215C
:109B500000F5A060F6F7E8FC002010BD5A4910B5EA
:109B600091F8322062B15B4AB1F87E10515CC907AE
:109B700006D05649085C002100F5A060F6F7D4FC39
:109B8000002010BD504910B591F832206AB1514AF9
:109B9000B1F87E10515CC90707D04C490844012137
:109BA000807800F5FA50F6F7BFFC002010BD46495A
:109BB00010B591F832206AB1464AB1F87E10515C76
:109BC000C90707D0414908440021807800F5FA50C0
:109BD000F6F7AAFC002010BD2DE9F04F3E493F4F9B
:109BE0004A6E394907F17C0491F8325091F83330CC
:109BF00072B1364A354EDFF8D890125C4FF0000B48
:109C000002F00F020644A9F15009082A07D018E013
:109C100047F82300E5545B1C81F8333032E08D7641
:109C20005A4681F81BB045B1DFF8A8C0B1F87E8074
:109C30001CF808C05FEACC7C03D196F802C009F892
:109C40000C20002291F81AA091F81BE018E000BF48
:109C500057F82210814211D1BAF1000F0DD014F83B
:109C600002C0A554B178F44504D14FF0010809F8B9
:109C7000018003E009F801B000E0A554521C92B243
:109C80009A42E5D30220BDE8F08F2DE9F84F124942
:109C90000D4BDFF848904C6E93F8322093F8331058
:109CA00009F17C0AE4B1094CDFF824B00026245CF9
:109CB0004FF0010E04F00F05044CABF1500B0444BF
:109CC000092D15D02DE000000000002000C0030881
:109CD000C1100020521D0020000100200C5F002058
:109CE00049F821000AF80120491C83F8331037E0B5
:109CF000F84D83F81BE0DFF8D8C3B5F87E507746FF
:109D000032B11CF805805FEAC87801D09E7605E084
:109D10009F7632B11CF80550ED0702D0A5780BF8FC
:109D200005609F7EDB7E0025009317E059F8253003
:109D3000834211D177B11AF80580DDF800C00AF826
:109D40000520A378E04502D10BF803E004E00BF80E
:109D5000036001E00AF805206D1CADB28D42E5D329
:109D60000220BDE8F88F2DE9F0470646DA48D94CC5
:109D7000DFF86883406E94F8321008F17C0940B136
:109D8000D748D74A805D971900F00F00082809D0FE
:109D900016E014F8330F48F8206009F80010401C52
:109DA00020702FE0A1760020E07629B1C848B4F8F1
:109DB0007E10405CC00703D1B8780021F6F7B4FBF1
:109DC00000251BE058F82500B04215D1A07E78B1DF
:109DD00019F80510E27E914294F8321009F8051046
:109DE000B87801D1012100E00021F6F79DFB03E0E6
:109DF00094F8321009F805106D1CADB294F83300D8
:109E00008542DFD30220BDE8F0872DE9F047064602
:109E1000B148B04CDFF8C482406E94F8321008F1BB
:109E20007C0940B1AE48805D00F00F02AC48871954
:109E3000092A09D01EE014F8330F48F8206009F809
:109E40000010401C207037E0A2480122E276A04BAF
:109E5000B0F87E0029B11D5CED0702D00020A0768D
:109E600004E0A27631B1185CC00703D0B8780021B5
:109E7000F6F75AFB00251BE058F82500B04215D133
:109E8000A07E78B119F80510E27E914294F8321064
:109E900009F80510B87801D1012100E00021F6F79A
:109EA00043FB03E094F8321009F805106D1CADB2C5
:109EB00094F833008542DFD30220A4E72DE9F04770
:109EC00006468548834CDFF81482416E94F83200D0
:109ED00008F17C0941B18249814A895D971901F0F5
:109EE0000F01082909D018E014F8331F48F8216041
:109EF00009F80100491C217034E0A0760021E176C8
:109F000028B17348B4F87E10405CC00705D1B8781A
:109F1000002100F58070F6F707FB00251EE000BF6A
:109F200058F82500B04217D1A07E88B119F8051065
:109F3000E27E914294F8321009F80510B87800F5E5
:109F4000807001D1012100E00021F6F7EDFA03E075
:109F500094F8321009F805106D1CADB294F8330076
:109F60008542DDD302204EE72DE9F04705465A48E9
:109F7000584EDFF86881406E96F8321008F17C097F
:109F800040B15748564A405D571900F00F00092864
:109F900009D020E016F8330F48F8205009F80010D7
:109FA000401C30703CE04B480123F376484AB0F83F
:109FB0007E0029B1145CE40702D00020B07604E0F2
:109FC000B37641B1105CC00705D0B878002100F528
:109FD0008070F6F7A9FA00241EE000BF58F82400AC
:109FE000A84217D1B07E88B119F80410F27E9142D0
:109FF00096F8321009F80410B87800F5807001D195
:10A00000012100E00021F6F78FFA03E096F8321004
:10A0100009F80410641CA4B296F833008442DDD31E
:10A020000220F0E62DE9F04706462B48294CDFF8E0
:10A03000AC80416E94F8320008F17C0941B12849A6
:10A04000274A895D971901F00F01082909D018E006
:10A0500014F8331F48F8216009F80100491C2170E9
:10A0600034E0A0760021E17628B11948B4F87E10DA
:10A07000405CC00705D1B878002100F50070F6F704
:10A0800053FA00251EE000BF58F82500B04217D152
:10A09000A07E88B119F80510E27E914294F8321042
:10A0A00009F80510B87800F5007001D1012100E031
:10A0B0000021F6F739FA03E094F8321009F8051098
:10A0C0006D1CADB294F833008542DDD302209AE6D0
:10A0D000521D002000000020000100200C5F002025
:10A0E00000C003082DE9F0470546FA48FB4EDFF8AB
:10A0F000E883406E96F8321008F17C0940B1F848C8
:10A10000F74A405D571900F00F00092809D020E0F8
:10A1100016F8330F48F8205009F80010401C307032
:10A120003CE0EE480123F376EE4AB0F87E0029B118
:10A13000145CE40702D00020B07604E0B37641B1AD
:10A14000105CC00705D0B878002100F50070F6F764
:10A15000EBF900241EE000BF58F82400A84217D1F4
:10A16000B07E88B119F80410F27E914296F8321050
:10A1700009F80410B87800F5007001D1012100E061
:10A180000021F6F7D1F903E096F8321009F804102F
:10A19000641CA4B296F833008442DDD3022032E678
:10A1A0002DE9F0470646CB48CC4CDFF82C83416EB6
:10A1B00094F8320008F17C0941B1C949C84A895D67
:10A1C000971901F00F01082909D018E014F8331F7E
:10A1D00048F8216009F80100491C217034E0A0769C
:10A1E0000021E17628B1BF48B4F87E10405CC0077A
:10A1F00005D1B878002100F54070F6F795F90025F3
:10A200001EE000BF58F82500B04217D1A07E88B1EB
:10A2100019F80510E27E914294F8321009F8051001
:10A22000B87800F5407001D1012100E00021F6F777
:10A230007BF903E094F8321009F805106D1CADB2FB
:10A2400094F833008542DDD30220DCE52DE9F047A8
:10A250000546A048A14EDFF88082406E96F8321085
:10A2600008F17C0940B19E489D4A405D571900F0B5
:10A270000F00092809D020E016F8330F48F82050C5
:10A2800009F80010401C30703CE094480123F3763C
:10A29000944AB0F87E0029B1145CE40702D0002093
:10A2A000B07604E0B37641B1105CC00705D0B87851
:10A2B000002100F54070F6F737F900241EE000BFDA
:10A2C00058F82400A84217D1B07E88B119F80410BC
:10A2D000F27E914296F8321009F80410B87800F531
:10A2E000407001D1012100E00021F6F71DF903E0E3
:10A2F00096F8321009F80410641CA4B296F83300E2
:10A300008442DDD302207EE52DE9F0470646714800
:10A31000724CDFF8C481416E94F8320008F17C0978
:10A3200041B16F496E4A895D971901F00F01082903
:10A3300009D018E014F8331F48F8216009F801002B
:10A34000491C217034E0A0760021E17628B16548EF
:10A35000B4F87E10405CC00705D1B878002100F544
:10A360008060F6F7E1F800251EE000BF58F82500F0
:10A37000B04217D1A07E88B119F80510E27E914253
:10A3800094F8321009F80510B87800F5806001D112
:10A39000012100E00021F6F7C7F803E094F832103D
:10A3A00009F805106D1CADB294F833008542DDD379
:10A3B000022028E52DE9F04705464648474EDFF8DC
:10A3C0001881406E96F8321008F17C0940B144487B
:10A3D000434A405D571900F00F00092809D020E0DA
:10A3E00016F8330F48F8205009F80010401C307060
:10A3F0003CE03A480123F3763A4AB0F87E0029B1AE
:10A40000145CE40702D00020B07604E0B37641B1DA
:10A41000105CC00705D0B878002100F58060F6F721
:10A4200083F800241EE000BF58F82400A84217D18A
:10A43000B07E88B119F80410F27E914296F832107D
:10A4400009F80410B87800F5806001D1012100E01E
:10A450000021F6F769F803E096F8321009F80410C5
:10A46000641CA4B296F833008442DDD30220CAE40F
:10A470002DE9F04706461748184CDFF85C80416E1E
:10A4800094F8320008F17C0941B11549144A895DFC
:10A49000971901F00F01082909D018E014F8331FAB
:10A4A00048F8216009F80100491C21703EE0A076BF
:10A4B0000021E17628B10B48B4F87E10405CC0075B
:10A4C00005D1B878002100F5A060F6F72DF8002539
:10A4D00028E00000000100200C5F002000000020A8
:10A4E00000C00308521D002058F82500B04217D1C3
:10A4F000A07E88B119F80510E27E914294F83210DE
:10A5000009F80510B87800F5A06001D1012100E03C
:10A510000021F6F709F803E094F8321009F8051065
:10A520006D1CADB294F833008542DDD302206AE49D
:10A530002DE9F0470546FB48FC4EDFF8EC83406E02
:10A5400096F8321008F17C0940B1F948F84A405DAC
:10A55000571900F00F00092809D020E016F8330F32
:10A5600048F8205009F80010401C30703CE0EF48DB
:10A570000123F376EF4AB0F87E0029B1145CE407BA
:10A5800002D00020B07604E0B37641B1105CC00781
:10A5900005D0B878002100F5A060F5F7C5FF0024CC
:10A5A0001EE000BF58F82400A84217D1B07E88B141
:10A5B00019F80410F27E914296F8321009F804104E
:10A5C000B87800F5A06001D1012100E00021F5F785
:10A5D000ABFF03E096F8321009F80410641CA4B233
:10A5E00096F833008442DDD302200CE4D049D24AED
:10A5F0000144C97852F821100847CD49CF4A014497
:10A60000C97852F821100847C94B10B5C74903440F
:10A610003231987801F5E1740A782254401C887030
:10A62000C749187902B101220A54042010BDC04A5A
:10A6300010B5BE4902443231907801F5E1740B78CF
:10A640002354401C887010790BB1012100E00021D7
:10A65000F5F76AFF042010BDB54B10B5B34A0344AB
:10A660003232987802F5E17411782154401C9070D0
:10A67000187900F5807001B10121F5F755FF04202C
:10A6800010BDAB4B10B5A94A03443232987802F59D
:10A69000E17411782154401C9070187900F5007015
:10A6A00001B10121F5F740FF042010BDA04B10B50A
:10A6B0009E4A03443232987802F5E17411782154AD
:10A6C000401C9070187900F5407001B10121F5F738
:10A6D0002BFF042010BD964B10B5944A0344323230
:10A6E000987802F5E17411782154401C9070187923
:10A6F00000F5806001B10121F5F716FF042010BDBF
:10A700008B4B10B5894A03443232987802F5E174D4
:10A7100011782154401C9070187900F5A06001B1A7
:10A720000121F5F701FF042010BD814908447F494C
:10A73000807881F83400022070477D49814A0144C5
:10A74000497952F8211008472DE9F05F784B002134
:10A750001D180A466C784FF00109102C05D101092B
:10A76000C0F3420209FA02F082B2704B764893F8C5
:10A770003260002E7ED06F4EB3F87E30F35CDB0784
:10A78000F8D0435C134201D024B142E1102C01D136
:10A7900013434354634CA87804F18006A067A8795A
:10A7A000E067A97A3160A97B7160297A0A09ECD146
:10A7B00001F00F010529E8D30D29E6D8083906294B
:10A7C0000AD2DFE801F009030612151800F58070BF
:10A7D00001E000F50070E067DFF864A100270AF1EE
:10A7E000500ABB46DFF8588123E000F54070F2E7DD
:10A7F00000F58060EFE700F5A060ECE7287A00F054
:10A800000F000528E06F384408D00844F5F77FFEB4
:10A810000146E06F3844F5F787FE08E042181AF861
:10A82000021011B108F8009001E008F800B07F1C98
:10A83000BFB2D6E90001401AB842DFD8287905280E
:10A8400041D1B08887B23CE0A06F3844504410F842
:10A85000010C012812D1287A316800F00F00052878
:10A86000E06F084471683844A0EB0100A0F10100DA
:10A870000CD000E0C8E00121F5F756FEA06FC11929
:10A8800001EB0A0010F8010C18B118E008F800906C
:10A8900015E0287A316800F00F000528E06F0844C1
:10A8A00007D071683844401A401E0021F5F73CFE7D
:10A8B00005E0C1197068081A401E08F800B07F1E34
:10A8C000BFB2002FC0D12879042845D1B08887B203
:10A8D00040E0A06F3844401EF5F7C7FD0028287AF5
:10A8E00000F00F000FD00528E16F30680844716850
:10A8F0003844A0EB0100A0F1010001D000210EE0DE
:10A9000008F800B024E00528E06F31680844716859
:10A910003844A0EB0100A0F1010017D00121F5F7A8
:10A9200003FE15E0000100200C5F00200000002065
:10A9300000C00308521D0020E06E0020E0720020DD
:10A9400071100020E06A00206028002008F80090C4
:10A950007F1EBFB2002FBCD12879010959D100F068
:10A960000F00082855D30D2853D8083806280CD2D4
:10A97000DFE800F00B03070E1216A06F00F58070E1
:10A9800002E0A06F00F50070A067B08887B238E0E1
:10A99000A06F00F54070F7E7A06F00F58060F3E767
:10A9A000A06F00F5A060EFE7A06F3844401EF5F7F8
:10A9B000AEFD0028287A00F00F000FD00528E06FC8
:10A9C0003168084471683844A0EB0100A0F101002F
:10A9D00001D001210EE008F8009010E00528E06F9A
:10A9E0003168084471683844A0EB0100A0F101000F
:10A9F00003D00021F5F798FD01E008F800B07F1EB4
:10AA0000BFB2002FD0D104E0102C02D1435C93439D
:10AA100043541020BDE8F09F2DE9F05FFF4B00226A
:10AA20001D1811466C784FF00109102C05D1020950
:10AA3000C0F3420109FA01F081B2F94BF94893F8E9
:10AA40003260002E7ED0B3F87E30A0F60E36F35C76
:10AA5000DB07F7D0835C0B4201D024B113E1102C4B
:10AA600001D10B438354F04CA87804F18006A06711
:10AA7000A879E067AF7A3760A97B7160297A0A0903
:10AA8000ECD101F00F010529E8D30D29E6D80839EA
:10AA900006290AD2DFE801F009030610131600F5B3
:10AAA000807001E000F50070E067DFF880A34FF0F0
:10AAB000000BAAF1500829E000F54070F4E700F51A
:10AAC0008060F1E700F5A060EEE7287A00F00F0063
:10AAD0000528E06F38440AD0401A401EF5F717FDEC
:10AAE0000146E06F3844401EF5F71EFD0CE0421AA7
:10AAF00002EB0A01A0F1010011F8011C11B108F8E4
:10AB0000009001E008F800B07F1EBFB271688F426C
:10AB1000DBD82879052837D1B08887B232E0A06F1A
:10AB2000C11901EB0A0010F8010C01280DD1287A97
:10AB300000F00F000528E06F3844A0F101000CD0B0
:10AB4000012100E09AE0F5F7EFFCA06FC11901EBDD
:10AB50000A0010F8010C18B112E008F800900FE09C
:10AB6000287A00F00F000528E06F05D03844401E19
:10AB70000021F5F7D9FC03E0C119491E08F801B01E
:10AB80007F1EBFB2002FCAD12879042828D1B088EF
:10AB900087B223E0A06F3844401EF5F766FC00281A
:10ABA000287A00F00F000AD00528E06F3844A0F1A1
:10ABB000010001D0002108E008F800B00CE00528F1
:10ABC000E06F05D03844401E0121F5F7ADFC03E0ED
:10ABD000C119491E08F801907F1EBFB2002FD9D1BC
:10ABE000287901094FD100F00F0008284BD30D2818
:10ABF00049D8083806280CD2DFE800F00B03070E0E
:10AC00001216A06F00F5807002E0A06F00F50070D2
:10AC1000A067B08886B22EE0A06F00F54070F7E71D
:10AC2000A06F00F58060F3E7A06F00F5A060EFE78C
:10AC3000A06F3044401EF5F76AFC0028287A00F027
:10AC40000F000AD00528E06F3044A0F1010001D0C8
:10AC5000012109E008F800900BE00528E06F30447E
:10AC6000A0F1010003D00021F5F75EFC01E008F837
:10AC700000B0761EB6B2002EDAD104E0102C02D15C
:10AC8000835C8B4383541020C4E610B5644A634B45
:10AC9000664992F83240185C503944B1B2F87E20CF
:10ACA00001F6E1439A5CD20701D0012200E00022C4
:10ACB0000A54002010BD10B55949584A91F8323055
:10ACC000105C3BB15A4AB1F87E10515CC90701D003
:10ACD000012100E00021F5F727FC002010BD4F4ABC
:10ACE00010B54F49105C91F8323000F580703BB1DF
:10ACF0004F4AB1F87E10515CC90701D0012100E034
:10AD00000021F5F711FC002010BD444A10B544495C
:10AD1000105C91F8323000F500703BB1444AB1F854
:10AD20007E10515CC90701D0012100E00021F5F738
:10AD3000FBFB002010BD394A10B53949105C91F871
:10AD4000323000F540703BB1394AB1F87E10515CA9
:10AD5000C90701D0012100E00021F5F7E5FB002043
:10AD600010BD2E4A10B52E49105C91F8323000F516
:10AD700080603BB12E4AB1F87E10515CC90701D00A
:10AD8000012100E00021F5F7CFFB002010BD234A90
:10AD900010B52349105C91F8323000F5A0603BB14A
:10ADA000234AB1F87E10515CC90701D0012100E0AF
:10ADB0000021F5F7B9FB002010BD184910B5084473
:10ADC000C1788F2914D1164991F8322052B1184A0E
:10ADD000B1F87E10515CC90704D08078012100F5DC
:10ADE000FA5003E08078002100F5FA50F5F79CFB5B
:10ADF000002010BDF0B509490B4C095CE165F9F77D
:10AE000072FA606E30B90B4A206E94F85C101154DF
:10AE1000401C2066024890F832600DE000C0030834
:10AE2000000000206028002000010020C110002048
:10AE3000521D00200C5E0020FD4D002105F58073A1
:10AE400003F2EA629EB1B0F87E00A2F2EA36305C0C
:10AE5000C0070CD0E06D01261E5452F82070E46A41
:10AE6000A74209DB2E54195442F8204004E0E06D5B
:10AE70001954295442F820100420F0BD2DE9F14F57
:10AE8000EC490098EC4C4FF0000A085CA4F5807186
:10AE9000E06591F83220002A7AD08946E74AB1F875
:10AEA0007E10515CC907F7D00126A4F1800502F697
:10AEB000FA67A2F50078C82825D2A2F580710A5C4D
:10AEC000EABB01F6EA0B0E545BF82010491C4BF864
:10AED00020100098F9F707FAE16AE963E06D5BF882
:10AEE00020208A4203D308F800604BF8201099F81C
:10AEF0003220002AD0D0D14AB9F87E10515CC9075F
:10AF0000CAD0C82838D3E06DEA2835D8CC490A5CC5
:10AF1000AAB90E5400F5FA50F5F7F9FA0028E06DD9
:10AF200007EB8000A0F54870016832D0491E01602F
:10AF30000098F9F75EFFE06AE863E06D00E01BE06F
:10AF400000F5FA50F5F7E3FA0028E06DEA6B07EB3D
:10AF50008001A1F5487109681DD0914202D800BF57
:10AF600008F8006099F83210002995D0B349B9F873
:10AF70007E00085CC0078FD0E06DEB287DD3B1491F
:10AF8000DFF8C4924FF0804BB1F8661031B13CE06D
:10AF9000F8E1491CCBE79142E2D2E3E7EB2803D08A
:10AFA000F12801D0F42830D1A649C838A1F866604C
:10AFB000A880584616F08EFA0121084616F079F955
:10AFC0004FF6FF70A9F80400A9F800A0A9F806A0A0
:10AFD000E06D4A46534600F5FA50F5F798FAC0B1CD
:10AFE000102050809849584616F0C9FA00231A4696
:10AFF0001946584616F01CFD4FF40041584616F00D
:10B00000A4FE0121584616F0A7FC8E48C07C10B162
:10B0100036E05380E6E7E06DEC2831D18948C6740C
:10B0200024202881894816F055FA0121C80216F01B
:10B0300037F94FF6FF70A9F80400A9F800A0A9F8A5
:10B0400006A0288942F208014A460844F5F75FFA4B
:10B05000D0B1102050807C497C4816F090FA002333
:10B060001A461946794816F0E3FC4FF40041774838
:10B0700016F06BFE0121754800E087E116F06CFCCC
:10B080007048C07B18B156E0A2F802A0E3E7E06D7B
:10B09000F62803D0F72801D0F9284CD16949C838DF
:10B0A000CE73A880584616F015FA0121084616F00E
:10B0B00000F94FF6FF70A9F80400A9F800A0A9F85C
:10B0C00006A0A9F802A06049584616F058FA0023D5
:10B0D0001A461946584616F0ABFC4FF40041584644
:10B0E00016F033FE0121584616F036FC574816F08C
:10B0F000F1F90121C80216F0D3F84FF6FF70A9F854
:10B100000400A9F800A0A9F806A01020A9F80200E0
:10B110004D494E4816F033FA00231A4619464B485B
:10B1200016F086FC4FF40041484816F00EFE01214F
:10B13000464816F011FC4348407BD8BBE06DFB2825
:10B1400003D0FC2801D0FE2834D13E49C8384E73C4
:10B15000A880584616F0BEF90121084616F0A9F855
:10B16000394816F0D5FBA9F800A04FF6FF72A9F8F0
:10B170000420A9F806A0A9F802A03349584616F001
:10B18000FEF900231A460321584616F064FC2E48A7
:10B190001A3016F0D0FB2C4906201A310881584687
:10B1A00016F018FB4FF400415846ABF8241001216B
:10B1B00016F0D2FB2348407CC8BBE06DFD2801D0CF
:10B1C000FF2849D11F49C8384E74E880204816F03E
:10B1D00081F90121480316F063F81B4816F098FB2B
:10B1E000A9F800A04FF6FF72A9F80420A9F806A05C
:10B1F000A9F802A01449164816F0C1F900231A460E
:10B200000321134816F027FC0F481A3016F093FB61
:10B210000D4906201A3108810D4816F0DBFA0C4959
:10B220004FF40040243108800121094812E013E066
:10B230005219002000C0030800010020521D002008
:10B24000521C002000000020C4030020002C0140FC
:10B250000034014016F080FBFE48017D49B9E16DE4
:10B26000ED2903D0F22901D0F52902D10675C8399C
:10B270006981417D29B9E16DEE2902D1467526210A
:10B28000A981817D39B9E16DEF2901D0F32902D17E
:10B290008675C839E981C17D29B9E16DF02902D1EE
:10B2A000C67528212982814690F8530040B9E06D87
:10B2B000F82801D0FA2803D189F85360C838688289
:10B2C0000098F9F796FDE16AE963E06DF02847D848
:10B2D000EB280ED0EC282AD000F5FA50F5F717F934
:10B2E0000028E06D07EB8001A1F5487109682FD0B7
:10B2F00032E042F22B00F5F70AF90028E06D07EB87
:10B300008001A1F548710A68BBF824101144EA6B6A
:10B31000A1F5004108D0914202D800BF08F80060B2
:10B32000E06DEC2803D024E09142F7D2F8E742F236
:10B330002C00F5F7ECF80028E06DC74907EB800218
:10B34000A2F54872098812681144A1F5004103D1A1
:10B35000EA6B91420BD20CE0EA6B914207D908E00C
:10B3600007EB8002A2F5487212688A4201D308F8FE
:10B37000006099F8321029B1B849B9F87E00085C2C
:10B38000C00703D1B649E26D01F802A0E06DC828FC
:10B3900002D20420BDE8F88F0820FBE72DE9F05F1A
:10B3A000AC4D8046AF4A284602EB080695F832308D
:10B3B00090F84B100024B078002B6FD0A74AB5F856
:10B3C0007E30D25CD207F8D0052868D8DFF8989292
:10B3D0004FF6FF7B01274FF0804A30BB00297AD11E
:10B3E000A5F8664085F84B70504616F073F80121B9
:10B3F000084615F05EFFA9F804B0A9F80040A9F8C6
:10B400000640A9F802404946504616F0B8F8002315
:10B410001A461946504616F00BFB0021504616F00E
:10B4200094FC0121504616F097FAB07801282BD1F0
:10B4300095F84C0088BB8848EC7485F84C7024382B
:10B4400016F048F80121C80215F02AFFA9F804B047
:10B45000A9F800408048A9F80640A9F802408249AE
:10B46000243816F08CF800237B481A4619462438F5
:10B4700016F0DEFA78480021243816F066FC76488B
:10B480000121243816F068FAB078022808D0032881
:10B490000DD0042812D0052817D01CE08FE04AE018
:10B4A00095F84D00B8B92C7585F84D7013E095F8F6
:10B4B0004E0080B96C7585F84E700CE095F84F0021
:10B4C00048B9AC7585F84F7005E095F8500010B993
:10B4D000EC7585F8507008F1040080B2F8F703FFAE
:10B4E000624FB178624DB88D25F8110008F108005F
:10B4F00080B2FC62FAF738FBB27805F11001B88D22
:10B5000021F812005B48062A15D2DFE802F0031585
:10B510002632404CBAF8243052460E8800EB4601E1
:10B520004B80B1F90430002B76DC4B8820F81630C4
:10B530002888888094846FE0474A13884E8800EBFF
:10B5400046014B80B1F90430002B65DC4B8820F8B4
:10B5500016306888888014805EE08A8800EB42019B
:10B56000B1F90430002B57DC4B8820F81230A88842
:10B570000AE0CA8800EB4201B1F90430002B4BDC31
:10B580004B8820F81230E88888804C8044E00A8993
:10B5900000EB4201B1F90430002B3DDC4B8820F870
:10B5A00012302889F0E74A8900EB4201B1F90430F2
:10B5B000002B31DC4B8820F812306889E4E750B169
:10B5C00001280CD0022810D0032814D0042818D049
:10B5D00005281CD020E0F9B185F84B401CE095F817
:10B5E0004C00C8B185F84C4016E095F84D0098B174
:10B5F00085F84D4010E095F84E0068B185F84E4052
:10B600000AE095F84F0038B185F84F4004E095F80E
:10B61000500008B185F850400C20BDE8F09FF0B50F
:10B620000C4D95F8321000293CD00C49B5F87E201D
:10B63000895CC90736D00B4908440C498478CC652D
:10B64000C07800F00F01002006291ED10A4A1055CB
:10B6500014E0000000000020242C0140521D0020B6
:10B66000521C002000C00308C40300200001002079
:10B67000C86200202C2D00205219002002F5807293
:10B68000105502F2EA6242F824000E297DD1FE4AEA
:10B69000C82C02F5807306D2105502F6EA1118552F
:10B6A00041F8240071E0F9491055EB2C185505D2EA
:10B6B00001EB8401A1F54871086066E04FF4004297
:10B6C000EB3CD603F24FDFF8CCC3152C5DD2DFE89C
:10B6D00004F00B171B1E21240E272A112D31343E96
:10B6E00038414649524D5700C1F88C003CE0C1F842
:10B6F000A40039E0C1F8B000B284A5F8680044E0C5
:10B70000C1F890003A8040E0C1F894003DE0C1F8F3
:10B7100098003AE0C1F89C0037E0C1F8A00034E09E
:10B72000C1F8A80031E0C1F8AC002EE0C1F8B400C7
:10B7300028762AE0C1F8B80001E0C1F8BC003A80E0
:10B7400012E0C1F8C4003A80B28428741DE0C1F848
:10B75000C0001AE0C1F8C80085F8540015E0C1F82F
:10B76000CC0001E0C1F8D000B2840EE0C1F8D800EE
:10B77000B284A87309E0C1F8D400ACF8002004E05A
:10B78000C1F8DC00ACF80020A8740220F0BD2DE95F
:10B79000F04FC149002201448BB04E781346102E61
:10B7A00005D10209C0F342030120984083B2BB4D8A
:10B7B000BB4895F83240002C7DD0B5F87E50A0F6FD
:10B7C0000E34655DED07F7D0855C1D4201D026B1D2
:10B7D000F3E1102E01D11D438554C878002284283E
:10B7E00002D0862868D0E8E148798028F0D1C8796D
:10B7F0008428EDD1487A8028EAD10879A94B042819
:10B8000014D20D7A042D11D28A7802EB0020D86070
:10B81000897901EB0521996004E0225C02F07E0247
:10B820002254401C80B28842F7D9C6E1052802D1D3
:10B830000C7A052C02D004090ED0BEE18878D860BD
:10B8400089799960984B04E04E2800D81A54401C1E
:10B8500080B28842F8D9B0E100F00F05082DB7D3C7
:10B860000D2DB5D8087A0409B2D100F00F04082CC8
:10B87000AED30D2CACD88B488038082D00D1C265D2
:10B880004FF48076092D00D1C6654FF400790A2D5A
:10B8900001D1C0F85C904FF4407A0B2D01D1C0F873
:10B8A0005CA04FF480670C2D00D1C7654FF4A06CED
:10B8B0000D2D04D101E07BE12CE0C0F85CC08D7857
:10B8C000D0F85C80082C4544DD6000D1C265092CAD
:10B8D00000D1C6650A2C01D1C0F85C900B2C01D1B7
:10B8E000C0F85CA00C2C00D1C7650D2C01D1C0F8AC
:10B8F0005CC08979C06D4FF4C06401449960A8B2FE
:10B900006A4B04E0A04200D21A54401C80B2884224
:10B91000F8D952E161484B798030862B03D0802BD7
:10B9200001D0882B09D1CC79862C06D14C7A862C73
:10B9300008D0802C06D0882C04D0842B7ED0822B7B
:10B940007DD03AE18D780E7905EB06256D08C0E9CA
:10B95000105641F27076882B02D0802B04D005E07F
:10B9600005F57A75056401E0AB1903648B79097AF2
:10B97000C16403EB012149088164882C02D0802C2A
:10B9800003D004E001F57A7100E0314481640C4693
:10B990003E4D016CE03541F66F068C420AD98BB200
:10B9A00005E0B34201D825F813205B1C9BB2A342EB
:10B9B000F7D909E0A3B205E0B34201D825F8132076
:10B9C0005B1C9BB28B42F7D9304C42F60470E034DA
:10B9D00004EB0009801E04EB0008001F2718801EDE
:10B9E0002618801EDFF8C8A004F53C55044441F237
:10B9F0007D720AF110000A9091422ED3501D8142AF
:10BA00002BD8B9F90010CAF81410B8F90010491E63
:10BA1000CAF81010B5F90010CAF80C100991B7F95E
:10BA20000010CAF808100891B6F90010CAF80410FE
:10BA30000791B4F900101C228B4601E054E085E028
:10BA4000CAF8001068460A9916F099FC58460DF19C
:10BA50001C0BBBE80E0014F0D9F8104841F27D71C0
:10BA60008030806C88423ED3491D88423BD8B9F96A
:10BA70000010CAF81410B8F90010491ECAF81010C6
:10BA8000B5F9005016E00000521B00204C2C00209D
:10BA9000242C01402434014000C003080000002091
:10BAA0006028002080010020711000205212002028
:10BAB00030630020CAF80C50B7F90070CAF808705B
:10BAC000B6F90060CAF80460B4F90040CAF8004052
:10BAD0001C2268460A9916F052FC2B463A4631461B
:10BAE000204614F093F868E0CB79862B65D14B7A29
:10BAF000842B62D18C780B79436404EB03235B08BD
:10BB000003648C79097AC16404EB012149088164DA
:10BB1000FB488B42A0F6EA14A0F6EA0508D312E02F
:10BB2000C82B03D240F82320E254EA545B1C9BB29A
:10BB30008B42F5D941E0C82903D240F82120625454
:10BB40006A54491C89B29942F5D936E0CB79862BE3
:10BB500033D14B7A822B30D18C780B79436404EB50
:10BB600003235B0803648C79097AC16404EB012127
:10BB70004908E44C8164A4F2EA75A4F2EA608B42BD
:10BB800008D312E0FF2B03D844F82320EA54C25410
:10BB90005B1C9BB28B42F5D90FE0FF2903D844F818
:10BBA00021206A544254491C89B29942F5D904E0D3
:10BBB000102E02D1815C994381540BB00820BDE85E
:10BBC000F08FF0B5D04900230144012591F801C060
:10BBD0001C46BCF1100F05D10309C0F3420005FA61
:10BBE00000F084B2C94ECA4A96F83200A8B3B6F83B
:10BBF0007E60A2F60E30875DFF074ED0D75C2742ED
:10BC000003D0BCF1000F05D04DE0BCF1100F01D105
:10BC10002743D754CA78842A45D14A79802A42D109
:10BC20000B79BC4C032BA4F1800217D81B02A36034
:10BC300089781944D165425CD30703D002F07E02B3
:10BC4000425430E042F081024254B6F57A7F2AD065
:10BC5000815D01F07F01815525E01EE0052B02D0BA
:10BC6000180904D01FE08878F4F7F7FB1BE0082BD5
:10BC700019D30D2B17D81802A0F50060A0608978A1
:10BC80000844D065F4F743FCA34918B1D26D0020F5
:10BC9000885408E0D06D0D5405E0BCF1100F02D1BE
:10BCA000D05CA043D0540420F0BD2DE9F04F020930
:10BCB000C0F342034FF0010B0BFA03F18CB292492F
:10BCC000DFF848A2DFF844920D180AF16A0A95F8E5
:10BCD000038099F855C09AF8017099F83210002045
:10BCE000DFF82CE209F58076B8F1840F24D2AB7826
:10BCF0008A4DBCF1010F05EB08251D444B46F56547
:10BD00000ED08AF800708AF8011000BF83F8320064
:10BD10001EF80210824E214207D0735DDB077CE0E3
:10BD200083F8550083F85600F0E7755DED077EE077
:10BD3000A1430EF80210E0E027D14B46BCF1010F01
:10BD40000CD08AF800708AF8011000BF83F8320026
:10BD50001EF802007646204205D00DE083F855001B
:10BD600083F85600F2E7A878F4F77FFB20B9B05CBF
:10BD70002043B05483F832B0A878F4F776FB00285B
:10BD800002D0B05CA043B054B7E0B8F1850F13D037
:10BD9000B8F1860F30D0B8F18E0F4ED0B8F1880FC1
:10BDA00022D3A8F18808B8F1080F6DD2DFE808F0B7
:10BDB00066687C8084886C8C4B46BCF1010F0BD08C
:10BDC0008AF800708AF8011083F832001EF8020029
:10BDD000544E00EA040740E083F8550083F856000B
:10BDE000F2E700BF89F832B087E0AB78F35CE3BBE1
:10BDF000A0430EF8020080E04B46BCF1010F0FD0CB
:10BE00008AF800708AF8011083F832001EF80210D8
:10BE1000454E214209D0AB78F35C002B88D06CE012
:10BE200083F8550083F85600EEE7AD78755D002D78
:10BE3000F4D021430EF80210D4E74B46BCF1010FB9
:10BE400017D08AF800708AF8011000BF83F832001A
:10BE50001EF80200354E00EA0407002FC5D1AD7868
:10BE6000755D002DC4D0204300E046E00EF80200CE
:10BE7000B8E783F8550083F85600E7E7AB7802E0AF
:10BE8000AB7803F58073F3654B46BCF1010F1FD00F
:10BE90008AF800708AF8011083F832001EF8020058
:10BEA0007546204219D021E0AB7803F50073EAE72C
:10BEB000AB7803F54073E6E7AB7803F58063E2E720
:10BEC000AB7803F5A063DEE7AB7803F5FA53DAE766
:10BED00083F8550083F85600DEE7F06DF4F717FBA2
:10BEE00020B1A85C2043A85483F832B0F06DF4F779
:10BEF0000EFB10B9A85CA043A85402205FE6000026
:10BF00003C2500203C21002000C003080000002048
:10BF10006028002080010020521200200080FFFFD6
:10BF2000521D0020C110002052190020521B002079
:10BF30002DE9F04F0209C0F342034FF0010B0BFA59
:10BF400003F18CB2FB49DFF8F0A30D18AAF16A09DE
:10BF500095F8038099F855C09AF8017099F8321055
:10BF60000020DFF8D8E309F58076B8F1840F29D2F4
:10BF7000AB78F34DBCF1010F05EB08251D444B4692
:10BF8000F5650DD08AF800708AF8011083F8320048
:10BF90001EF80200EB4E20420DD0755DED077BE0F0
:10BFA00083F8550083F85600F0E7A0430EF802002E
:10BFB00089F832B0CFE0735DDB0758E020430EF81C
:10BFC0000200C8E026D14B46BCF1010F19D08AF817
:10BFD00000708AF8011000BF83F832001EF80200DA
:10BFE0007646204208D0A878F4F73FFA20B1B05C3A
:10BFF000A043B05483F832B0A878F4F736FA28B1E9
:10C00000A9E083F8550083F85600E5E7B05C2043CB
:10C01000B054A0E0B8F1850F13D0B8F1860F29D045
:10C02000B8F18E0F40D0B8F1880F22D3A8F188085C
:10C03000B8F1080F56D2DFE808F04F51696D7175FD
:10C0400055794B46BCF1010F0CD08AF800708AF884
:10C05000011000BF83F832001EF80200BA4E00EA59
:10C06000040716E083F8550083F85600F2E7002B2A
:10C07000A4D170E04B46BCF1010F10D08AF80070DB
:10C080008AF8011083F832001EF80200AF4E00EA71
:10C090000407F7B1AD78755D002D8FD185E783F882
:10C0A000550083F85600EDE74B46BCF1010F0BD06D
:10C0B0008AF800708AF8011083F832001EF8020036
:10C0C000A34E00EA0407E4E783F8550083F856001E
:10C0D000F2E7AB78F35CCAE7AB7802E0AB7803F544
:10C0E0008073F3654B46BCF1010F23D08AF80070D2
:10C0F0008AF8011083F832001EF8020075462042CB
:10C1000022D0F06DF4F703FAC8B11DE0AB7803F567
:10C110000073E6E7AB7803F54073E2E7AB7803F52D
:10C120008063DEE7AB7803F5A063DAE7AB7803F56D
:10C13000FA53D6E783F8550083F85600DAE7A85C8F
:10C14000A043A85483F832B0F06DF4F7E0F910B1D1
:10C15000A85C2043A854022031E52DE9F0430209F0
:10C16000C0F342014FF0010C0CFA01F18CB271499D
:10C17000714E08446A3EC17896F832806F4D4FF098
:10C18000000906F5807784291AD26D4B807803EB7D
:10C1900001210144F965B8F1000F10D0A85C694B8A
:10C1A000204205D15F5CFF0702D02043A8541EE067
:10C1B00086F83290595CC90701D1A043A85484E0A5
:10C1C00018D1B8F1000F35D0A95C5F4B214203F1C3
:10C1D000510303D1877833F81770A7B386F83290EC
:10C1E000807833F8100028B3A143A9546DE086F895
:10C1F00032C06AE085290ED086291CD08E2923D032
:10C20000882962D38839082934D2DFE801F02D2F3C
:10C210003A3E4246334AB8F1000F56D0A95C4A4B29
:10C2200001EA040717E000BF86F832908078185CB6
:10C230000028D9D049E0B8F1000F46D0A95C434BA3
:10C2400001EA040707E00CE0B8F1000F3DD0A95C5B
:10C250003F4B01EA0407002FE6D18778DF5D002F0E
:10C26000E2D02143A954C2E7807802E0807800F54B
:10C270008070F865B8F1000F27D0A85C204214D078
:10C280001DE0807800F50070F3E7807800F54070DD
:10C29000EFE7807800F58060EBE7807800F5A0603C
:10C2A000E7E7807800F5FA50E3E7F86DF4F72FF947
:10C2B00028B1A85C2043A85486F832C001E086F873
:10C2C0003290F86DF4F723F910B10220BDE8F08345
:10C2D000A85C72E72DE9F0430209C0F342014FF078
:10C2E000010C0CFA01F18CB21249134E08446A3E5B
:10C2F000C17896F83280114D4FF0000906F580772D
:10C3000084292AD20E4B807803EB01210144F96580
:10C31000B8F1000F0DD0A85C0A4B204202D05F5C40
:10C32000FF0717D086F83290595CC90701D0204327
:10C33000A85497E000C003086A000020602800208D
:10C340000080FFFF521D0020C11000205219002064
:10C35000521B0020A043A8540CE017D1B8F1000FE5
:10C360000AD0A95CFE4B214207D0877833F81770BA
:10C37000AFBB02E086F832C074E086F83290807875
:10C3800033F8100010BB2143A9546BE085290ED06F
:10C3900086291CD08E2923D0882963D3883908297F
:10C3A00034D2DFE801F02D2F45494D513355B8F116
:10C3B000000F57D0A95CEA4B01EA0407513B16E095
:10C3C00086F832908078185C0028DCD14AE0B8F119
:10C3D000000F47D0A95CE34B01EA040707E00CE03B
:10C3E000B8F1000F3ED0A95CDF4B01EA0407002F33
:10C3F000E6D08778DF5D002FE2D1A143A954B9E7E9
:10C40000807802E0807800F58070F865B8F1000F60
:10C4100028D0A85C204203D0F86DF4F778F8D8B1A2
:10C4200086F83290F86DF4F772F8D8B1A85C7EE720
:10C43000807800F50070E8E7807800F54070E4E768
:10C44000807800F58060E0E7807800F5A060DCE7A8
:10C45000807800F5FA50D8E7A85CA043A85486F885
:10C4600032C0DFE7022031E7F0B50209C0F3420134
:10C47000012707FA01F18CB2BC49DFF8F4C2084485
:10C48000BC4DC1780CF58076842916D2BA4B8078E1
:10C4900003EB01210144F165A5F60E33A85C595C5C
:10C4A00020424FEAC17101D021B16EE011B12043A9
:10C4B000A85410E0A043A85467E00FD1A84B80789F
:10C4C000A95C33F81000214203D000B3A143A95462
:10C4D0005BE060B3FAE78CF8327056E085290ED045
:10C4E0008E2915D0862918D088294ED38839082955
:10C4F00026D2DFE801F01F21292D31352539A95C2D
:10C50000974B01EA0406513B0BE00028DED03CE0EB
:10C51000A95C954B01EA040603E0A95C914B01EA92
:10C5200004068078002E185CEFD10028CED021437D
:10C53000A954D0E7807802E0807800F58070F0653B
:10C54000A85C204214D01CE0807800F50070F6E76B
:10C55000807800F54070F2E7807800F58060EEE7C3
:10C56000807800F5A060EAE7807800F5FA50E6E709
:10C57000F06DF3F7CCFF20B1A85C2043A8548CF8F1
:10C580003270F06DF3F7C3FF08B10220F0BDA85C74
:10C5900090E7F0B50209C0F34201012707FA01F163
:10C5A0008CB27249DFF8C8C10844724DC1780CF5ED
:10C5B0008076842915D2704B807803EB01210144E9
:10C5C000F165A5F60E33A85C595C20424FEAC171B3
:10C5D00003D019B9A043A8540DE061B32043A85477
:10C5E00069E00FD15E4B8078A95C33F810002142DE
:10C5F00004D080BB03E08CF832705CE0D8B92143F2
:10C60000A95458E085290ED08E2915D0862918D036
:10C61000882950D38839082926D2DFE801F01F2164
:10C620002D313539253DA95C4D4B01EA0406513BBE
:10C630000BE00028E3D13EE0A95C4B4B01EA040685
:10C6400003E0A95C474B01EA04068078002E185CE1
:10C65000EFD00028D3D1A143A954CCE7807802E0E1
:10C66000807800F58070F065A85C20421DD0F06DE8
:10C67000F3F74DFFA0B118E0807800F50070F2E705
:10C68000807800F54070EEE7807800F58060EAE79A
:10C69000807800F5A060E6E7807800F5FA50E2E7E0
:10C6A000A85CA043A8548CF83270F06DF3F72FFF0C
:10C6B00008B1A85C92E70220F0BD2DE9F0412B49BA
:10C6C0000446214400204D780246102D05D1200952
:10C6D000C4F34202012191408AB2254B254993F8C7
:10C6E0003260DEB3B3F87E30A1F60E36F35CDB07C2
:10C6F0005DD00B5C134201D025B15DE0102D01D15E
:10C7000013430B542046F7F7EEFD1C4BA3F18007B3
:10C71000D86AC21700EB127121F00F05461B0911F0
:10C72000CD1701EB157525F00F054D1B00EB1261C0
:10C73000091200EB1250C7E914654FEAE17C0013BF
:10C7400001EB1C7CC2172CF00F0C00EB127203F1F2
:10C750008007A1EB0C0122F00F0211E027E000009E
:10C760001211002052190020521B002000C00308A3
:10C7700000000020602800200080FFFF0001002052
:10C78000801AC7E904104FF47A72504301EBC102DA
:10C7900002EB011100EB810005EB850100EB41008C
:10C7A0003044241DD862A0B2F9F7DEF904E0102D60
:10C7B00002D10B5C93430B540820BDE8F0812DE9B6
:10C7C000F0470446FF48002120440A464378102BD6
:10C7D00005D12109C4F342020120904082B2FA4DF2
:10C7E000FA4895F83260002E7ED0B5F87E50A0F65B
:10C7F0000E36755DED077DD0455C154201D023B145
:10C800007DE0102B01D1154345542046F8F7F1FA8D
:10C81000DFF8BCA3DAF82C00C21700EB127323F088
:10C820000F01451AAAF18001A9461B110D65DD17FC
:10C8300003EB157525F00F05A3EB050800EB12635C
:10C840001D12EE1705EB167626F00F06A5EB060C6B
:10C8500000EB12552D13EE1705EB167601F58073DC
:10C8600026F00F06AF1BC1F85480C3E904C700EBE4
:10C8700012400014C21700EB127323F00F05461B81
:10C88000C3F3031500EB126300EB1250C3F3032351
:10C89000C0F30330C1E91230C1E91065CD49484306
:10C8A00043F609514B4340F635414D4340F2712167
:10C8B00000EB83104E4300EB451000EB061107EB35
:10C8C0004700C0EBC71001EBC0000CEBCC0101EB43
:10C8D0000C1100EB810008EB880100EB410000EB3C
:10C8E00009010834A0B200E004E0CAF82C10FAF7FD
:10C8F00059FB04E0102B02D1435C934343541020B6
:10C90000BDE8F0872DE9F041AE49044621440020FE
:10C910004D780246102D05D12009C4F342020121B1
:10C9200091408AB2A84BA94993F83260F6B3B3F8A4
:10C930007E30A1F60E36F35CDB073BD00B5C134276
:10C9400001D025B13BE0102D01D113430B542046FB
:10C95000F7F7C9FC9E4B0A20A3F18006DA6A92FB26
:10C96000F0F191FBF0F700FB112500FB1711C6E970
:10C970001451642692FBF6F797FBF0FC00FB1C7742
:10C980004FF47A7C92FBFCF292FBF0FC03F1800600
:10C9900000FB1C20C6E9047007EB0010000200EB4E
:10C9A00001102844241DD862A0B200E002E0F9F78B
:10C9B000DBF804E0102D02D10B5C93430B540820EC
:10C9C000FBE62DE9F05F7F490446214400204D78C5
:10C9D0000246102D05D12009C4F3420201219140E5
:10C9E0008AB2794B794993F83260002E71D0B3F84E
:10C9F0007E30A1F60E36F35CDB076AD00B5C134287
:10CA000001D025B16AE0102D01D113430B5420460B
:10CA1000F8F7EFF9DFF8B8B10A21ABF18000DBF8E5
:10CA20002C2000F5807792FBF1F301FB1325AA4639
:10CA3000056593FBF1F501FB1533994643656423C6
:10CA400092FBF3F393FBF1F501FB15354FF47A7389
:10CA500092FBF3F393FBF1F601FB163642F21073EF
:10CA600092FBF3F3C7E90456B3FBF1F701FB173769
:10CA7000594B083492FBF3F3B3FBF1FC01FB1C3C74
:10CA8000564B92FBF3F3B3FBF1F801FB1833DFF8DD
:10CA9000448192FBF8F2B2FBF1F801FB1821C0E9E6
:10CAA0001231C0E9107C03EB0110000600EB0C50C2
:10CAB00000EB074000EB063000EB052000EB09100F
:10CAC00000EB0A01A0B2CBF82C10FAF76BFA05E0E4
:10CAD000FFE7102D02D10B5C93430B541020BDE8EF
:10CAE000F09FF0B537490023014401224E781C46DF
:10CAF000102E05D10309C0F3420002FA00F084B2FF
:10CB0000314D324895F83270002F73D0B5F87E5011
:10CB1000A0F60E377D5DED076CD0C55C254201D0D7
:10CB200026B1A4E0102E01D12543C554264C0F791F
:10CB30008034042F21D188790B7A00EB03232364FE
:10CB400058077DD18878C5184E2D79D2254EDFF84B
:10CB500090E04FF6FF75B6F90060AEF1A00CC6F19B
:10CB60000F06F540034406E03EF810602E402CF816
:10CB70001060401C80B28342F6D8052F77D18879A7
:10CB80000B7A00EB03252564680770D18B78581960
:10CB90004E286CD214495C1901F1500003E0CD5CC1
:10CBA000C5545B1C9BB29C42F9D8104C00232578DD
:10CBB0002DB90E780425F6B10D4E356002706478FB
:10CBC000ECB123E000C00308000000206028002032
:10CBD0000001002080969800A086010040420F00CE
:10CBE000B2110020345C002071100020A803002046
:10CBF0001408014036E0F84E35600370DFE74E78E8
:10CC0000F64D4FF48074F6B16C614270F44C8F783D
:10CC10004FF48046251DCFB12E608270CF784FF43F
:10CC20000056B7B12E60C2700F794FF480569FB195
:10CC30002E6002714E794FF4006186B1296000E0E8
:10CC400015E0427113E02C614370DFE726608370CA
:10CC5000E4E72660C370E7E726600371EAE7216036
:10CC6000437104E0102E02D1C15CA143C1540820DD
:10CC7000F0BDF0B50446DC49DA480D1900F501763F
:10CC800090F83220A97ACAB1D84AB0F87E00105C78
:10CC9000C00713D0022918D22046F7F724FBA6F5C7
:10CCA0008277A97AA6F10802F86A42F82100241DC9
:10CCB000A0B2F7F718FBA97AF86A04E0022904D2B7
:10CCC000CB4A0020505446F821000C20F0BD2DE93D
:10CCD000F05F0746C4480021C5190A466E784FF038
:10CCE0000108102E05D13909C7F3420208FA02F0F3
:10CCF00082B2BC4CBF4894F83230002B7ED0BB4B84
:10CD0000B4F87EC013F80C30DB0777D0435C1342D5
:10CD100001D026B185E0102E01D11343435438468B
:10CD2000F7F7E1FA41F69070F3F7F1FB0100DFF855
:10CD3000C8C2B24EDFF8C892DFF8C8B24FF00002A6
:10CD40004FF003004FF0060340F2277A0AD0A9798A
:10CD50009A2907D1E979862904D1297A11B9697A02
:10CD6000862908D041F69070F3F7D1FB00B3A8797B
:10CD70009E2815D01CE0E41D04F8052CA24FBCF839
:10CD80002C10317039807070B9F99800C11700EB20
:10CD90001161090AB170F070327186F8058023E0E4
:10CDA000E879862804D1287A10B9687A862804D0D0
:10CDB0003F1DB8B2F8F7D8FE33E0E41D04F8052CA7
:10CDC0009CF82C0030707370B9F99600C21700EB14
:10CDD0001262120AB270F070B9F99400C11700EB38
:10CDE0001161090A31717071E37706218348F3F705
:10CDF0000DFAC0F30722CCF8280000E00CE0E17F38
:10CE00007254491CC9B201227054491CE177514641
:10CE1000584615F089F804E0102E02D1435C934384
:10CE2000435408205BE670B56F4904462144002056
:10CE30004B780246102B05D12009C4F34202012190
:10CE400091408AB2674D6B4995F83260B6B1674E32
:10CE5000B5F87E50755DED0710D00D5C154201D020
:10CE600023B110E0102B01D115430D542046F7F7E4
:10CE7000C0FF0834A0B2FAF795F804E0102B02D1F5
:10CE80000B5C93430B54102070BDF0B5564987B02E
:10CE90000144C878862806D14879862806D080289B
:10CEA00004D0882802D0002007B0F0BD4D4A92F887
:10CEB0003230E3B34D4BB2F87E209A5CD2074ED0AD
:10CEC000484A8B7880320979516403EB0121490883
:10CED000116400224A4B862804D0882805D0802877
:10CEE00008D03CE023F8112039E003EB4100A0F822
:10CEF000D02734E003EB410042F6E063C2520D2933
:10CF00002DD312292BD840488038B0F9001000F5F5
:10CF1000E0604161A0F20271B1F90010491E0161A7
:10CF2000A0F20471B1F90070891EC76000E016E03C
:10CF3000B1F90060891E8660B1F90050891E456014
:10CF4000B1F9004000F1100104601C22684615F0A0
:10CF500016FA3B4632462946204612F057FE042078
:10CF6000A2E770B5044620480022204413464078CA
:10CF7000102805D12209C4F34203012199408BB244
:10CF8000184D1C4995F83260FEB1184EB5F87E5028
:10CF9000755DED0719D08D5C1D4201D020B119E0FF
:10CFA000102801D11D438D542046F7F79CF91248F3
:10CFB000C16AA1F5FE42FF3A01D1144900E0491CC3
:10CFC000C1622046F8F7D0FD04E0102802D1885C49
:10CFD00098438854042070BD10080140001001409F
:10CFE000101801400000002000C00308521D00205E
:10CFF000711000206028002000010020DB070020C5
:10D000002C2D002000480040B05C00200080FFFF75
:10D0100070B50446F8480022204413464578102D88
:10D0200005D12209C4F342010120884083B2F348AC
:10D03000F34990F8326006B3B0F87E00A1F60E36E0
:10D04000305CC00719D0885C184201D025B119E0C6
:10D05000102D01D1184388542046F7F744F9E948C8
:10D06000C16A11F5004F05D0491EC1622046F8F78C
:10D070007BFD07E047F6FF71F7E7102D02D1885CD2
:10D08000984388540420A6E770B50446DA48002285
:10D09000204413464078102805D12209C4F34203E6
:10D0A000012199408BB2D54DD54995F8326006B330
:10D0B000B5F87E50A1F60E36755DED0719D08D5C82
:10D0C0001D4201D020B119E0102801D11D438D541B
:10D0D0002046F7F78EFECB486FF00042C16A9142BE
:10D0E00001D1C90700E0491CC1622046F9F75AFF87
:10D0F00004E0102802D1885C9843885408206AE72D
:10D1000070B50446BC480022204413464578102DD3
:10D1100005D12209C4F342010120884083B2B748F7
:10D12000B74990F8326006B3B0F87E00A1F60E362B
:10D13000305CC00719D0885C184201D025B119E0D5
:10D14000102D01D1184388542046F7F752FEAD4800
:10D15000C16AB1F1004F05D0491EC1622046F9F7FE
:10D1600021FF07E06FF00041F7E7102D02D1885C46
:10D170009843885408202EE770B504469E48002145
:10D1800020440A464378102B05D12109C4F34202FA
:10D190000120904082B2994D994895F832602EB3A3
:10D1A000B5F87E50A0F60E36755DED071ED0455CD5
:10D1B000154201D023B11EE0102B01D11543455477
:10D1C0002046F7F790F88F4DA5F18006E86A3065A4
:10D1D000201D80B2F7F787F8E86A7065316D083472
:10D1E0000140A0B2E962F8F7BFFC04E0102B02D1C5
:10D1F000435C934343540C20EDE670B504467E48EF
:10D20000002120440A464378102B05D12109C4F39C
:10D2100042020120904082B2784D794895F8326000
:10D2200036B3B5F87E50A0F60E36755DED071FD00B
:10D23000455C154201D023B11FE0102B01D11543ED
:10D2400045542046F7F7D5FD6E4DA5F18006E86AF6
:10D25000B06504F1080080B2F7F7CBFDE86AF0652D
:10D26000B16D10340140A0B2E962F9F79BFE04E011
:10D27000102B02D1435C934343541820ABE670B5A6
:10D2800004465D48002120440A464378102B05D10E
:10D290002109C4F342020120904082B2574D584800
:10D2A00095F832602EB3B5F87E50A0F60E36755D57
:10D2B000ED071ED0455C154201D023B11EE0102BB6
:10D2C00001D1154345542046F7F70DF84D4DA5F112
:10D2D0008006E86A3065201D80B2F7F704F8E86A36
:10D2E0007065316D08340143A0B2E962F8F73CFC87
:10D2F00004E0102B02D1435C934343540C206AE6B4
:10D3000070B504463C48002120440A464378102B5F
:10D3100005D12109C4F342020120904082B2374D69
:10D32000374895F8326036B3B5F87E50A0F60E3621
:10D33000755DED071FD0455C154201D023B11FE09C
:10D34000102B01D1154345542046F7F752FD2D4DC2
:10D35000A5F18006E86AB06504F1080080B2F7F72D
:10D3600048FDE86AF065B16D10340143A0B2E9628E
:10D37000F9F718FE04E0102B02D1435C93434354A9
:10D38000182028E670B504461B48002120440A46B0
:10D390004378102B05D12109C4F3420201209040AB
:10D3A00082B2164D164895F832606EB3B5F87E50CD
:10D3B000A0F60E36755DED0727D0455C154201D00D
:10D3C00023B127E0102B01D1154345542046F6F731
:10D3D0008AFF0C4DA5F18006E86A3065201D80B2F9
:10D3E000F6F781FFE86A7065316D08344140A0B2FC
:10D3F000E962F8F7B9FB0DE000C003080000002067
:10D400006028002000010020FFE7102B02D1435CC0
:10D41000934343540C20DEE570B50446F8480021E0
:10D4200020440A464378102B05D12109C4F3420257
:10D430000120904082B2F34DF34895F8326036B344
:10D44000B5F87E50A0F60E36755DED071FD0455C31
:10D45000154201D023B11FE0102B01D115434554D3
:10D460002046F7F7C6FCE94DA5F18006E86AB065ED
:10D4700004F1080080B2F7F7BCFCE86AF065B16D12
:10D4800010344140A0B2E962F9F78CFD04E0102BA2
:10D4900002D1435C9343435418209CE52DE9FE4F91
:10D4A000D74900220C18012567781646102F05D1A0
:10D4B0000209C0F3420105FA01F18EB2D14BD24903
:10D4C00093F832C0BCF1000F7CD0B3F87E30A1F6E7
:10D4D0000E3B1BF80330DB07F6D08B5C334201D0E8
:10D4E00027B1CCE1102F01D133438B54F6F7FBFE6B
:10D4F000A07A217B002700EB0120C2494FF4C06EC7
:10D5000080310865E278842A73D16279802A70D1EB
:10D510002279042A15D10023DFF8F4C24F650EE00A
:10D52000A6781E444D2E08D83CF816602EB9D1F8C6
:10D53000548005FA03F646444E655B1C9BB2834259
:10D54000EEDB052A1AD1DFF8C8920023A9F15109B0
:10D550004F6511E0A67806EB030CBCF14D0F09D81E
:10D5600009EB030C16F80C6026B14E6D05FA03F8B2
:10D5700046444E655B1C9BB28342EBDB082A1CD3FE
:10D580000D2A1AD80023F046DFF888924F6512E082
:10D59000A67806EB022CA3F500666644464508DA39
:10D5A00019F806602EB1D1F854C005FA03F66644A6
:10D5B0004E655B1C9BB28342EADB032A19D8002329
:10D5C0004F6514E056E1A67803EB022806EB080C41
:10D5D000F4450AD206EB0B0C1CF80860F60704D0E1
:10D5E0004E6D05FA03F846444E655B1C9BB28342C0
:10D5F000E9DBE2790292842A76D1627A802A74D1B8
:10D60000082872DC002870DDDFF800C200230CF16E
:10D61000800C2A460646CCF8105002E052005B1CF3
:10D620009BB2B342FADBCCF81020237A9146052B4B
:10D6300024D1A6790096D1F854C066444E2E53DA10
:10D64000DFF8CC81E246A8F15108C4440026CDF8A9
:10D6500004C011E0564504D1DDE9008C08F80C50F7
:10D6600008E0DFF8AC81DDF800C0A8F15108B04453
:10D670000CF80870761CB6B29642EBDB082B23D36D
:10D680000D2B21D8D1F85480A279C44602EB032295
:10D69000A8F5006802EB08060E64764514D2E04651
:10D6A0000022B246A6EB080E0CE0424503D1594ECB
:10D6B00006F80A5004E0574E0EEB020C06F80C7008
:10D6C000521C92B24A45F0DB0F2B1FD1A6794A6D4E
:10D6D000B6461644FF2E39DCDFF83CC192460CEB0F
:10D6E0000A02002600920FE030E040E0564504D1E7
:10D6F000DDF800C00EF80C5004E0DFF81C81B044E7
:10D700000EF80870761CB6B24E45EFDB042B1DD226
:10D710004E6DA27906EB032302EB030CC1F840C067
:10D72000BCF57A7F12D24B460022E246ACEB0609EA
:10D730000AE0B24202D10BF80A5003E009EB0208FA
:10D740000BF80870521C92B29A42F2DB029A862AB7
:10D750000DD1667AFF222D4B304F862E08D0882EB1
:10D760001AD0802E32D0842E5AD0822E6DD086E0F0
:10D77000042810DC00280EDDC0F10800C240D86A81
:10D7800002400A65A079237A00EB03204008954007
:10D79000086427F8105072E0042870DC00286EDD61
:10D7A000C0F10800C240D86A02400A65A079237A15
:10D7B00000EB03204008086441F2873188425ED8BC
:10D7C00007EB40009540A0F8D05758E0042856DCFD
:10D7D000002854DDC0F10800C240D86A02400A6542
:10D7E000A079237A00EB032040080864FF2846D87C
:10D7F00007EB4000954042F6E06145523FE00000F3
:10D8000000C0030800000020602800200001002064
:10D810001211002052120020521800202C2D00203E
:10D8200004282CDC00282ADDC0F10800C240D86A98
:10D8300002400A65A079237A00EB032040080864BF
:10D84000C7281CD89540FE4911E0042817DC0028A1
:10D8500015DDC0F10800C240D86A02400A65A0790F
:10D86000237A00EB032040080864F649954041F80C
:10D87000205004E0102F02D1885CB04388540C2063
:10D88000BDE8FE8F2DE9F84FEF4900220C18012565
:10D8900067781346102F05D10209C0F3420105FA3B
:10D8A00001F18BB2E94EEA4996F832C0BCF1000FA3
:10D8B0007CD0B6F87E60A1F60E3E1EF80660F60734
:10D8C000F6D08E5C1E4201D027B16FE3102F01D13C
:10D8D0001E438E54DF4E4FF0000BA6F58073C6F842
:10D8E00014B0A17A227B01EB0227C3E914755A46D2
:10D8F000294602E04900521C92B2BA42FADBD34AEE
:10D90000DFF850A38032AAF1800A5165E278842AB8
:10D910006FD16279802A6CD12379042B1AD1756179
:10D920000022DFF83493CAF82CB011E0A77807EB97
:10D93000020CBCF14D0F09D839F81C7037B9DAF870
:10D940002C8005FA02F7B844CAF82C80521C92B217
:10D950008A42EBDB052B1ED1DFF8FC9275610022B9
:10D96000A9F15109CAF82CB013E0A77807EB020C13
:10D97000BCF14D0F0BD809EB020C17F80C7037B146
:10D98000DAF82CC005FA02F8C444CAF82CC0521CBC
:10D9900092B28A42E9DB082B21D30D2B1FD8756187
:10D9A0000022DFF8B892CAF82CB016E0F9E2A778A6
:10D9B00007EB032CA2F500676744B7F5C06F0ADADE
:10D9C00019F807703FB1DAF82C7005FA02F808EB85
:10D9D000070CCAF82CC0521C92B28A42E7DB032B18
:10D9E00020D87561CAF82CB000224FF4C06BA9464C
:10D9F00016E017E094F802C002EB03270CEB0708CF
:10DA0000D8450BD2F4441CF80770FF0706D0DAF8AB
:10DA10002CC009FA02F7BC44CAF82CC0521C92B2BE
:10DA20008A42E7DB716909B9F6F75DFC8748FF2197
:10DA30008030026DC2F10803D940DAF82C30194069
:10DA400093B2416507E05F1E05FA07F60E4201D06A
:10DA5000394602E0BBB2002BF5D14165E779DFF82A
:10DA6000E0B1DFF8E0E141F2873942F6E06A0BF518
:10DA7000FE63862F1ED07A4E962F38D0B51EA62F65
:10DA80006BD0862F19D0962F7ED0A62F7DD0862FD3
:10DA900016D0962F7AD0A62F79D0862F13D0962F16
:10DAA00076D0A62F75D0862F10D0962F72D0A62FA5
:10DAB00071D07BE2657A862D0CD0657A882D6BD08B
:10DAC000657A802D69D0637A842B67D0637A822B44
:10DAD0007DD06BE2042AECDC002AEADDA279247A0C
:10DAE00002EB04225208026423F812105EE2677A05
:10DAF000862F4BD3872F47D8042A2ADC002A28DD1B
:10DB000094F808C094F806904FEA9C15C5F10008F7
:10DB10000CEB881809EB082C4FEA5C0CC0E910C824
:10DB2000C564862F06D003EB850505F54055B5F98C
:10DB30005A5006E075B103EB850505F54055B5F97A
:10DB40004A5041F26F7765448564BD4201D823F89D
:10DB50001510E7E0B6F90050F3E7667A862E16D383
:10DB6000872E12D8042AA4DC002AA2DDA779247A01
:10DB7000A209C2F1000C04EB8C14446407EB0424EA
:10DB8000C264640804640AE037E085E0B4E0F7E0CA
:10DB900033E166E1B2E194E120E0B1E01EE1862EDE
:10DBA00006D003EB820202F54052B2F9582006E09B
:10DBB0008AB103EB820202F54052B2F948202244B6
:10DBC0008264104641F26F7290428FD800E09DE16E
:10DBD00023F81010EAE1B5F90020F0E7042A85DC0B
:10DBE000002AF7DDA279247A02EB042252080264AB
:10DBF0004A45EFD803EB42007BE0677A882F7BD35E
:10DC0000892F45D8042A43DC002A41DD94F806C058
:10DC1000CDF800C094F808C0882F4FEA9C15C5F1D4
:10DC200000080CEB8818C0F84480C564DDF800C01B
:10DC30000CEB082C4FEA5C0CC0F840C019D011E086
:10DC40003C2500203C21002000C0030800000020EB
:10DC500060280020800100201211002052120020B4
:10DC6000465C002003EB850505F54055B5F95A5093
:10DC700006E075B103EB850505F54055B5F94A5049
:10DC8000654485644D454DD803EB4505A5F8D0178F
:10DC900048E0B6F90050F3E7667A882E74D3892EEF
:10DCA00029D8042A27DC002A25DDA779247AA209AD
:10DCB000C2F1000C04EB8C14446407EB04246408E8
:10DCC000C2640464882E06D003EB820202F540523F
:10DCD000B2F9582006E082B103EB820202F540520D
:10DCE000B2F948202244826410464A4503D803EB27
:10DCF0004000A0F8D01759E111E0B5F90020F1E794
:10DD0000042A3CDC002A3ADDA279247A02EB0422C0
:10DD100052080264FF2A32D803EB42022DE0657AF2
:10DD2000802D2CD3657A812D67D8042A27DC002A20
:10DD300025DDA779247AA209C2F1000C04EB8C142A
:10DD4000446407EB04246408C2640464802D06D094
:10DD500003EB820202F54052B2F95A2006E082B18A
:10DD600003EB820202F54052B2F94A202244826457
:10DD70001046FF2A03D803EB400222F80A1015E1EF
:10DD800002E0B6F90020F1E7667A802E34D3812EC6
:10DD900067D8042A30DC002A2EDDA779247AA2096C
:10DDA000C2F1000C04EB8C14446407EB04246408F7
:10DDB000C2640464802E06D003EB820202F5405256
:10DDC000B2F95820D2E732B103EB820202F5405299
:10DDD000B2F94820CAE7B5F90020C7E7042A0BDCEE
:10DDE000002A09DDA279237A02EB03225208026499
:10DDF000C72A01D84BF82210D8E0677A842F7DD348
:10DE0000852F2AD8042A28DC002A26DD94F808C0A9
:10DE100094F806904FEA9C15C5F100080CEB8818A1
:10DE200009EB082C4FEA5C0CC0E910C8C564842FCC
:10DE300006D003EB850505F54055B5F95A5006E0C7
:10DE400065B103EB850505F54055B5F94A506544C4
:10DE50008564C72D6AD84BF8251067E0B6F90050E5
:10DE6000F5E7677A842F2CD3852F5BD8042A28DC2A
:10DE7000002A26DD94F808C094F806904FEA9C1614
:10DE8000C6F100080CEB881809EB082C4FEA5C0C73
:10DE9000C0E910C8C664842F06D003EB860606F5D9
:10DEA0004056B6F9586006E04EB303EB860606F519
:10DEB0004056B6F9486066448664C72E01D84BF8D0
:10DEC0002610667A822E71D3832E6FD8042A6DDCD9
:10DED000002A6BDDA779247AA209C2F1000C04EBB9
:10DEE0008C14446407EB04246408C2640464822E26
:10DEF00047D003EB820202F5405201E013E002E05A
:10DF0000B2F9582044E0B5F90060D4E7042A4DDCAA
:10DF1000002A4BDDA279237A02EB03225208026425
:10DF20004EF8221042E0657A822D3FD3657A832D28
:10DF30003CD8042A3ADC002A38DDA779247AA209E1
:10DF4000C2F1000C04EB8C14446407EB0424640855
:10DF5000C2640464822D06D003EB820202F54052B3
:10DF6000B2F95A2014E032B103EB820202F54052BA
:10DF7000B2F94A200CE0B6F9002009E04EF8201072
:10DF800014E05AB103EB820202F54052B2F9482084
:10DF9000224482641046FF2AF0D907E0B5F9002038
:10DFA000F6E7102F02D1885C984388540C20BDE816
:10DFB000F88F2DE9F05F04460709C0F342014FF0E6
:10DFC000010808FA01F086B2FE48DFF8FC9390F8E9
:10DFD000321000297ED0B0F87E00A9F60E31085C20
:10DFE000C007F7D02046F6F77EF9DFF8E0A3AAF1E4
:10DFF0008005DAF82C002865201D80B2F6F773F949
:10E00000DAF82C00686504F10C0080B2F6F76BF9C1
:10E0100005F58073DAF82C001861D5E914129142E5
:10E020000ADDA1EB020C9CFBF0FCC3F814C0BCF1B0
:10E03000000F01D1C3F81480AA46914206DA551A9E
:10E0400095FBF0F55D610DB9C3F8148001287CDB08
:10E050009B46B0F5004F78DADD4B1D19EB7A862B25
:10E0600073D16B7BDB4C862B62D1AB7A95F80CC0FD
:10E0700003EB0C235B08CAF8403019F807C01CEA10
:10E08000060F0DD14CEA060C09F807C004EB430853
:10E090004FF0000CA8F802C0DFF83C8388F81DC0E0
:10E0A00004EB430CBCF80280B8F1000F01D124F856
:10E0B0001310BCF902808045CDDA914213DD34F8AB
:10E0C0001380BBF81410A8EB010109B224F8131057
:10E0D000914200E0F9E006DCACF80200012141F6D3
:10E0E0005D70F2F721FADAE91412D046914215DA9E
:10E0F000D8F84000BBF814C034F8103063441BB2A9
:10E1000024F81030934209DB04EB4000BBF81010F8
:10E110004180012141F65D70F2F706FAD8F840001F
:10E1200004EB40004188491C4180E87A86280CD1E4
:10E13000687B882866D1A97A287B534601EB0020AA
:10E140004FF47A7101EB500000E083E041F26E7110
:10E15000CAF8400088427DD819F80710314208D12A
:10E16000314309F8071004EB4002002151809A4A1C
:10E17000517704EB40014A881AB9B3F8502024F8CB
:10E180001020B1F902C0DBF81020944562DA1B6D53
:10E19000DAF85480434510DD34F810C0BBF8143071
:10E1A000ACEB03031BB224F81030434505DC4A8076
:10E1B000012141F65D70F2F7B7F9DAE91412D046A1
:10E1C000914215DAD8F84000BBF814C034F810308A
:10E1D00063441BB224F81030934209DB04EB400087
:10E1E000BBF810104180012141F65D70F2F79CF9F7
:10E1F000D8F8400004EB40004188491C4180E87A8F
:10E20000862869D1687B802866D1A97A287B554603
:10E2100001EB002041F2707101EB500041F66E01FC
:10E22000CAF84000884257D819F80710314208D17F
:10E23000314309F8071004EB400200215180664A7F
:10E24000517704EB40014A881AB9B5F8502024F8F8
:10E25000102000E038E0B1F90230DBF810205E4613
:10E26000934239DAD5E91437BB4210DD34F8103067
:10E27000B6F814C0A3EB0C031BB224F81030BB4259
:10E2800005DC4A80012141F65D70F2F74DF9D5E9D0
:10E290001402904212DA286CB38A34F81010194430
:10E2A00009B224F81010914208DB04EB4000318AD7
:10E2B0004180012141F65D70F2F736F9286C04EBDC
:10E2C00040014888401C488006E019F807003042A9
:10E2D00002D0B04309F807001020BDE8F09F70B5E8
:10E2E00004463B48002120440A464578102D05D1BC
:10E2F0002109C4F342020120904082B2314B3248DE
:10E3000093F832602EB3B3F87E30A0F60E36F35C8D
:10E31000DB071ED0435C134201D025B11EE0102D57
:10E3200001D1134343542046F5F7DDFF274DA5F1F6
:10E330008006E86A3065201D80B2F5F7D4FFE86AF0
:10E340007065316D08340844E862A0B2F7F70CFC40
:10E3500004E0102D02D1435C934343540C2070BD64
:10E3600070B504461A48002120440A464578102D0D
:10E3700005D12109C4F342020120904082B2114B21
:10E38000114893F832604EB3B3F87E30A0F60E36E3
:10E39000F35CDB072CD0435C134201D025B12CE0A9
:10E3A000102D01D1134343542046F5F79CFF074D30
:10E3B000A5F18006E86A3065201D80B2F5F793FF6D
:10E3C000E86A0CE000000020602800200001002026
:10E3D00000C003082C2D00205218002008E07065B2
:10E3E000316D0834081AE862A0B2F7F7BDFB04E00B
:10E3F000102D02D1435C934343540C2070BD70B583
:10E400000646FF48002130440A464478102C05D1C6
:10E410003109C6F342020120904082B2F94BFA481A
:10E4200093F8325085B3B3F87E30A0F60E35EB5C2E
:10E43000DB0748D0435C134201D024B148E0102CE4
:10E4400001D1134343543046F5F74DFFEF4DA5F18D
:10E450008004E86A2065301D80B2F5F744FFE86A61
:10E460006065216D0A0408D5020406D4A1F10101FA
:10E470006FEA010189B221651CE041EA0002120441
:10E4800003D44143E96219E01DE00A044FEA004267
:10E490000AD5002A12DA491EC943401EC04389B278
:10E4A00080B2C4E91410ECE7002A07DA401EC0432A
:10E4B00080B260654143C843401CE8620836B0B290
:10E4C000F7F752FB04E0102C02D1435C9343435412
:10E4D0000C2070BD70B50646C948002130440A467C
:10E4E0004478102C05D13109C6F342020120904036
:10E4F00082B2C44BC44893F83250002D63D0B3F8B5
:10E500007E30A0F60E35EB5CDB075CD0435C13423B
:10E5100001D024B15CE0102C01D1134343543046A8
:10E52000F5F7E1FEB94DA5F18004E86A2065301DDC
:10E5300080B2F5F7D8FEE96A6165E9B3206D02049F
:10E5400011D50A040FD4A0F101006FEA000082B2D5
:10E5500092FBF1F06FEA000303F10103226501FB76
:10E560001020EB6224E040EA0102120406D400BF4E
:10E5700090FBF1F201FB1200EA621CE002044FEA98
:10E58000014209D5002A19DA401EC043491E80B253
:10E59000C94389B22065EBE7002A0FDA491EC94357
:10E5A0008AB290FBF2F1CB435B1C02FB1100EB62E1
:10E5B000C043401C80B200E00AE060650836B0B29B
:10E5C000F7F7D2FA04E0102C02D1435C9343435492
:10E5D0000C2070BDF0B504468948002105190A4693
:10E5E0006E78102E05D12109C4F34202012090401B
:10E5F00082B2844B844893F832704FB3B3F87E30C4
:10E60000A0F60E37FB5CDB0722D0435C134201D03F
:10E6100026B122E0102E01D1134343542046F5F7D2
:10E6200062FE7A4FA7F18006F86A3065201D80B23D
:10E63000F5F759FEF96A7165E87A84280DD1687B8F
:10E6400080280AD100232246306DF2F725F804E035
:10E65000102E02D1435C934343540C20F0BDF8B517
:10E6600004466748002106190A467578102D05D121
:10E670002109C4F342020120904082B2614B6248FA
:10E6800093F83270A7B3B3F87E30A0F60E37FB5C78
:10E69000DB072ED0435C134201D025B12EE0102DB4
:10E6A00001D1134343542046F5F71DFE574FA7F100
:10E6B0008005F86A2865201D80B2F5F714FEF86A17
:10E6C000686504F1080080B2F5F70DFE05F580706D
:10E6D000FA6A0261F07B842810D1707C80280DD109
:10E6E00000200090D5E914012346F2F74DF905E02A
:10E6F000FFE7102D02D1435C934343541020F8BD33
:10E700002DE9F04107463E480023C4191D466178B3
:10E71000112905D13B09C7F342020120904085B27F
:10E720003848394A90F83260002E73D0B0F87E0035
:10E73000A2F60E36305CC007F7D0D05C284202D07B
:10E74000012904D07EE2112901D12843D054384652
:10E75000F5F7C9FD2D4EA6F18005F06A2865381D34
:10E7600080B2F5F7C0FDF06A686507F1080080B275
:10E77000F5F7B9FDF06A80363061E07B8628E1D19B
:10E78000607CDFF88C8086287CD1A17B207C68644B
:10E7900001EB00204008286438F91000296D8842F8
:10E7A00005DA08233A4601210220F1F775FF296CAA
:10E7B00038F91100296D884205DD08233A46022107
:10E7C0000120F1F769FF296C2B6D38F911209A426D
:10E7D00055D108EB4100696DB0F90200884205DAB5
:10E7E00008233A4601210220F1F756FF296C08EB75
:10E7F0004100696DB0F90200884211DD08230AE08A
:10E8000000C0030800000020602800200001002054
:10E810002C2D002011E23A4602210120F1F73CFFA5
:10E82000296C6B6D08EB4101B1F902209A4226D1A7
:10E83000B1F904003169884205DA08233A4601211A
:10E840000220F1F729FF296C08EB41003169B0F98A
:10E850000400884205DD08233A4602210120F1F731
:10E860001BFF296C08EB41003169B0F904008842B4
:10E8700005D1012108233A460846F1F70DFFE07B58
:10E8800086287DD1607C882877D1A07B217C696433
:10E8900000EB01204FF47A7101EB500041F26D71F1
:10E8A000286488426CD838F91000296D884205DA4E
:10E8B00008233A4601210220F1F7EEFE296C38F9CF
:10E8C0001100296D884205DD08233A460221012006
:10E8D000F1F7E2FE296C2B6D38F911209A4249D1EB
:10E8E00008EB4100696DB0F90200884205DA08239F
:10E8F0003A4601210220F1F7CFFE296C08EB4100D6
:10E90000696DB0F90200884205DD08233A4602210C
:10E910000120F1F7C1FE296C6B6D08EB4101B1F9E3
:10E9200002209A4226D1B1F904003169884205DA01
:10E9300008233A4601210220F1F7AEFE296C08EBCC
:10E9400041003169B0F90400884205DD08233A46E8
:10E9500002210120F1F7A0FE296C08EB410031698A
:10E96000B0F90400884205D1012108233A4608463F
:10E97000F1F792FEE07B862802D1607C802800E0DF
:10E980008CE077D1A17B207C686401EB002041F210
:10E99000707101EB500041F66D01286488427DD80A
:10E9A00038F91000296D884205DA08233A4601211A
:10E9B0000220F1F771FE296C38F91100296D8842A7
:10E9C00005DD08233A4602210120F1F765FE296C96
:10E9D0002B6D38F911209A4249D108EB4100696D3D
:10E9E000B0F90200884205DA08233A4601210220E4
:10E9F000F1F752FE296C08EB4100696DB0F9020095
:10EA0000884205DD08233A4602210120F1F744FE41
:10EA1000296C6B6D08EB4101B1F902209A4226D1B5
:10EA2000B1F904003169884205DA08233A46012128
:10EA30000220F1F731FE296C08EB41003169B0F991
:10EA40000400884205DD08233A4602210120F1F73F
:10EA500023FE296C08EB41003169B0F904008842BB
:10EA600005D1012108233A460846F1F715FEE07B5F
:10EA7000862813D1607C842870D1A07B217C00EB98
:10EA800001204008C5E91001C52888D8DFF8DC84DA
:10EA9000296D58F82000884207DA00E0CCE008230E
:10EAA0003A4601210220F1F7F7FD296C58F82100C0
:10EAB000296D884205DD08233A4602210120F1F73D
:10EAC000EBFD296C2B6D58F821209A4243D108EBBD
:10EAD0008100696D4068884205DA08233A460121C1
:10EAE0000220F1F7D9FD296C08EB8100696D4068BF
:10EAF000884205DD08233A4602210120F1F7CCFDCA
:10EB0000296C6B6D08EB81014A689A4223D18868B1
:10EB10003169884205DA08233A4601210220F1F7DB
:10EB2000BBFD296C08EB810031698068884205DDF6
:10EB300008233A4602210120F1F7AEFD296C08EBCB
:10EB4000810031698068884205D1012108233A4655
:10EB50000846F1F7A1FDE07B862873D1607C82280E
:10EB600070D1A07B217C00EB01204008C5E9100199
:10EB7000FD2867D8FE4C296D54F82000884205DA3C
:10EB800008233A4601210220F1F786FD286C296D01
:10EB900054F82000884205DD08233A46022101206E
:10EBA000F1F77AFD286C2A6D54F82010914249D172
:10EBB00004EB8000696D4068884205DA08233A4614
:10EBC00001210220F1F768FD286C696D04EB8000DB
:10EBD0004068884205DD08233A4602210120F1F70A
:10EBE0005BFD286C6A6D04EB80004168914229D17D
:10EBF00080683169884205DA08233A4601210220FB
:10EC0000F1F74AFD286C316904EB80008068884286
:10EC100005DD08233A4602210120F1F73DFD286C6D
:10EC2000316904EB8000806888420BD10121082300
:10EC30003A460846F1F730FD04E0112902D1D05CD4
:10EC4000A843D0541420BDE8F0812DE9F0430446D8
:10EC5000C848002120440A464578112D05D12109D4
:10EC6000C4F342020120904082B2C34BC34893F8E0
:10EC70003260002E66D0B3F87E70A0F60E36F65DD8
:10EC8000F6075FD0465C164202D0012D04D05EE04C
:10EC9000112D01D1164346545221994683F859103B
:10ECA0002046F5F720FBB44D4FF46161803505F542
:10ECB0008078286D4843696DC1EB011100EB81013B
:10ECC000D8F810000F18201D80B2F5F70CFB286D46
:10ECD0004FF461614843696DC1EB011100EB8101A3
:10ECE000D8F810000E1804F1080080B2F5F7FBFA0E
:10ECF000286D4FF461614843696DC1EB011100EB70
:10ED00008101D8F810000D18002189F85910BD4272
:10ED100005D20423224601210220F1F7BDFCBD42A9
:10ED200007D3B54205D80121042322460846F1F74E
:10ED3000B3FCB5420BD90423224603210220F1F78C
:10ED4000ABFC04E0112D02D1435C934343541020EB
:10ED5000BDE8F0832DE9F0410446864800212044B7
:10ED60000A464678112E05D12109C4F3420201203A
:10ED7000904082B2804D814895F83230F3B3B5F8B7
:10ED80007E70A0F60E33DB5DDB073ED0435C1342A2
:10ED900002D0012E04D03DE0112E01D11343435483
:10EDA000522005F8590F2046F5F79DFA724E4FF4A0
:10EDB0006161803606F58078306D4843716DC1EB36
:10EDC000011100EB8101D8F810000F18201D80B24E
:10EDD000F5F789FA306D4FF461614843716DC1EB0D
:10EDE000011100EB8101D8F81000084406F1800100
:10EDF0003844C86254202870083400E005E0A0B20E
:10EE0000F6F7B2FE0020287004E0112E02D1435C18
:10EE1000934343540C2016E72DE9F041044655482E
:10EE2000002120440A464678112E05D12109C4F359
:10EE300042020120904082B24F4D504895F8323046
:10EE4000F3B3B5F87E70A0F60E33DB5DDB073ED082
:10EE5000435C134202D0012E04D03DE0112E01D1BB
:10EE600013434354522005F8590F2046F5F73BFA57
:10EE7000414E4FF46161803606F58078306D48432D
:10EE8000716DC1EB011100EB8101D8F810000F1872
:10EE9000201D80B2F5F727FA306D4FF461614843C9
:10EEA000716DC1EB011100EB8101D8F8100008442D
:10EEB00006F18001381AC86256202870083400E034
:10EEC00005E0A0B2F6F750FE0020287004E0112EF5
:10EED00002D1435C934343540C20B4E62DE9F04146
:10EEE00024490022014413464D78112D05D1020911
:10EEF000C0F34203012199408BB21F4C1F4994F883
:10EF00003260C6B1B4F87E70A1F60E36F65DF60733
:10EF100011D08E5C1E4202D0012D04D010E0112DC4
:10EF200001D11E438E545C2104F8591FF6F71CFED4
:10EF30000020207004E0112D02D1885C9843885491
:10EF4000042080E62DE9F0410A49002201441346DD
:10EF50004D78112D05D10209C0F3420301219940DA
:10EF60008BB2054C054994F8326009E03C2500203D
:10EF70003C21002000C00308000000206028002081
:10EF8000C6B1B4F87E70A1F60E36F65DF60711D064
:10EF90008E5C1E4202D0012D04D010E0112D01D153
:10EFA0001E438E545E2104F8591FF6F7DDFD002044
:10EFB000207004E0112D02D1885C9843885404200D
:10EFC00041E62DE9F04F8346FF48002600EB0B0594
:10EFD00037466878102806D1CBF3420101208840DB
:10EFE0004FEA1B1687B2F94890F8321000297DD0FD
:10EFF000F749B0F87E00085CC007F8D05846F5F72E
:10F0000072F9E879862855D1697AF24C4FF4616A31
:10F010004FF00009862955D1EC48AA798030297A29
:10F02000416402EB01214A08EB49026431F9120004
:10F0300000283FDD47F6FF7398423BDAA1F2CC434C
:10F04000985D384237D001EB4200B4F90030B0F996
:10F0500004C09C4505DAB0F802804344A3EB0C03DE
:10F060004380B0F90430B4F900C0634506DDB0F860
:10F070000280C444ACEB03033C3343802388838089
:10F08000B0F90230534506DB31F812305B1C21F831
:10F090001230A0F80290D14831F91210C06A8142B2
:10F0A00008DB00235A4601210220F1F7F5FAE8793E
:10F0B000862807D0CAE03843985501EB42002388E0
:10F0C00083805FE0687A882863D1A8792A7ABF496B
:10F0D00000EB02208031400800F57A70C1E910028F
:10F0E000BD4A32F91010002945DD00E0AAE047F6DC
:10F0F000FF7399423FDA41F26D7188423BD8A2F228
:10F10000CC43995D394237D002EB4001B4F900C0DD
:10F11000B1F90430634505DAB1F80280C444ACEBC0
:10F1200003034B80B1F90430B4F900C0634506DD38
:10F13000B1F80280C444ACEB03033C334B8023881A
:10F140008B80B1F90230534506DB32F810305B1C7E
:10F1500022F81030A1F8029032F910109F48C06ACE
:10F16000814273DB00235A4601210220F1F794FA11
:10F17000E87986280DD069E03943995502EB4000C3
:10F1800021888180B0F9021051455FD3A0F8029028
:10F190005CE0687A802859D18C48A97980302A7A35
:10F1A000426401EB022141F2707202EB51010164F1
:10F1B000894830F91120002A48DD47F6FF739A424A
:10F1C00044DA41F66D02914240D8A0F2CC439A5DF8
:10F1D0003A4230D000EB4102B4F90030B2F90450A9
:10F1E0009D4203DA568833445B1B5380B2F90450C6
:10F1F000B4F900309D4204DD568833445B1B3C3338
:10F20000538023889380B2F90230534506DB30F8EF
:10F2100011305B1C20F81130A2F8029030F9111067
:10F220006E48C06A814211DB00235A460121022048
:10F23000F1F732FA0AE03A439A5500EB410022888E
:10F2400082809FE76648815DB94381550C20BDE807
:10F25000F08F2DE9F04F83465B48002600EB0B054D
:10F2600037466878102806D1CBF342010120884048
:10F270004FEA1B1687B2554890F83210002977D014
:10F280005349B0F87E00085CC007F8D05846F5F73F
:10F29000B0FDE87A86286AD1697B4E4C4FF4616AEA
:10F2A0004FF00009862969D14848AA7A8030297B25
:10F2B000416402EB01214A08474B026403EB420020
:10F2C00033F91210B0F802C001EB0C41DFF80CC1A9
:10F2D0000029CCF830104ADD6FF0004C614546D073
:10F2E000DFF8FCE01EF806C01CEA070F41D09E467E
:10F2F000B0F906C0B4F900309C4505DAB0F80480D6
:10F300004344A3EB0C038380B0F906C0B4F900308A
:10F310009C4506DDB0F804804344A3EB0C033C336A
:10F320008380B4F800C0A0F806C0B0F904C0D4458A
:10F330000FDBDFF8A8C0491CCCF83010A0F804900F
:10F340004FEAE17C01EB1C4C2EF812104FEA2C41E5
:10F3500041802248D0E90B10814208DC08235A463C
:10F3600001210220F1F798F9E87A862806D0EBE02F
:10F37000E6E04CEA070C0EF806C077E0687B8828C8
:10F380007DD1124AA97A8032287B506401EB00209B
:10F390004FF47A7101EB500141F26C7011648142BB
:10F3A0005FD8DFF834E00EEB41003EF911204388CE
:10F3B00002EB0342094B002A1A6352DD6FF000434F
:10F3C0009A424ED00EE0000000C00308000000206A
:10F3D000521D0020265C00202C2D00200001002062
:10F3E00060280020DFF83CC41CF806303B423AD0CD
:10F3F000B0F906C0B4F900309C4505DAB0F80480D5
:10F400004344A3EB0C038380B0F906C0B4F9003089
:10F410009C4506DDB0F804804344A3EB0C033C3369
:10F4200083802388C380B0F9043053450BDBFE4B47
:10F43000521C1A63A0F80490D31702EB13432EF862
:10F44000112019144180F848D0E90B1081427BDC6F
:10F4500008235A4601210220F1F71EF9E87A86288E
:10F460000DD071E00BE03B430CF806302188C180E1
:10F47000B0F90410514567D3A0F8049064E0687BAC
:10F48000802861D1E848A97A80382A7B426401EB60
:10F49000022141F2707202EB5103036441F66C00E9
:10F4A000834251D8DFF884E30EEB43003EF913109A
:10F4B000428801EB0241DC4A0029116344DD6FF010
:10F4C0000045A94240D0DFF85CC31CF806503D421D
:10F4D00032D0B0F90670B4F90060B74204DAB0F87F
:10F4E00004C06644F61B8680B0F90670B4F900606B
:10F4F000B74205DDB0F804C06644F61B3C36868092
:10F500002488C480B0F9044054450ADB491C1163C7
:10F51000A0F80490CC1701EB14442EF8131021141A
:10F520004180D2E90B0188420EDC08235A460121B2
:10F530000220F1F7B1F807E03D430CF8065095E7DB
:10F54000B848815DB9438155182080E62DE9FC5FFC
:10F550000546B748DFF8D4B24619B64CB07A317BCD
:10F56000012700EB0120B049ABF1E00B80394FF0EF
:10F57000000A01F5B0790864B0F5337F05D0B0F525
:10F58000347F02D0B0F5367F5ED1AB4991F832209E
:10F59000002A6FD0A94AB1F87E10515CC90769D022
:10F5A0002846F5F726FCA0489F498039C06A88653F
:10F5B0000090B07C8864B27A337B02EB0322C1E90D
:10F5C0001023B2F5007F0AD29D4B52080A6453F80B
:10F5D00022C003EB820292880CEB024205E0A2F506
:10F5E000007222F003035BF80320CA658E49DFF83E
:10F5F00044C2803953460A6CACF1180C9646A2F509
:10F600000072C2F38F028A80C1F850A000214A46DE
:10F6100012F80180B8F1010F07D13CF81180A8451C
:10F6200003D18148803807650BE0491C89B206295F
:10F63000EED333B90021535C3BB1491C89B2062992
:10F64000F9D37D48417BB1B197E0DFF8E881009BB9
:10F65000A8F13008022248F82130734B09F80170F4
:10F66000E6332CF811505A54327DDFF8C4C1102A09
:10F670000ED201E06CE02AE0DFE802F008171A1D64
:10F680000A080A0A08171A1D20230A2624F811005E
:10F6900068480C3820F811201CF805307D2BD0D19B
:10F6A00042F0100220F81120CBE700F58070EDE762
:10F6B00000F50070EAE700F54070E7E700F58060CC
:10F6C000E4E700F5A060E1E700F5FA50DEE7BEF5FB
:10F6D000337F08D0BEF5347F05D0BEF5367F4CD1E0
:10F6E000817B01297CD147734FF08048404611F05F
:10F6F000F1FE0121084611F0DCFD524812F008F934
:10F7000050484FF6FF720146A0F800A08280A0F892
:10F7100006A0A0F802A0404611F031FF00231A46CF
:10F720000321404612F097F946481A3012F003F9C7
:10F73000444906201A310881404612F04BF84FF434
:10F7400000414046A8F82410012112F005F914E008
:10F750003549A0F500708039C0F38F0088803549A5
:10F760000020183931F81020AA4202D109F800A06F
:10F7700003E0401C80B20628F4D32B488038006C8C
:10F78000B0F5357F02D0B0F5377F72D12A4991F8B4
:10F790003220002A7ED0294AB1F87E10515CC90778
:10F7A00078D02846F5F725FB1F481F498039C06AE5
:10F7B00088650090B07C8864B27A337B02EB0322C8
:10F7C000C1E91023B2F5007F0BD21D4B52080A6429
:10F7D00053F822C003EB820292880CEB024206E04F
:10F7E0000BE1A2F5007222F003035BF80320CA6567
:10F7F0000D49DFF840C0803953460A6CACF1180C53
:10F800009646A2F50072C2F38F02CA80C1F850A0DA
:10F8100000214A4612F80180B8F1010F19D13CF8D5
:10F82000118011E060280020000100202C2D002014
:10F8300000C003081863002000000020521D0020B3
:10F840003C250020C4030020A84502D1FE480765DE
:10F850000BE0491C89B20629DCD333B90021535C83
:10F8600043B1491C89B20629F9D3F7488038417C55
:10F8700079B392E0DFF8D483009B082248F8213066
:10F8800009F80170F24B2CF81150DFF8C8C35A5434
:10F89000327D00E06CE0102A0BD2DFE802F008179E
:10F8A0001B1E0A080A0A08171B1E21240A2724F80F
:10F8B0001100E648243020F811201CF805307D2B7B
:10F8C000D3D142F0100220F81120CEE700F580706D
:10F8D000EDE70EE000F50070E9E700F54070E6E7BF
:10F8E00000F58060E3E700F5A060E0E700F5FA507E
:10F8F000DDE7BEF5357F05D0BEF5377F4DD1817C84
:10F9000001297AD1DFF850834774404611F0E2FDB7
:10F910000121480311F0C4FCD04811F0F9FFCF4891
:10F920004FF6FF720146A0F800A08280A0F806A062
:10F93000A0F802A0404611F022FE00231A4603213F
:10F94000404612F088F8C5481A3011F0F4FFC34958
:10F9500006201A310881404611F03CFFBE494FF4A1
:10F960000040243108800121404611F0F5FF14E0E9
:10F97000B549A0F50070C0F38F00C880B3490020DE
:10F9800011F1180131F81020AA4202D109F800A0A3
:10F9900003E0401C80B20628F4D3AB48006CB0F5FD
:10F9A000247F5FD1A848803890F8321000297DD09C
:10F9B000AB49B0F87E00085CC00777D02846F5F761
:10F9C00018FAA148A04A8030C06A90658646B07C8B
:10F9D0009064B17A337B01EB0321C2E91013B1F5D6
:10F9E000007F0BD24B089F49136451F823C001EBF1
:10F9F000830189880CEB014106E000E2A1F500716A
:10FA000021F003035BF80310D1658F49DFF83CC296
:10FA100053460A6C0CF1180CA2F50072C2F38F0267
:10FA20000A81C1F850A000214A4600BF12F80180A7
:10FA3000B8F1010F06D13CF81180A84502D18248E7
:10FA400007650BE0491C89B20629EFD333B90021C1
:10FA5000535C43B1491C89B20629F9D37A488038EE
:10FA6000C17C81B381E0DFF8E481794A48F821E084
:10FA700009F801702CF811505754327DDFF8D4C1C9
:10FA8000102A0BD2DFE802F008191C200A080A0A23
:10FA900008191C2023260A2924F811006B48243059
:10FAA00020F811201CF805307D2B00E04BE0D5D16B
:10FAB00042F0100220F81120D0E700F58070EBE74B
:10FAC00000F50070E8E70BE000F54070E4E700F5B2
:10FAD0008060E1E700F5A060DEE700F5FA50DBE7C3
:10FAE000DFF88481C774404611F0F4FC0121C8029C
:10FAF00011F0D6FB594A4FF6FF705346908052489A
:10FB0000A2F800A0A2F806A0018942F20800084469
:10FB1000F0F7FDFCA8B1102050805049404611F08C
:10FB20002EFD00231A461946404611F081FF4FF47E
:10FB30000041404612F009F90121404611F00CFF46
:10FB400013E05380E9E74048242101813F49002028
:10FB500011F1180131F81020AA4202D109F800A0D1
:10FB600003E0401C80B20628F4D33748006CB0F59F
:10FB7000237F05D0B0F5297F02D0B0F52C7F75D159
:10FB80003149803991F83220002A70D0344AB1F8D6
:10FB90007E10515CC9076AD02846F5F72AF92A4831
:10FBA00029498030C06A88650190B07C8864B37A46
:10FBB000327B4A6403EB02220A64B2F5007F0AD268
:10FBC000284B52080A6453F822C003EB8202928841
:10FBD0000CEB024205E0A2F5007222F003035BF891
:10FBE0000320CA651849194BCC460A6C9646A2F503
:10FBF0000072C2F38F028A800092C1F850A00021E7
:10FC0000524618331CF80180B8F1010F06D133F8C1
:10FC10001180A84502D10C48076510E0491C89B243
:10FC20000629EFD35AB900214FEA0C0212F801C09D
:10FC3000BCF1000F1ED0491C89B20629F6D3024838
:10FC40008038B0F8660013E080000020E8620020F1
:10FC5000E601002000C0030800340140C403002076
:10FC6000521D00203C250020002C0140C6E007E189
:10FC700080B31AE1DFF80884DDF804C048F821C039
:10FC8000575423F81150FF4B0222DFF8FCC35A549B
:10FC9000327D102A0BD2DFE802F008171A1E0A087C
:10FCA0000A0A08171A1E21240A2724F81100F4480A
:10FCB000243020F811201CF805307D2BBFD142F0F4
:10FCC000100220F81120BAE700F58070EDE700F58A
:10FCD0000070EAE70BE000F54070E6E700F58060B1
:10FCE000E3E700F5A060E0E700F5FA50DDE7BEF5D8
:10FCF000237F0AD0BEF5297F07D0BEF52C7F7DD1AA
:10FD0000E248B0F86800012879D100984FF0000867
:10FD100042F20801C4460844F0F7F9FB68B1DC4937
:10FD20001020DFF85CE34880D849002080318A88C1
:10FD300019F80010012948D053E0D5490020DFF818
:10FD400040E3A1F802A0D14980318A8819F8001057
:10FD500001290BD15EF820105BF82230994205DBB7
:10FD6000BCF1000F22D0414500D88846401C80B22B
:10FD70000628EBD3BCF1000F40D0C448A0F8667051
:10FD80004FF0804011F0A6FB0121084611F091FAD6
:10FD9000BE4980318A885BF82220A8EB02004FF42C
:10FDA0000048404506D800F5004005E088464FF081
:10FDB000010CDBE74FF6FF70B54A90808882114650
:10FDC000A1F800A0A1F806A03BE05EF820105BF8C7
:10FDD0002230994205DCBCF1000F25D0414500D30B
:10FDE0008846401C80B20628A2D3BCF1000F5CD02C
:10FDF000A648A0F866704FF0804001E055E07CE135
:10FE000011F068FB0121084611F053FA9F48803039
:10FE100082885BF82220A2EB08014FF4004841459C
:10FE200006D8C1F5004104E088464FF0010CD8E740
:10FE30005146974A918081821046A0F800A0A0F810
:10FE400006A093494FF0804011F099FB00231A4619
:10FE500019464FF0804011F0EBFD41464FF08040D5
:10FE600011F073FF0121880711F097FF012211465D
:10FE7000900711F087FD0121880711F06DFD14E056
:10FE80008249A0F500708031C0F38F0088807C49E2
:10FE90000020183131F81020AA4202D109F800A040
:10FEA00003E0401C80B20628F4D378488030006C10
:10FEB000B0F52E7F05D0B0F52F7F02D0B0F5317FA1
:10FEC00060D1724991F83220EAB3724AB1F87E10DB
:10FED000515CC90737D02846F4F78BFF69486B4956
:10FEE000E6388031C06A88650090B07C8864B27A58
:10FEF000337B02EB0322C1E91023B2F5007F0AD263
:10FF0000654B52080A6453F822C003EB82029288C0
:10FF10000CEB024205E0A2F5007222F003035BF84D
:10FF20000320CA65594953468031DFF854C10A6C31
:10FF30009646A2F50072C2F38F028A80C1F850A0E3
:10FF400000214A4600E0C8E00CF1180C12F80180CC
:10FF5000B8F1010F07D13CF81180A84503D14B48F7
:10FF6000803007650BE0491C89B20629EED333B90E
:10FF70000021535C3BB1491C89B20629F9D343489F
:10FF8000C17B79B3BEE0DFF8F880009B3D4A48F8BA
:10FF9000213009F801702CF811505754327DDFF8E8
:10FFA000E8C0102A0BD2DFE802F008171A1E0A0870
:10FFB0000A0A08171A1E21240A2724F811003048BB
:10FFC000243020F811201CF805307D2BD7D142F0C9
:10FFD000100220F81120D2E700F58070EDE700F55F
:10FFE0000070EAE70BE000F54070E6E700F580609E
:10FFF000E3E700F5A060E0E700F5FA50DDE7BEF5C5
:020000040801F1
:100000002E7F08D0BEF52F7F05D0BEF5317F79D188
:10001000017C012971D1C7734FF0804011F05AFA69
:100020000121084611F045F9DFF864804FF6FF70B2
:100030004146A8F80400A8F800A0A8F806A0A8F86F
:1000400002A04FF0804011F09AFA00231A46194698
:100050004FF0804011F0ECFC4FF40041C80311F068
:1000600074FE0121880711F077FC0C4811F032FA78
:100070000121C80211F014F94FF6FF7010E00000E2
:10008000E8620020E601002000C003080000002014
:10009000C4030020521D00203C250020002C0140FC
:1000A000A8F80400A8F800A0A8F806A01020A8F856
:1000B00002004146FE4811F062FA00231A46194632
:1000C000FB4811F0B5FC4FF40041F94811F03DFE3A
:1000D0000121F74811F040FC14E0F649A0F500704A
:1000E000C0F38F008880F449002000BF31F8102051
:1000F000AA4203D109F800A004E032E1401C80B21A
:100100000628F3D3EB48006CB0F5257F05D0B0F599
:100110002A7F02D0B0F52D7F5DD1E649803991F874
:100120003220DAB3E54AB1F87E10515CC90735D008
:100130002846F4F75EFEDF48DE498030C06A8865F5
:100140000090B07C8864B27A337B02EB0322C1E971
:100150001023B2F5007F0AD2D94B52080A6453F833
:1001600022C003EB820292880CEB024205E0A2F56A
:10017000007222F003035BF80320CA65CD495346A1
:10018000DFF834C30A6C9646A2F50072C2F38F0200
:100190004A81C1F850A000214A4600E069E012F807
:1001A0000180B8F1010F06D13CF81180A84502D1B9
:1001B000C04807650BE0491C89B20629EDD333B965
:1001C0000021535C43B1491C89B20629F9D3B948CF
:1001D0008038017D79B360E0DFF8DC82009BA8F114
:1001E0001808072248F82130B64B09F801702CF89E
:1001F00011505A54327DDFF8D0C2102A0BD2DFE8FA
:1002000002F008171B1E0A080A0A08171B1E2124E1
:100210000A2724F81100A8480C3020F811201CF8F7
:1002200005307D2BD3D142F0100220F81120CEE70B
:1002300000F58070EDE70EE000F50070E9E700F5ED
:100240004070E6E700F58060E3E700F5A060E0E7D6
:1002500000F5FA50DDE7BEF5257F08D0BEF52A7F10
:1002600005D0BEF52D7F18D1017E012979D1077502
:1002700013E09049A0F50070C0F38F0048818E49CB
:10028000002000BF31F81020AA4202D109F800A0D6
:1002900003E0401C80B20628F4D38648006CB0F519
:1002A000267F5DD18348803890F83210E9B38349C6
:1002B000B0F87E00085CC00737D02846F4F799FDF7
:1002C0007C487C498030C06A88658646B07C8864FA
:1002D000B37A327B4A6403EB02220A64B2F5007FF0
:1002E0000AD2774B52080A6453F822C003EB820209
:1002F00092880CEB024205E0A2F5007222F00303A3
:100300005BF80320CA656B49DFF8ACC153460A6C41
:10031000A2F50072C2F38F028A81C1F850A00021B9
:100320004A4600BF12F8018000E05BE0B8F1010F1F
:1003300006D13CF81180A84502D15E4807650BE064
:10034000491C89B20629EDD333B90021535C4BB166
:10035000491C89B20629F9D356488038417D79B3C2
:1003600051E03FE2DFF85081564BA8F118082622F1
:1003700048F821E009F801702CF811505A54327DE8
:10038000DFF844C1102A0BD2DFE802F008171B1E69
:100390000A080A0A08171B1E21240A2724F811003C
:1003A00045480C3020F811201CF805307D2BD3D1A6
:1003B00042F0100220F81120CEE700F58070EDE742
:1003C0000EE000F50070E9E700F54070E6E700F5A3
:1003D0008060E3E700F5A060E0E700F5FA50DDE7B4
:1003E000477510E03348262181813349002000BF42
:1003F00031F81020AA4202D109F800A003E0401C05
:1004000080B20628F4D32B48006CB0F5277F02D0C9
:10041000B0F52B7F69D12749803991F83220E2B3BA
:10042000264AB1F87E10515CC90736D02846F4F749
:10043000E0FC20481F498030C06A88658646B07C51
:100440008864B37A327B4A6403EB02220A64B2F511
:10045000007F0AD21A4B52080A6453F822C003EBF9
:10046000820292880CEB024205E0A2F5007222F0B3
:1004700003035BF80320CA650E49DFF83CC053460E
:100480000A6CA2F50072C2F38F02CA81C1F850A0B3
:1004900000214A4612F8018000E065E0B8F1010F42
:1004A00014D13CF81180A84510D10248076519E025
:1004B000002C01408000002000630020521D00201D
:1004C0003C250020E601002000C00308491C89B239
:1004D0000629DFD333B90021535C3BB1491C89B2F3
:1004E0000629F9D3F948817D79B352E0DFF8E0833A
:1004F000F84B272248F821E009F801702CF8115038
:100500005A54327DDFF8D0C3102A0BD2DFE802F054
:1005100008171A1E0A080A0A08171A1E21240A2791
:1005200024F81100EA48243020F811201CF8053086
:100530007D2BD7D142F0100220F81120D2E700F530
:100540008070EDE700F50070EAE70BE000F5407021
:10055000E6E700F58060E3E700F5A060E0E700F57E
:10056000FA50DDE7877514E0D849A0F500708031B6
:10057000C0F38F00C881D6490020183131F810200F
:10058000AA4202D109F800A003E0401C80B206286C
:10059000F4D3CE488030006CB0F5287F5FD1CB48D3
:1005A00090F83210F1B3CD49B0F87E00085CC00776
:1005B00038D02846F4F71DFCC648C449E6388031D7
:1005C000C06A88658646B07C8864B37A327B4A64A8
:1005D00003EB02220A64B2F5007F0AD2C04B520834
:1005E0000A6453F822C003EB820292880CEB0242A9
:1005F00005E0A2F5007222F003035BF80320CA6550
:10060000B249DFF8CCC2803153460A6C0CF1180CA9
:10061000A2F50072C2F38F020A82C1F850A0002135
:100620004A4600E05AE012F80180B8F1010F07D104
:100630003CF81180A84503D1A448803007650BE041
:10064000491C89B20629ECD333B90021535C3BB174
:10065000491C89B20629F9D39C48C17D79B350E081
:10066000DFF86C829B4B282248F821E009F80170E2
:100670002CF811505A54327DDFF85CC2102A0BD28C
:10068000DFE802F008171A1E0A080A0A08171A1EDD
:1006900021240A2724F811008D48243020F8112045
:1006A0001CF805307D2BD7D142F0100220F8112024
:1006B000D2E700F58070EDE700F50070EAE70BE0A7
:1006C00000F54070E6E700F58060E3E700F5A06024
:1006D000E0E700F5FA50DDE7C77512E07B48282116
:1006E000803001827A49002011F1180131F8102080
:1006F000AA4202D109F800A003E0401C80B20628FB
:10070000F4D3DFF8C88108F18008D8F84000B0F5CC
:10071000307F02D0B0F5327F64D16C4991F832203D
:10072000F2B36E4AB1F87E10515CC90738D0284642
:10073000F4F75FFB6748DFF8A0E1E6384146D0F800
:100740002CC0C8F858C0B07CC8F84800B37A327BD7
:10075000C8F8442003EB0222C8F84020B2F5007F1D
:100760000AD25F4B52080A6453F8228003EB8202DC
:10077000928808EB024205E0A2F5007222F0030322
:100780005BF80320CA650A6C8B46A2F50072C2F3BF
:100790008F024A82C1F850A0534600214A4600E029
:1007A0005CE0DFF82C9109F1180900BF12F8018014
:1007B000B8F1010F06D139F81180A84502D1CBF864
:1007C00050700BE0491C89B20629EFD333B90021E0
:1007D000535C43B1491C89B20629F9D33B4890F8D0
:1007E000531071B34FE03A4B43F821C05754394B83
:1007F00029F8115030225A54327D102A0BD2DFE8EA
:1008000002F008171A1D0A080A0A08171A1D2124DF
:100810000A2724F811002E48243020F811201EF851
:1008200005307D2BDAD142F0100220F81120D5E7F7
:1008300000F58070EDE700F50070EAE700F5407024
:10084000E7E708E000F58060E3E700F5A060E0E797
:1008500000F5FA50DDE780F8537014E0A0F5007061
:10086000C0F38F00A8F812001949002011F11801F7
:1008700031F81020AA4202D109F800A003E0401C80
:1008800080B20628F4D31820BDE8FC9F70B504465A
:100890001148002120440A464578102D05D1210930
:1008A000C4F342020120904082B2084B0D4893F8F5
:1008B0003260A6B3094EB3F87E30F35CDB072FD06D
:1008C000435C134210D09DB12FE0000000000020D7
:1008D000E8620020E601002000C00308521D00204D
:1008E0003C25002060280020102D01D113434354E3
:1008F0002046F4F77EFAFE4DA5F18006E86AB06561
:1009000004F1080080B2F4F774FAE86AF065B16D9A
:1009100010340844E862A0B2F6F744FB05E0FFE7B4
:10092000102D02D1435C93434354182070BD70B521
:100930000446F048002120440A464578102D05D190
:100940002109C4F342020120904082B2EA4BEB48F5
:1009500093F8326036B3B3F87E30A0F60E36F35C0F
:10096000DB071FD0435C134201D025B11FE0102DDF
:1009700001D1134343542046F4F73BFADC4DA5F173
:100980008006E86AB06504F1080080B2F4F731FA35
:10099000E86AF065B16D1034081AE862A0B2F6F7A3
:1009A00001FB04E0102D02D1435C93434354182013
:1009B00070BD2DE9F0410446CE48002120440A468E
:1009C0004678102E05D12109C4F34202012090403F
:1009D00082B2C94DC94895F8323043B3B5F87E703C
:1009E000A0F60E33DB5DDB0721D0435C134201D060
:1009F00026B121E0102E01D1134343543D2005F8C8
:100A0000590F2046F4F7F5F9B94EA6F18007F06AC0
:100A1000B86504F1080080B2F4F7EBF9F06A10341D
:100A2000F865A0B2F6F7BEFA0020287004E0102E98
:100A300002D1435C934343541820BDE8F0812DE973
:100A4000F0410446AB48002120440A464678102E67
:100A500005D12109C4F342020120904082B2A64D83
:100A6000A64895F8323053B3B5F87E70A0F60E3331
:100A7000DB5DDB0723D0435C134201D026B123E0CA
:100A8000102E01D1134343543F2085F859002046CE
:100A9000F4F7AFF9964FA7F18006F86AB06504F154
:100AA000080080B2F4F7A5F9F86AF06518B11034BF
:100AB000A0B2F6F777FA002085F8590004E0102E6E
:100AC00002D1435C934343541820B6E7F0B5044683
:100AD0008848002105190A466E78102E05D1210993
:100AE000C4F342020120904082B2834B834893F8C2
:100AF000327057B3B3F87E30A0F60E37FB5CDB07DD
:100B000023D0435C134201D026B123E0102E01D143
:100B1000134343542046F4F76CF9754FA7F1800650
:100B2000F86AB06504F1080080B2F4F762F9F96A76
:100B3000F165E87C84280DD1687D80280AD10823DE
:100B40002246B06DEFF7A8FD04E0102E02D1435C01
:100B5000934343541820F0BDF8B50446654800217E
:100B600006190A467578102D05D12109C4F34202F1
:100B70000120904082B2604B604893F832709FB37E
:100B8000B3F87E30A0F60E37FB5CDB072DD0435C5C
:100B9000134201D025B12DE0102D01D11343435450
:100BA0002046F4F726F9524FA7F18005F86AA865A8
:100BB00004F1080080B2F4F71CF9F86AE86504F162
:100BC000100080B2F4F715F9FA6A2A66F07E8428DC
:100BD00010D1707F80280DD10C200090D5E916012E
:100BE0002346EFF7D1FE05E0FFE7102D02D1435C6D
:100BF000934343542020F8BD70B50546F3F773FBCB
:100C00003B4E2D1DA6F18004F06A6066A8B2F3F792
:100C10006AFBF06AA066626E3749824201D1012008
:100C200000E0002081F83200082070BD70B5054654
:100C3000F4F7DFF82E4E083506F18004F06AA06163
:100C4000A8B2F4F7D6F8F06AE061A2692A498242B4
:100C500001D1012000E0002081F83200102070BD99
:100C600070B50546F4F7C5F8214E083506F1800445
:100C7000F06AA061A8B2F4F7BCF8F06AE061A2697A
:100C80001D49824201DD012000E0002081F8320090
:100C9000102070BD70B50546F4F7ABF8144E08355A
:100CA00006F18004F06AA061A8B2F4F7A2F8F06A35
:100CB000E061A2691049824201DA012000E00020CF
:100CC00081F83200102070BD70B50546F4F791F838
:100CD000074E083506F18004F06AA061A8B2F4F767
:100CE00088F8F06AE061A269034982420AD007E00D
:100CF0000001002000C00308000000206028002040
:100D0000012000E0002081F83200102070BD70B595
:100D10000546F4F76EF8FE4E083506F18004F06AD9
:100D2000A061A8B2F4F765F8F06AE061A269A4F5E1
:100D3000C071824201DB012000E0002081F8320016
:100D4000102070BD70B50546F4F753F8F04E083525
:100D500006F18004F06AA061A8B2F4F74AF8F06ADC
:100D6000E061A269A4F5C071824201DC012000E0CB
:100D7000002081F83200102070BD70B50546F4F7F0
:100D800038F8E34E083506F18004F06AA061A8B295
:100D9000F4F72FF8F16AE161A3690022A4F5C070AD
:100DA0008B4206D190F8321029B1012180F832101F
:100DB00001E080F83220102070BD70B50546F4F7D0
:100DC00018F8D34E083506F18004F06AA061A8B285
:100DD000F4F70FF8F16AE161A3690022A4F5C0708D
:100DE0008B4206DD90F8321029B1012180F83210D3
:100DF00001E080F83220102070BD70B50546F3F791
:100E0000F8FFC34E083506F18004F06AA061A8B26D
:100E1000F3F7EFFFF16AE161A3690022A4F5C07066
:100E20008B4206DA90F8321029B1012180F8321095
:100E300001E080F83220102070BD70B50546F3F750
:100E4000D8FFB34E083506F18004F06AA061A8B25D
:100E5000F3F7CFFFF16AE161A3690022A4F5C07046
:100E60008B4206D090F8321029B1012180F832105F
:100E700001E080F83220102070BD70B50546F3F710
:100E8000B8FFA34E083506F18004F06AA061A8B24D
:100E9000F3F7AFFFF16AE161A3690022A4F5C07026
:100EA0008B4206DB90F8321029B1012180F8321014
:100EB00001E080F83220102070BD70B50546F3F7D0
:100EC00098FF934E083506F18004F06AA061A8B23D
:100ED000F3F78FFFF16AE161A3690022A4F5C07006
:100EE0008B4206DC90F8321029B1012180F83210D3
:100EF00001E080F83220102070BD70B50546F3F790
:100F000078FF834E083506F18004F06AA061A8B22C
:100F1000F3F76FFFF06AE061A269A4F5C071824245
:100F200002D091F8320010B1012081F83200102077
:100F300070BD70B50546F3F75CFF754E083506F1D8
:100F40008004F06AA061A8B2F3F753FFF06AE06191
:100F5000A269A4F5C071824202DC91F8320010B19E
:100F6000012081F83200102070BD70B50546F3F7FE
:100F700040FF674E083506F18004F06AA061A8B210
:100F8000F3F737FFF06AE061A269A4F5C07182420D
:100F900002DB91F8320010B1012081F832001020FC
:100FA00070BD70B50546F3F724FF594E083506F1BC
:100FB0008004F06AA061A8B2F3F71BFFF06AE06159
:100FC000A269A4F5C071824202D191F8320010B139
:100FD000012081F83200102070BD70B50546F3F78E
:100FE00008FF4B4E083506F18004F06AA061A8B2F4
:100FF000F3F7FFFEF06AE061A269A4F5C0718242D6
:1010000002DA91F8320010B1012081F8320010208C
:1010100070BD70B50546F3F7ECFE3D4E083506F1A0
:101020008004F06AA061A8B2F3F7E3FEF06AE06121
:10103000A269A4F5C071824202DD91F8320010B1BC
:10104000012081F83200102070BD70B50546F3F71D
:101050004AF92F4E2D1DA6F18004F06A6066A8B2F1
:10106000F3F741F9F06AA066626EA4F18001824252
:1010700001DD012000E0002081F83200082070BD71
:1010800070B50546F3F72FF9214E2D1DA6F180040A
:10109000F06A6066A8B2F3F726F9F06AA066626E9D
:1010A000A4F18001824201DA012000E0002081F8F1
:1010B0003200082070BD70B50546F3F714F9144EE0
:1010C0002D1DA6F18004F06A6066A8B2F3F70BF953
:1010D000F06AA066626EA4F18001824201D0012014
:1010E00000E0002081F83200082070BD70B5054690
:1010F000F3F7F9F8064E2D1DA6F18004F06A60663C
:10110000A8B2F3F7F0F8F06AA066A4F1800101E05C
:1011100000010020626E824201DB012000E000201D
:1011200081F83200082070BD70B50546F3F7DBF892
:10113000FB4E2D1DA6F18004F06A6066A8B2F3F79D
:10114000D2F8F06AA066626EA4F18001824201DCEE
:10115000012000E0002081F83200082070BD70B549
:101160000546F3F7C0F8EE4E2D1DA6F18004F06A97
:101170006066A8B2F3F7B7F8F16AA166636E002261
:10118000A4F180008B4206D190F8321029B10121E0
:1011900080F8321001E080F83220082070BD70B570
:1011A0000546F3F7A0F8DE4E2D1DA6F18004F06A87
:1011B0006066A8B2F3F797F8F16AA166636E002241
:1011C000A4F180008B4206DD90F8321029B1012194
:1011D00080F8321001E080F83220082070BD70B530
:1011E0000546F3F780F8CE4E2D1DA6F18004F06A77
:1011F0006066A8B2F3F777F8F16AA166636E002221
:10120000A4F180008B4206DA90F8321029B1012156
:1012100080F8321001E080F83220082070BD70B5EF
:101220000546F3F760F8BE4E2D1DA6F18004F06A66
:101230006066A8B2F3F757F8F16AA166636E002200
:10124000A4F180008B4206D090F8321029B1012120
:1012500080F8321001E080F83220082070BD70B5AF
:101260000546F3F740F8AE4E2D1DA6F18004F06A56
:101270006066A8B2F3F737F8F16AA166636E0022E0
:10128000A4F180008B4206DB90F8321029B10121D5
:1012900080F8321001E080F83220082070BD70B56F
:1012A0000546F3F720F89E4E2D1DA6F18004F06A46
:1012B0006066A8B2F3F717F8F16AA166636E0022C0
:1012C000A4F180008B4206DC90F8321029B1012194
:1012D00080F8321001E080F83220082070BD70B52F
:1012E0000546F3F700F88E4E2D1DA6F18004F06A36
:1012F0006066A8B2F2F7F7FFF06AA066626EA4F12A
:101300008001824202D091F8320010B1012081F8B0
:101310003200082070BD70B50546F2F7E4FF804E3C
:101320002D1DA6F18004F06A6066A8B2F2F7DBFF1B
:10133000F06AA066626EA4F18001824202DC91F83C
:10134000320010B1012081F83200082070BD70B564
:101350000546F2F7C8FF724E2D1DA6F18004F06A13
:101360006066A8B2F2F7BFFFF06AA066626EA4F1F1
:101370008001824202DB91F8320010B1012081F835
:101380003200082070BD70B50546F2F7ACFF644E20
:101390002D1DA6F18004F06A6066A8B2F2F7A3FFE3
:1013A000F06AA066626EA4F18001824202D191F8D7
:1013B000320010B1012081F83200082070BD70B5F4
:1013C0000546F2F790FF564E2D1DA6F18004F06AF7
:1013D0006066A8B2F2F787FFF06AA066626EA4F1B9
:1013E0008001824202DA91F8320010B1012081F8C6
:1013F0003200082070BD70B50546F2F774FF484E04
:101400002D1DA6F18004F06A6066A8B2F2F76BFFAA
:10141000F06AA066626EA4F18001824202DD91F85A
:10142000320010B1012081F83200082070BD2DE992
:10143000F04F83460309C0F342010120884081B286
:101440003848DFF8EC804FEA1B1290F832C0DFF822
:10145000D8A0DFF8E090354F18F8020010268FB0C2
:101460000AF6C94509EB0B04BCF1000F68D0DFF8A0
:10147000B4C005F6E142BCF87EC012F80C20D207D9
:10148000F4D0084308F80300A27A5046805C002894
:101490006FD105F6E14000F580710B9100F5007108
:1014A00000F54070CDE9090105F2E120089000F552
:1014B0008070079000F58070019000F580700390B7
:1014C00000F5807005900BF10400DFF86C900C9033
:1014D0001A4809F1040A0490002A75D1DFF8448003
:1014E00098F80800C007D3D15846F2F7FCFE11481F
:1014F00010F80B10114808384E2906D10849B0F9E8
:101500000020CB6AA3EB0202CA62B0F900100448C3
:101510008160C06A010414D401498039C86615E0AD
:101520000001002000000020A8030020001001405E
:101530006028002000C00308101401402C5D00202A
:10154000FEE3411EFF4AC94389B2D166217C41B105
:1015500001290FD0022915D003291BD0052921D03C
:10156000F5E0000401D4012100E00021A27BF6484F
:1015700003E1ACE2000401D4012100E00021A27BE0
:101580000B981BE1000401D4012100E00021A27BA3
:101590000A9813E1000401D4012100E00021A27B9C
:1015A00009980BE1020401D4012200E00022A37B90
:1015B000EA54A27BE54B182A15F802C003F802C0D2
:1015C00088F85B206FD200E016E2DFE802F00C132F
:1015D00019292F383E454A52595F656F787F858BB0
:1015E000959AA0A9B0B6287800284FF004000FD033
:1015F000D7490860687800284FF480700BD0786174
:10160000A87800284FF4004007D0D1490860EAE0EC
:10161000CF49091FEDE73861F2E7CD49091FF5E72A
:10162000E87800284FF4806005D006E0287900288B
:101630004FF4006001D13861D5E07861D3E068797A
:1016400000284FF48050F8D1F5E7A8794FF0010158
:1016500058B10CE00160C6E0E8794FF0020120B11A
:1016600005E0287A4FF0080108B94846F2E75046ED
:10167000F0E7687A10B150460660B4E04846FBE7F0
:10168000A87A00284FF020000BD00DE0E87A00285F
:101690004FF0400005D007E0287B00284FF0800085
:1016A00002D14946B2E752E05146AFE7687B4FF0BE
:1016B000080108B1A748CDE7A648001FCAE7A87BE4
:1016C00008B1A448D8E7A348001FD5E7E87B002865
:1016D0004FF020000BD00DE0287C00284FF0400098
:1016E00005D007E0687C00284FF0800002D19949BE
:1016F000091F8BE7974989E7A87C4FF0020150B199
:101700000BE0E87C00284FF004001BD01CE0287D93
:101710004FF0080108B990489CE78F48001D99E7F1
:10172000687D10B18C48001DA6E78B48A4E7A87D12
:1017300000284FF0200005D006E0E87D00284FF09B
:10174000400001D1844961E78349091D5EE708290A
:101750000CD0092913D00A2919D00B291FD00C2924
:1017600025D00D292CD00F2932D03CE0000401D423
:10177000012100E00021A27B7848815433E000047D
:1017800001D4012100E00021A27B089816E00004AA
:1017900001D4012100E00021A27B07980EE00004A3
:1017A00001D4012100E00021A27B019806E00004A1
:1017B00001D4012100E00021A27B0398115412E022
:1017C000000401D4012100E00021A27B0598F5E787
:1017D00000040028A07B00F5FA5001DB012100E0A5
:1017E0000021EEF7A1FEA27A5D49012088545549F7
:1017F0008039C8725B490020487752488030C16AFE
:101800000A0405D4A0F58073012283F8572004E070
:101810004C4A0223803A82F85730804621B9494920
:101820000020803981F857000C9880B2F2F75BFDF8
:10183000444AD8F82C1002F5807E0A23CEF84010D6
:1018400091FBF3F11167D2F86CC0CEF848C0049850
:101850006423B0F90800322804DB41F2883840459F
:1018600000DC03464048DFF8DCE003654FF090639E
:1018700093FBF1F24FEAE27802EB18421214026392
:10188000521C514393FBF1F0401ECEF87000BCF1A6
:10189000000F3CDD35480FF01DFE012108200FF040
:1018A00008FD284818217830C17002218170042178
:1018B00001800146264814380FF08FF921484FF077
:1018C0000008B0F8701026481C3081802649098E27
:1018D0000180A0F806804680014624480FF04FFEA4
:1018E0001F48602126300180012141801549096F80
:1018F00001EBD171C1F34F01C180A0F8088001460E
:101900001A480FF0BDFE0821184810F016F90D4BCB
:1019100017494FF00008D86E088013490028C1F815
:1019200020808864A1F5C07181F827605EDD012800
:101930004EDD012102200FF0BCFC0248B0F86C1013
:10194000491E17E080000020521D0020C110002019
:1019500014080140140C01401018014052120020DC
:10196000A80300205218002080010020000C004035
:10197000705C0020FE488180A0F80080A0F80680FE
:10198000A0F802800146FB480FF0F9FD00231A463B
:101990001946F84810F04CF80021F64810F0D5F937
:1019A0000121F44810F0F9F901221146F1480FF035
:1019B000E9FF0121EF480FF0CFFFEF48012100F5CB
:1019C000C0720177C2F8588080F85F8080F85D802F
:1019D00001220421E9480FF0D5FF0121E7480FF06B
:1019E000BBFF012141F6D370EEF79EFDE048A17ADE
:1019F0001C38405C00286AD1A07A0128FBD1DFF8AE
:101A0000788398F80800800761D45846F2F76BFC99
:101A1000DB4810F80B10DB484E2907D108F5807120
:101A2000B0F90020CB6AA3EB0202CA62DFF858B318
:101A3000B0F90010CBF80C10DBF82C00010403D433
:101A4000ABF18001C86605E0411ECB4AC943803234
:101A500089B2D166217C41B101290ED0022914D06E
:101A600003291AD0052920D0F2E0000401D4012175
:101A700000E00021A27BC54800E1000401D401215F
:101A800000E00021A27B0B9819E1000401D40121A0
:101A900000E00021A27B0A9811E1000401D4012199
:101AA00000E00021A27B099809E1020401D401228F
:101AB00000E00022A37BEA54A27BB54B182A15F85C
:101AC00002C003F802C088F85C206FD200E044E254
:101AD000DFE802F00C1319292F383E454A52595FAE
:101AE000656F787F858B959AA1A8AFB52878002877
:101AF0004FF004000FD0A7490860687800284FF421
:101B000080700BD07861A87800284FF4004007D08F
:101B1000A0490860E8E09F49091FEDE73861F2E756
:101B20009C49091FF5E7E87800284FF4806005D04C
:101B300006E0287900284FF4006001D13861D3E035
:101B40007861D1E0687900284FF48050F8D1F5E74A
:101B5000A8794FF0010158B10CE00160C4E0E879C8
:101B60004FF0020120B105E0287A4FF0080108B9D2
:101B70004846F2E75046F0E7687A10B150460660F2
:101B8000B2E04846FBE7A87A00284FF020000BD0CF
:101B90000DE0E87A00284FF0400005D007E0287BF0
:101BA00000284FF0800002D14946B2E750E051468C
:101BB000AFE7687B4FF0080108B17748CDE776487A
:101BC000001FCAE7A87B08B17348D8E77248001F16
:101BD000D5E7E87B00284FF020000BD00DE0287CF3
:101BE00000284FF0400005D007E0687C00284FF047
:101BF000800002D16849091F8BE7674989E7A87C03
